S01D00006963655F69637265616D5F736F64615F626F6172642E7372656399
S3150802000000000A20711A0408E10E0408E90E040821
S31508020010F10E0408F90E0408010F0408C11A0408AF
S31508020020000000000000000000000000C11A0408D9
S31508020030090F04080000000041030208E102020851
S31508020040C11A0408C11A0408C11A0408C11A040804
S31508020050C11A0408C11A0408C11A0408C11A0408F4
S31508020060C11A0408C11A0408C11A0408170F040899
S31508020070C11A0408C11A0408C11A0408C11A0408D4
S31508020080C11A0408C11A0408C11A0408C11A0408C4
S31508020090C11A0408C11A0408C11A0408C11A0408B4
S315080200A0250F0408C11A0408C11A0408C11A04084B
S315080200B0350F0408C11A0408C11A0408C11A04082B
S315080200C0C11A0408C11A0408C11A0408C11A040884
S315080200D000000000C11A0408C11A0408490F0408DE
S315080200E0C11A0408C11A0408C11A0408C11A040864
S315080200F0C11A0408C11A0408C11A0408C11A040854
S31508020100C11A04085D0F0408C11A0408C11A0408B2
S31508020110C11A0408C11A0408C11A0408C11A040833
S31508020120C11A0408C11A0408710F0408C11A04087E
S31508020130C11A0408C11A0408850F0408C11A04085A
S31508020140C11A0408C11A0408C11A0408C11A040803
S31508020150C11A0408C11A0408C11A0408C11A0408F3
S31508020160C11A0408C11A0408C11A0408C11A0408E3
S31508020170C11A0408C11A0408C11A0408C11A0408D3
S31508020180C11A0408C11A0408C11A0408C11A0408C3
S31508020190C11A0408C11A0408C11A0408C11A0408B3
S315080201A0C11A0408C11A0408C11A0408C11A0408A3
S315080201B0C11A0408C11A0408C11A0408C11A040893
S315080201C0C11A0408C11A0408990F0408C11A0408B6
S315080201D0C11A0408C11A040800000000C11A04085A
S315080201E0C11A0408C11A0408000000000000000031
S315080201F0C11A04080000000000000000C11A040821
S31508020200C11A0408C11A0408C11A04080000000029
S3150802021000000000C11A040800000000C11A040800
S31508020220C11A0408C11A0408C11A0408C11A040822
S31508020230C11A0408C11A0408C11A0408C11A040812
S31508020240C11A0408C11A0408C11A040800000000E9
S3150802025010B5054C237833B9044B13B10448AFF3F0
S3150802026000800123237010BDA805002000000000AD
S315080202701CBF050808B5034B1BB103490348AFF376
S31508020280008008BD00000000AC0500201CBF050860
S3150802029072B64FF0E0201749C0F8081D16480168E3
S315080202A041F00101016015481249096801604FF0E1
S315080202B0E020134941614FF0070101614FF0000147
S315080202C0C0F8181D4FF07F41C0F81C1D0D49C0F833
S315080202D0201D7047FFF7FEBF01B5BDE80140704714
S315080202E001B500F09DF8BDE801407047FFF7FEBF73
S315080202F0FFF7FEBF00000208001000E0C828012030
S315080203008FD003000000FF40EFF3108180F31088BE
S31508020310081C70474FF000002D4A1060EFF3148056
S3150802032020F0040080F3148862B64FF080504FF034
S31508020330E021C1F8040DBFF34F8FBFF36F8FFEE7BD
S315080203402448254A4FF00003016891B10360EFF390
S31508020350098C2CE9F00F1EF0100F01D12CED108A32
S315080203601E4C4CF804EDC1F808C025680DB18D6124
S31508020370236072B61168D1B1016062B64F68174C34
S315080203808D6907F101074F602560D1F80CC08CF31F
S315080203900B88D1F808C05CF804EB1EF0100F01D1E7
S315080203A0BCEC108ABCE8F00F8CF30988704772B669
S315080203B01168016009B962B6F9E74FF000674FF0B4
S315080203C0E028C8F8047D62B6D8E700BF7047000087
S315080203D064290120CC280120D0280120D02E012012
S315080203E0026922F00702A2F144026FF04303136086
S315080203F04FF0000353609360D360136153619361B6
S31508020400D361136253629362D362136353634FF0E9
S31508020410FF339363D1634FF080731364826070472E
S315080204202249086800F101000860214B1A683AB1AE
S31508020430A2F101021A601AB91E4B4FF001001860A8
S315080204401D490868026822B11C4B4FF001021A6066
S3150802045008E000F104001A4B1A68904201D1194BC0
S3150802046018680860134B1A6812B914490868C8B1A3
S3150802047001B51249086808B131F08CFF0D4B1A68AC
S3150802048072B131F0F9FE1048016849B90F4801689E
S315080204900F4A13680F484FF08052994200D0026003
S315080204A0BDE80140BFF34F8F704700007029012055
S315080204B0D02E012074290120002A0120042A0120B5
S315080204C0FC290120F829012064290120CC280120D1
S315080204D0D028012004ED00E0034613F8012B002A78
S315080204E0FBD1181A0138704781F0004102E000BFBB
S315080204F083F0004330B54FEA41044FEA430594EAD4
S31508020500050F08BF90EA020F1FBF54EA000C55EA0E
S31508020510020C7FEA645C7FEA655C00F0E2804FEADF
S315080205205454D4EB5555B8BF6D420CDD2C4480EAC1
S31508020530020281EA030382EA000083EA010180EAF1
S31508020540020281EA0303362D88BF30BD11F0004F3F
S315080205504FEA01314FF4801C4CEA113102D0404275
S3150802056061EB410113F0004F4FEA03334CEA1333B0
S3150802057002D0524263EB430394EA050F00F0A780C8
S31508020580A4F10104D5F1200E0DDB02FA0EFC22FAC3
S3150802059005F2801841F1000103FA0EF2801843FAB7
S315080205A005F359410EE0A5F120050EF1200E012AA8
S315080205B003FA0EFC28BF4CF0020C43FA05F3C018E6
S315080205C051EBE37101F0004507D54FF0000EDCF15F
S315080205D0000C7EEB00006EEB0101B1F5801F1BD308
S315080205E0B1F5001F0CD349085FEA30004FEA3C0C0C
S315080205F004F101044FEA445212F5800F80F09A8002
S31508020600BCF1004F08BF5FEA500C50F1000041EB05
S31508020610045141EA050130BD5FEA4C0C404141EB09
S315080206200101013C28BFB1F5801FE9D291F0000F04
S3150802063004BF01460020B1FA81F308BF2033A3F1B3
S315080206400B03B3F120020CDA0C3208DD02F1140CAA
S31508020650C2F10C0201FA0CF021FA02F10CE002F1E5
S315080206601402D8BFC2F1200C01FA02F120FA0CFCDE
S31508020670DCBF41EA0C019040E41AA2BF01EB045127
S31508020680294330BD6FEA04041F3C1CDA0C340EDC25
S3150802069004F11404C4F1200220FA04F001FA02F368
S315080206A040EA030021FA04F345EA030130BDC4F126
S315080206B00C04C4F1200220FA02F001FA04F340EA1B
S315080206C00300294630BD21FA04F0294630BD94F0CC
S315080206D0000F83F4801306BF81F480110134013DB3
S315080206E04EE77FEA645C18BF7FEA655C29D094EA24
S315080206F0050F08BF90EA020F05D054EA000C04BFA2
S315080207001946104630BD91EA030F1EBF002100208C
S3150802071030BD5FEA545C05D14000494128BF41F02B
S31508020720004130BD14F580043CBF01F5801130BD8F
S3150802073001F0004545F0FE4141F470014FF000001A
S3150802074030BD7FEA645C1ABF194610467FEA655CCB
S315080207501CBF0B46024650EA013406BF52EA03356D
S3150802076091EA030F41F4002130BD00BF90F0000F5B
S3150802077004BF0021704730B54FF4806404F1320497
S315080207804FF000054FF0000150E700BF90F0000F50
S3150802079004BF0021704730B54FF4806404F1320477
S315080207A010F0004548BF40424FF000013EE700BF47
S315080207B042004FEAE2014FEA31014FEA02701FBFD7
S315080207C012F07F4393F07F4F81F06051704732F009
S315080207D07F4208BF704793F07F4F04BF41F4002160
S315080207E0704730B54FF4607401F0004521F00041BE
S315080207F01CE700BF50EA010208BF704730B54FF048
S3150802080000050AE050EA010208BF704730B511F048
S31508020810004502D5404261EB41014FF4806404F180
S3150802082032045FEA915C3FF4D8AE4FF003025FEA06
S31508020830DC0C18BF03325FEADC0C18BF033202EB8A
S31508020840DC02C2F1200300FA03FC20FA02F001FAE4
S3150802085003FE40EA0E0021FA02F11444BDE600BF87
S3150802086070B54FF0FF0C4CF4E06C1CEA11541DBF36
S315080208701CEA135594EA0C0F95EA0C0F00F0DEF801
S315080208802C4481EA030621EA4C5123EA4C5350EAE6
S31508020890013518BF52EA033541F4801143F4801337
S315080208A038D0A0FB02CE4FF00005E1FB02E506F0C8
S315080208B00042E0FB03E54FF00006E1FB03569CF01D
S315080208C0000F18BF4EF0010EA4F1FF04B6F5007F23
S315080208D064F5407404D25FEA4E0E6D4146EB060695
S315080208E042EAC62141EA55514FEAC52040EA5E501E
S315080208F04FEACE2EB4F1FD0C88BFBCF5E06F1ED8C8
S31508020900BEF1004F08BF5FEA500E50F1000041EBFE
S31508020910045170BD06F0004646EA010140EA0200AB
S3150802092081EA0301B4EB5C04C2BFD4EB0C0541EACD
S31508020930045170BD41F480114FF0000E013C00F3E2
S31508020940AB8014F1360FDEBF002001F0004170BD06
S31508020950C4F10004203C35DA0C341BDC04F114041F
S31508020960C4F1200500FA05F320FA04F001FA05F2AB
S3150802097040EA020001F0004221F0004110EBD37078
S3150802098021FA04F642EB06015EEA430E08BF20EAA4
S31508020990D37070BDC4F10C04C4F1200500FA04F347
S315080209A020FA05F001FA04F240EA020001F00041D9
S315080209B010EBD37041F100015EEA430E08BF20EA4C
S315080209C0D37070BDC4F1200500FA05F24EEA020E94
S315080209D020FA04F301FA05F243EA020321FA04F0C3
S315080209E001F0004121FA04F220EA020000EBD3707A
S315080209F05EEA430E08BF20EAD37070BD94F0000F7A
S31508020A000FD101F00046400041EB010111F4801FAD
S31508020A1008BF013CF7D041EA060195F0000F18BF5E
S31508020A20704703F00046520043EB030313F4801F9A
S31508020A3008BF013DF7D043EA0603704794EA0C0F54
S31508020A400CEA135518BF95EA0C0F0CD050EA41066A
S31508020A5018BF52EA4306D1D181EA030101F00041E7
S31508020A604FF0000070BD50EA410606BF104619460F
S31508020A7052EA430619D094EA0C0F02D150EA01361B
S31508020A8013D195EA0C0F05D152EA03361CBF10465C
S31508020A9019460AD181EA030101F0004141F0FE41FB
S31508020AA041F470014FF0000070BD41F0FE4141F47F
S31508020AB0780170BD70B54FF0FF0C4CF4E06C1CEA7F
S31508020AC011541DBF1CEA135594EA0C0F95EA0C0F34
S31508020AD000F0A7F8A4EB050481EA030E52EA0335EF
S31508020AE04FEA013100F088804FEA03334FF0805510
S31508020AF045EA131343EA12634FEA022245EA11153D
S31508020B0045EA10654FEA00260EF000419D4208BFED
S31508020B10964244F1FD0404F5407402D25B084FEA9A
S31508020B203202B61A65EB03055B084FEA32024FF446
S31508020B3080104FF4002CB6EB020E75EB030E22BFA3
S31508020B40B61A754640EA0C005B084FEA3202B6EB63
S31508020B50020E75EB030E22BFB61A754640EA5C0012
S31508020B605B084FEA3202B6EB020E75EB030E22BFA2
S31508020B70B61A754640EA9C005B084FEA3202B6EBA3
S31508020B80020E75EB030E22BFB61A754640EADC0062
S31508020B9055EA060E18D04FEA051545EA16754FEAC4
S31508020BA006164FEAC30343EA52734FEAC2025FEAE2
S31508020BB01C1CC0D111F4801F0BD141EA00014FF071
S31508020BC000004FF0004CB6E711F4801F04BF014342
S31508020BD00020B4F1FD0C88BFBCF5E06F3FF6AFAE5E
S31508020BE0B5EB030C04BFB6EB020C5FEA500C50F1EE
S31508020BF0000041EB045170BD0EF0004E4EEA113171
S31508020C0014EB5C04C2BFD4EB0C0541EA045170BD77
S31508020C1041F480114FF0000E013C90E645EA060EBB
S31508020C208DE60CEA135594EA0C0F08BF95EA0C0FE9
S31508020C303FF43BAF94EA0C0F0AD150EA01347FF431
S31508020C4034AF95EA0C0F7FF425AF104619462CE708
S31508020C5095EA0C0F06D152EA03353FF4FDAE10466B
S31508020C60194622E750EA410618BF52EA43067FF4BC
S31508020C70C5AE50EA41047FF40DAF52EA43057FF44C
S31508020C80EBAE12E74FF0FF3C06E000BF4FF0010C57
S31508020C9002E000BF4FF0010C4DF804CD4FEA410CBB
S31508020CA07FEA6C5C4FEA430C18BF7FEA6C5C1BD088
S31508020CB001B050EA410C0CBF52EA430C91EA030F09
S31508020CC002BF90EA020F0020704710F1000F91EA66
S31508020CD0030F58BF994208BF90422CBFD8176FEA34
S31508020CE0E37040F0010070474FEA410C7FEA6C5C02
S31508020CF002D150EA013C07D14FEA430C7FEA6C5C09
S31508020D00D6D152EA033CD3D05DF8040B704700BF34
S31508020D108446104662468C461946634600E000BF82
S31508020D2001B5FFF7B7FF002848BF10F1000F01BD54
S31508020D304DF808EDFFF7F4FF0CBF012000205DF81F
S31508020D4008FB00BF4DF808EDFFF7EAFF34BF0120A4
S31508020D5000205DF808FB00BF4DF808EDFFF7E0FF3D
S31508020D6094BF012000205DF808FB00BF4DF808ED8E
S31508020D70FFF7CEFF94BF012000205DF808FB00BFF5
S31508020D804DF808EDFFF7C4FF34BF012000205DF8D7
S31508020D9008FB00BF4FEA410C7FEA6C5C02D150EABD
S31508020DA0013C0AD14FEA430C7FEA6C5C02D152EA53
S31508020DB0033C02D14FF0000070474FF00100704724
S31508020DC04FEA410212F5001215D211D56FF4787363
S31508020DD0B3EB625212D94FEAC12343F0004343EA06
S31508020DE0505311F0004F23FA02F018BF40427047E1
S31508020DF04FF00000704750EA013005D111F000406B
S31508020E0008BF6FF0004070474FF00000704700BF00
S31508020E104A0011D212F5001211D20DD56FF4787369
S31508020E20B3EB62520ED44FEAC12343F0004343EABE
S31508020E30505323FA02F070474FF00000704750EA09
S31508020E40013002D14FF0FF3070474FF00000704773
S31508020E504FEA4102B2F1E04324BFB3F5001CDCF1CC
S31508020E60FE5C0DD901F0004C4FEAC0024CEA507004
S31508020E70B2F1004F40EB830008BF20F00100704733
S31508020E8011F0804F21D113F13872BCBF01F0004036
S31508020E90704741F480114FEA5252C2F11802C2F168
S31508020EA0200C10FA0CF320FA02F018BF40F00100E9
S31508020EB04FEAC1234FEAD32303FA0CFC40EA0C009B
S31508020EC023FA02F34FEA4303CCE77FEA625307D1D8
S31508020ED050EA01331EBF4FF0FE4040F4400070470F
S31508020EE001F0004040F0FE4040F40000704700BFA9
S31508020EF053B94AB9002908BF00281CBF4FF0FF3171
S31508020F004FF0FF3000F0B4B9ADF1080C6DE904CE2C
S31508020F1000F03CF8DDF804E0DDE9022304B070478E
S31508020F2038B50022002304460D46FFF70BFF28B901
S31508020F3020462946BDE8384000F00AB8204605F1A1
S31508020F40004100F005F8404261EB410138BD00BF9F
S31508020F50D0B500220B4B06460F46FFF781FCFFF77A
S31508020F6057FF0446FFF702FC0022074BFFF778FCFF
S31508020F7002460B4630463946FFF7BAFAFFF748FFEC
S31508020F802146D0BD0000F03D0000F0412DE9F04FAA
S31508020F90099D0C46002B4DD18A420F468446964639
S31508020FA0B2FA82F360D94BB102FA03FEC3F1200208
S31508020FB09F4000FA03FC20FA02F217434FEA1E4644
S31508020FC01FFA8EF44FEA1C42B7FBF6F106FB1177BD
S31508020FD001FB04F042EA0742904208D91EEB0202DC
S31508020FE001F1FF3702D2904200F22D813946121AD8
S31508020FF01FFA8CFCB2FBF6F006FB102200FB04F487
S315080210004CEA024C644508D91EEB0C0C00F1FF327F
S3150802101002D2644500F21A81104640EA0140ACEB5E
S31508021020040C002125B12CFA03F30022C5E900328B
S31508021030BDE8F08F8B4205D90DB1C5E90001002143
S315080210400846F5E7B3FA83F100294DD1A342C0F069
S31508021050F280904280F0EF80064623460846002D2D
S31508021060E6D0C5E90063E3E7002B40F0A2808A1ABE
S315080210704FEA1E471FFA8EF60121B2FBF7F407FB69
S3150802108014204FEA1C4242EA004206FB04F0904250
S315080210900FD91EEB020204F1FF382CBF4FF00109EB
S315080210A04FF00009904203D9B9F1000F00F0C88049
S315080210B04446121A1FFA8CFCB2FBF7F007FB102201
S315080210C000FB06F64CEA024C664508D91EEB0C0CE8
S315080210D000F1FF3202D2664500F2BB801046ACEB45
S315080210E0060C40EA04409DE7C1F120068B4004FA4B
S315080210F001FE22FA06F720FA06FCF4408A401F434C
S315080211004EEA0C0300FA01FE4FEA17484FEA134962
S315080211101FFA87FCB4FBF8F008FB104449EA0444BA
S3150802112000FB0CF9A1450ED93C1900F1FF3A2CBF78
S315080211304FF0010B4FF0000BA14503D9BBF1000F8D
S3150802114000F093805046A4EB09041FFA83F9B4FB16
S31508021150F8F308FB134403FB0CFC49EA0444A445D0
S3150802116006D93C1903F1FF3801D2A4457AD8434679
S3150802117043EA0040A4EB0C04A0FB02984445CC4683
S31508021180434602D306D1CE4504D20138B9EB020C46
S3150802119068EB07035DB1BEEB0C0264EB030404FAC9
S315080211A006F622FA01F3CC401E43C5E90064002183
S315080211B03EE702FA03FEC3F1200104FA03F200FA3B
S315080211C003FCCC404FEA1E4720FA01F11FFA8EF6BD
S315080211D0B4FBF7F00A4307FB1044110C41EA044139
S315080211E000FB06F48C420ED91EEB010100F1FF3812
S315080211F02CBF4FF001094FF000098C4202D9B9F110
S31508021200000F2CD04046091B92B2B1FBF7F407FB3C
S31508021210141142EA014204FB06F1914207D91EEB78
S31508021220020204F1FF3801D2914215D84446521AF5
S3150802123044EA004121E7861A64EB030301200EE71C
S31508021240023C724435E702397244D0E6F444023865
S31508021250E3E6F444023842E7023C7244E7E702381E
S315080212607144D0E7023B3C4482E702383C446AE7D1
S31508021270704700BF80B586B002AF78600023FB6076
S31508021280342300934FF448430B4A0C490C4831F077
S315080212902BFB0346002B0AD1094BBB60B8680EF03C
S315080212A071FDF860FB68002B01D000BFFDE700BFA7
S315080212B01037BD4680BD00BFC405002040BF0508E3
S315080212C0C4CD002080B400AF034B1B681846BD4648
S315080212D05DF8047B704700BFF8CD002080B483B068
S315080212E000AF7860044A7B681360012318460C37FE
S315080212F0BD465DF8047B7047F8CD002080B400AF88
S31508021300034B1B681846BD465DF8047B704700BF51
S3150802131004CE002080B483B000AF0346FB71054BB0
S315080213201E221A60012318460C37BD465DF8047B57
S31508021330704700BF04CE002080B483B000AF786047
S315080213400A4B1B68002B03D1084B00221A6005E0E2
S31508021350064B1A687B68D31A044A13600023184698
S315080213600C37BD465DF8047B704700BF04CE0020EB
S3150802137080B400AF044B00221A6000231846BD460B
S315080213805DF8047B704700BF04CE002080B400AF2E
S31508021390034B1B781846BD465DF8047B704700BFB1
S315080213A0FCCD002080B483B000AF0346FB71054A2A
S315080213B0FB791370012318460C37BD465DF8047B8A
S315080213C0704700BFFCCD002080B400AF034B1B88DA
S315080213D01846BD465DF8047B704700BFFECD002067
S315080213E080B483B000AF0346FB80054AFB881380AE
S315080213F0012318460C37BD465DF8047B704700BFCB
S31508021400FECD002080B400AF034B1B881846BD46AC
S315080214105DF8047B704700BF00CE002080B483B01D
S3150802142000AF0346FB80054AFB8813800123184652
S315080214300C37BD465DF8047B704700BF00CE00201E
S3150802144080B485B000AF786039600023FB607B68A2
S315080214501B78FB607B6801331B781B02FA6813440E
S31508021460FB607B6802331B781B04FA681344FB6033
S315080214707B6803331B781B06FA681344FB603B68D8
S31508021480FA681A6000BF1437BD465DF8047B7047D8
S315080214902DE9B04392B002AF78600B467B800023F9
S315080214A0FB604FF000024FF00003C7E90E23FFF777
S315080214B06DFF0346002B00F09882FFF785FF03466F
S315080214C040F29F32934200F03382B3F5687F80F28E
S315080214D06E8240F24222934200F3908040F2022248
S315080214E09342C0F26482A3F20223402B00F25F8287
S315080214F001A252F823F000BFF516020843160208A5
S31508021500AF180208AF190208AF190208AF19020884
S31508021510AF190208AF190208AF190208AF19020873
S31508021520AF190208AF190208AF190208AF19020863
S31508021530AF190208AF190208AF190208AF19020853
S31508021540AF190208AF190208AF190208AF19020843
S31508021550AF190208AF190208AF190208AF19020833
S31508021560AF190208AF190208AF190208AF19020823
S31508021570EF17020829180208AF190208AF1902085C
S315080215804F18020889180208AF190208AF1902088B
S31508021590AF190208AF190208AF190208AF190208F3
S315080215A0AF190208AF190208AF190208AF190208E3
S315080215B0AF190208AF190208AF190208AF190208D3
S315080215C0AF190208AF190208AF190208AF190208C3
S315080215D0AF190208AF190208AF190208AF190208B3
S315080215E0AF190208AF190208AF190208AF190208A3
S315080215F0A5170208AF1902080916020840F29E3218
S31508021600934200F0C581D2E107F10C0319467868C6
S31508021610FFF716FFFB681946BB481FF081FFBB4B55
S315080216201B68002B09D0BA481FF07AFF0220FFF781
S3150802163055FEB64B00221A60C9E11220FFF74EFE8C
S31508021640C5E107F10C0319467868FFF7F9FE18F0A9
S31508021650CDF9034618461AF079FBFB68184600F0DE
S315080216605DFC10EE103A1846FFF7A2F802460B4642
S31508021670C7E90E2318F0BAF9034618461AF031FCE0
S31508021680B0EE407AF0EE607A07F110008DED007B3D
S31508021690D7E90E239F4937F075F818F0A7F90346DC
S315080216A018461AF0FAFB51EC100BD7E90E23FEF78F
S315080216B01FFF02460B46904623F000494FF00002F0
S315080216C04FF0804340464946FFF750FB0346002B3E
S315080216D004D007F1100318461FF04EFE18F086F9DB
S315080216E0034697ED0E0B18461AF0E9FB1320FFF78F
S315080216F0F5FD6CE107F10C0319467868FFF7A0FEC1
S3150802170018F074F9034618461AF020FBFB681846C7
S3150802171000F022FC10EE103A1846FFF749F8024686
S315080217200B46C7E90E2318F061F9034618461AF064
S31508021730B4FB59EC108B07F11000D7E90E23CDE95B
S31508021740002342464B46734937F01CF818F04EF907
S31508021750034618461AF0C5FB51EC100BD7E90E23BF
S31508021760FEF7C6FE02460B46144623F0004564A35E
S31508021770D3E9002320462946FFF7F8FA0346002B49
S3150802178004D007F1100318461FF0F6FD18F02EF9DB
S31508021790034697ED0E0B18461AF0B5FB1420FFF711
S315080217A09DFD14E107F10C0319467868FFF748FE18
S315080217B0FB6803F00103002B0CD1FFF783FD0346F8
S315080217C0072B03D10820FFF789FD00E10320FFF765
S315080217D085FDFCE0FFF776FD0346072B03D10920BA
S315080217E0FFF77CFDF3E00420FFF778FDEFE007F151
S315080217F00C0319467868FFF723FEFB681A46464B20
S315080218001A60FB68DB0A07EE903AF8EE677A424BF3
S31508021810C3ED017AFB68DB0A194640481FF080FED1
S315080218200D20FFF75BFDD2E007F10C031946786835
S31508021830FFF706FEFB681A46374B9A60FB6819469D
S3150802184037481FF06DFE0E20FFF748FDBFE007F18F
S315080218500C0319467868FFF7F3FDFB681A462E4B08
S31508021860DA60FB68DB0A07EE903AF8EE677A2A4BEB
S31508021870C3ED047AFB68DB0A19462A481FF050FEB4
S315080218800F20FFF72BFDA2E007F10C031946786833
S31508021890FFF7D6FDFB681A461F4B5A61FB681946C5
S315080218A021481FF03DFE1020FFF718FD8FE007F1D3
S315080218B00C0319467868FFF7C3FDFC68FB681846EF
S315080218C000F068FB10EE103A1846FEF771FF024662
S315080218D00B46214615481FF023FEFB68184600F002
S315080218E059FB10EE103A1846FEF762FF02460B46FF
S315080218F0C7E90E231620FFF7F1FC68E0AFF3008074
S315080219009A9999999999B93F54BF05080CCE00201E
S315080219106CBF050884BF050830CE002098BF0508AD
S31508021920A8BF0508C0BF0508D0BF0508E8BF050857
S3150802193007F10C0319467868FFF782FDFC68FB6815
S315080219401846FEF713FF02460B4643EC102B00F02F
S315080219503FFB53EC102B214626481FF0E1FDFB689E
S315080219601846FEF703FF02460B4643EC102B00F01F
S315080219702FFB87ED0E0BFFF7A5FC0346192B03D1A8
S315080219801A20FFF7ABFC22E01420FFF7A7FC1EE0A3
S3150802199007F10C0319467868FFF752FDFB681946EA
S315080219A015481FF0BDFD1420FFF798FC0FE007F15C
S315080219B00C0319467868FFF743FDFFF705FD034652
S315080219C01946FB681A460D481FF0AAFD00BF0020FB
S315080219D0FFF7E8FC0020FFF703FD0020FFF71EFDD6
S315080219E0FFF7C6FC064B00221A7000BF4037BD46F9
S315080219F0BDE8B08308C005082CC0050848C005081C
S31508021A0008CE002080B500AFFFF7C0FC0346002BC6
S31508021A1024D0FFF7D9FC0346002B21D00120FFF77B
S31508021A208BFCFFF76BFC0346002B10D10D4B1B7882
S31508021A300133DAB20B4B1A700B481FF09DFC0020DB
S31508021A40FFF7B0FC0020FFF7CBFC1EF0BBFB054BF3
S31508021A501B78022B04D90EF03BFE01E0FFF788FC47
S31508021A6000BF80BD08CE002064C0050880B584B0DA
S31508021A7000AF0346FB800B46BB801346FB70002370
S31508021A80FB7307F1080305220021184636F00EFFFC
S31508021A900023BB73FB881B01FB80BB7B5A1CBA73F2
S31508021AA0FA88D2B210333B4403F8082CFB881B0A87
S31508021AB09AB2BB7B591CB973D2B210333B4403F8B2
S31508021AC0082CBB7B5A1CBA73BA88D2B210333B4471
S31508021AD003F8082CBB881B0A9AB2BB7B591CB9733C
S31508021AE0D2B210333B4403F8082CFB78002B08D1FA
S31508021AF0BB7B9AB207F10803114618461FF0E6FEA9
S31508021B0007E0BB7B9AB207F10803114618461FF095
S31508021B1019FEFB7B18461037BD4680BD80B586B0D8
S31508021B2000AF03463960FB8013467B710023FB75C1
S31508021B3007F10C0307220021184636F0B7FE0023E8
S31508021B40BB75FB881B01FB80BB7D5A1CBA75FA88DC
S31508021B50D2B218333B4403F80C2CFB881B0A9AB200
S31508021B60BB7D591CB975D2B218333B4403F80C2C09
S31508021B70BB7D5A1CBA753A68D2B218333B4403F88D
S31508021B800C2C3B681A0ABB7D591CB975D2B218339C
S31508021B903B4403F80C2C3B681A0CBB7D591CB975DF
S31508021BA0D2B218333B4403F80C2C3B681A0EBB7DA1
S31508021BB0591CB975D2B218333B4403F80C2C7B79FD
S31508021BC0002B08D1BB7D9AB207F10C0311461846C1
S31508021BD01FF07CFE07E0BB7D9AB207F10C031146A3
S31508021BE018461FF0AFFDFB7D18461837BD4680BD67
S31508021BF080B588B000AF0346FB800023FB7707F168
S31508021C000C0310220021184636F050FE0023BB773B
S31508021C10FB88BB83BB8B1B01BB83BB8B43F00803CF
S31508021C20BB83BB8B43F00403BB83BB7F5A1CBA77C7
S31508021C30BA8BD2B220333B4403F8142CBB8B1B0A53
S31508021C409AB2BB7F591CB977D2B220333B4403F808
S31508021C50142CFFF79BFB0346002B18D1BB7F9AB2C5
S31508021C6007F10C03114618461FF030FEFB8818468A
S31508021C70FFF7B6FBBB8B1846FFF7D0FB0120FFF731
S31508021C8091FBFB88DBB21846FFF744FB01E0002311
S31508021C90FB77FB7F18462037BD4680BD80B500AF6F
S31508021CA000220421114824F0FDFB0A201FF050FFF0
S31508021CB0012204210D4824F0F5FB64201FF048FF99
S31508021CC0002000F0D1F864201FF042FF002000F047
S31508021CD011F800224FF070410020FFF71FFF044B56
S31508021CE001221A700123184680BD00BF0004024271
S31508021CF010CE002080B582B000AF0346FB71FB7997
S31508021D001A46022140F2B940FFF7B0FE64201FF0DE
S31508021D101FFFFB791A4608212020FFF7FFFE6420E1
S31508021D201FF016FFFB791A464FF4417140F28140C3
S31508021D30FFF79CFE64201FF00BFFFB791A464FF44F
S31508021D40406140F2AF40FFF791FE64201FF000FFAA
S31508021D50FB791A46002140F29340FFF787FE64207A
S31508021D601FF0F6FEFB791A46002140F29240FFF771
S31508021D707DFE64201FF0ECFEFB791A46394940F2D3
S31508021D800F40FFF7CBFE64201FF0E2FEFB791A46EE
S31508021D90002140F29A40FFF769FE64201FF0D8FE40
S31508021DA0FB791A464FF4807140F20540FFF7B6FEFA
S31508021DB064201FF0CDFEFB791A4643F2C83140F281
S31508021DC01C40FFF7ABFE64201FF0C2FEFB791A46E1
S31508021DD043F2C83140F21D40FFF7A0FE64201FF00F
S31508021DE0B7FEFB791A4643F2C83140F21E40FFF7A6
S31508021DF095FE64201FF0ACFEFB791A46052140F2D7
S31508021E009140FFF78BFE64201FF0A2FEFB791A466B
S31508021E104FF47A714C20FFF781FE64201FF098FE7A
S31508021E20FB791A464FF47A7140F2B240FFF71EFE6A
S31508021E3064201FF08DFEFB791A460C2140F2B6404B
S31508021E40FFF714FE64201FF083FEFB791A46012170
S31508021E504FF49660FFF70AFE012318460837BD4677
S31508021E6080BD00BFE8112C0080B588B000AF0346DC
S31508021E70FB710023FB7707F108031022002118469D
S31508021E8036F014FD0023BB774FF49063BB8301231E
S31508021E907B83BB8B1B01BB83BB7F5A1CBA77BA8B6E
S31508021EA0D2B220333B4403F8182CBB8B1B0A9AB2D6
S31508021EB0BB7F591CB977D2B220333B4403F8182C9E
S31508021EC0BB7F5A1CBA777A8BD2B220333B4403F8CB
S31508021ED0182C7B8B1B0A9AB2BB7F591CB977D2B2D4
S31508021EE020333B4403F8182CFB79002B08D1BB7F1F
S31508021EF09AB207F10803114618461FF0E7FC07E0F5
S31508021F00BB7F9AB207F10803114618461FF01AFC5E
S31508021F10FB7F18462037BD4680BD000080B485B0D9
S31508021F2000AF78600B4BFB607B6807EE903AF8EEE1
S31508021F30677A97ED037A67EE277AC7ED037AFB6825
S31508021F4007EE903AB0EE670A1437BD465DF8047B91
S31508021F50704700BFCEFF603780B485B000AF7860A7
S31508021F600B4BFB607B6807EE903AF8EE677A97EDC3
S31508021F70037A67EE277AC7ED037AFB6807EE903A8B
S31508021F80B0EE670A1437BD465DF8047B704700BF9A
S31508021F904815E13580B485B000AF78600B4BFB601D
S31508021FA07B6807EE903AF8EE677A97ED037A67EE62
S31508021FB0277AC7ED037AFB6807EE903AB0EE670A0E
S31508021FC01437BD465DF8047B704700BFDCB8453B55
S31508021FD080B584B000AF87ED000B0DA3D3E90023CB
S31508021FE0C7E90223D7E90023D7E90201FEF738FC3D
S31508021FF002460B46C7E90223D7E9022343EC172B0D
S31508022000B0EE470AF0EE670A1037BD4680BD00BF3C
S3150802201055DB2CE264B0BC3EB0B582B000AF4FF0DF
S3150802202000037B6000233B60C74B1B681A2B00F238
S31508022030348201A252F823F0A52002089B24020842
S31508022040BB200208D1200208EF2002080D2102084F
S315080220502B210208492102085F2102087D21020874
S315080220609B210208BB210208D9210208EF21020896
S31508022070052202081B22020831220208AD220208A2
S315080220806123020887230208D72302089B23020832
S31508022090AF230208C3230208F3230208072402080F
S315080220A01B240208FFF772F90346002B40F0C4818D
S315080220B040F24220FFF79CFDBEE1FFF767F90346AF
S315080220C0002B40F0BB814FF41070FFF791FDB5E18C
S315080220D09E4B1B685A1C9D490A600B2B40F2B08125
S315080220E0994B04221A60994B00221A60A8E1FFF75D
S315080220F04DF90346002B40F0A5810022132130201A
S31508022100FFF70CFD904B05221A609BE18F4B1B686B
S315080221105A1C8E490A60C72B40F296818A4B0622C0
S315080221201A608A4B00221A608EE1FFF72FF90346DE
S31508022130002B40F08B81002200213020FFF7EEFCB5
S31508022140814B07221A6081E1FFF720F90346002B2B
S3150802215040F07E814FF41070FFF74AFD78E17B4B21
S315080221601B685A1C79490A600F2B40F27381764B19
S3150802217009221A60754B00221A606BE1FFF706F90D
S315080221800346002B40F06881002243213020FFF7E6
S31508022190C5FC6D4B0A221A605EE16C4B1B685A1C21
S315080221A06A490A60B3F5C87FC0F05881664B0B22AC
S315080221B01A60664B00221A6050E1FFF7E7F80346F9
S315080221C0002B40F04D81002200213020FFF7A6FCAB
S315080221D05D4B0C221A6043E1FFF7D8F80346002B41
S315080221E040F040814FF40870FFF702FD3AE1FFF72D
S315080221F0CDF80346002B40F0378140F22120FFF745
S31508022200F7FC31E1FFF7C2F80346002B40F02E81B6
S315080222104FF40970FFF7ECFC28E1FFF7B7F803461D
S31508022220002B40F0258140F22520FFF7E1FC1FE153
S31508022230FFF7ACF80346002B40F01C81444B5B6861
S315080222401846FEF7B5FA3CA3D3E90023FEF732FC9B
S3150802225002460B46144683F000454FF000023D4BFA
S3150802226020462946FEF744F902460B461046194609
S315080222704FF00002384BFEF7F3FA02460B461046B9
S315080222801946FEF7E5FD03467B60D7ED017AFDEEBA
S31508022290E77A17EE903A3B603B680022194600201F
S315080222A0FFF73CFC284B11221A60E3E0FFF76EF8B1
S315080222B00346002B40F0E080254B1B691846FEF7C3
S315080222C077FA1FA3D3E90023FEF7F4FB02460B466F
S315080222D0104619464FF000021E4BFEF709F9024650
S315080222E00B46104619464FF000021B4BFEF7B8FA8A
S315080222F002460B4610461946FEF7AAFD03467B60C0
S31508022300D7ED017AFDEEE77A17EE903A3B603B6825
S31508022310002219460220FFF701FC0B4B12221A6013
S315080223200E4B1B78002B00F0A7800C4B00221A706C
S31508022330A2E000BFAFF300800000000000349A401C
S31508022340000000008031CA40F8CD002060CE00208F
S3150802235030CE00200000F03F0000A041DCD3002070
S31508022360FFF714F80346002B40F088804D4B1B6894
S31508022370002B03D04C4B00221A607FE040F2032068
S31508022380FFF736FC7AE0FFF701F80346002B77D110
S3150802239040F20220FFF72CFC72E0FEF7F7FF034635
S315080223A0002B6FD14FF40170FFF722FC6AE0FEF7AB
S315080223B0EDFF0346002B67D140F29F30FFF718FC6A
S315080223C062E0FEF7E3FF0346002B5FD140F29E3040
S315080223D0FFF70EFC5AE0354B1B685A1C33490A6054
S315080223E0092B55D9304B12221A60304B00221A603B
S315080223F04EE0002209214FF49660FFF737FB2A4B7D
S3150802240019221A6049E0FEF7C1FF0346002B41D1A3
S3150802241040F29F30FFF7ECFB3CE0FEF7B7FF0346BE
S31508022420002B39D1002201214FF49660FFF71EFBDB
S315080224301D4B14221A602FE000BF2EE000BF2CE0CD
S3150802244000BF2AE000BF28E000BF26E000BF24E064
S3150802245000BF22E000BF20E000BF1EE000BF1CE074
S3150802246000BF1AE000BF18E000BF16E000BF14E084
S3150802247000BF12E000BF10E000BF0EE000BF0CE094
S3150802248000BF0AE000BF08E000BF06E000BF04E0A4
S3150802249000BF02E000BF00E000BF00BF0837BD462C
S315080224A0B0BD00BF0CCE0020F8CD002060CE0020C3
S315080224B080B500AF00224FF48051124823F0F2FF94
S315080224C00A201FF045FB01224FF480510D4823F0E4
S315080224D0E9FF64201FF03CFB0120FFF7C5FC6420DE
S315080224E01FF036FB0120FFF705FC01224FF0704171
S315080224F00020FFF713FB044B01221A70012318462A
S3150802250080BD00BF001002422CCE002080B400AF6E
S31508022510034B1B681846BD465DF8047B704700BF2F
S3150802252014CE002080B483B000AF7860044A7B687A
S315080225301360012318460C37BD465DF8047B7047C5
S3150802254014CE002080B400AF034B1B681846BD4664
S315080225505DF8047B704700BF20CE002080B483B0AC
S3150802256000AF0346FB71054B1E221A60012318466B
S315080225700C37BD465DF8047B704700BF20CE0020AD
S3150802258080B483B000AF78600A4B1B68002B03D176
S31508022590084B00221A6005E0064B1A687B68D31AB4
S315080225A0044A1360002318460C37BD465DF8047BBF
S315080225B0704700BF20CE002080B400AF044B002233
S315080225C01A6000231846BD465DF8047B704700BFB3
S315080225D020CE002080B400AF034B1B781846BD46B8
S315080225E05DF8047B704700BF18CE002080B483B024
S315080225F000AF0346FB71054AFB791370012318469F
S315080226000C37BD465DF8047B704700BF18CE002024
S3150802261080B400AF034B1B881846BD465DF8047BA1
S31508022620704700BF1ACE002080B483B000AF0346BD
S31508022630FB80054AFB881380012318460C37BD46E2
S315080226405DF8047B704700BF1ACE002080B400AF45
S31508022650034B1B881846BD465DF8047B704700BFCE
S315080226601CCE002080B483B000AF0346FB80054A27
S31508022670FB881380012318460C37BD465DF8047B98
S31508022680704700BF1CCE002080B588B000AF034655
S31508022690FB800023FB7707F10C0310220021184662
S315080226A036F004F90023BB77FB88BB83BB8B1B017F
S315080226B0BB83BB8B43F00803BB83BB8B43F004038A
S315080226C0BB83BB7F5A1CBA77BA8BD2B220333B4440
S315080226D003F8142CBB8B1B0A9AB2BB7F591CB97719
S315080226E0D2B220333B4403F8142CFEF74FFE0346BE
S315080226F0002B18D1BB7F9AB207F10C031146184674
S315080227001FF020F8FB881846FFF78EFFBB8B18468A
S31508022710FFF7A8FF0120FFF769FFFB88DBB218461F
S31508022720FFF71CFF01E00023FB77FB7F18462037E3
S31508022730BD4680BD80B500AFFFF74CFF0346002BB0
S3150802274024D0FFF765FF0346002B21D00120FFF7AF
S3150802275017FFFFF7F7FE0346002B10D10D4B1B7828
S315080227600133DAB20B4B1A700B481EF005FE002035
S31508022770FFF73CFF0020FFF757FF1DF0ADFD054BA5
S315080227801B78022B04D90DF0A3FF01E0FFF714FF13
S3150802279000BF80BD24CE00207CC0050800000000D2
S315080227A0B0B582B000AF4FF000037B6000233B60F8
S315080227B0C74B1B681A2B00F2348201A252F823F087
S315080227C02D280208232C0208432802085928020841
S315080227D07728020895280208B3280208D128020891
S315080227E0E7280208052902082329020843290208BC
S315080227F061290208772902088D290208A3290208F5
S31508022800B9290208352A0208E92A02080F2B020802
S315080228105F2B0208232B0208372B02084B2B0208D0
S315080228207B2B02088F2B0208A32B0208FFF7D2FE86
S315080228300346002B40F0C48140F24220FFF724FFF2
S31508022840BEE1FFF7C7FE0346002B40F0BB814FF4FB
S315080228501070FFF719FFB5E19E4B1B685A1C9D497C
S315080228600A600B2B40F2B081994B04221A60994BED
S3150802287000221A60A8E1FFF7ADFE0346002B40F0DE
S31508022880A581012213213020FFF748F9904B052232
S315080228901A609BE18F4B1B685A1C8E490A60C72B2C
S315080228A040F296818A4B06221A608A4B00221A60E7
S315080228B08EE1FFF78FFE0346002B40F08B81012243
S315080228C000213020FFF72AF9814B07221A6081E19D
S315080228D0FFF780FE0346002B40F07E814FF410700E
S315080228E0FFF7D2FE78E17B4B1B685A1C79490A60CE
S315080228F00F2B40F27381764B09221A60754B002220
S315080229001A606BE1FFF766FE0346002B40F068810A
S31508022910012243213020FFF701F96D4B0A221A6082
S315080229205EE16C4B1B685A1C6A490A60B3F5C87F9C
S31508022930C0F05881664B0B221A60664B00221A6059
S3150802294050E1FFF747FE0346002B40F04D81012276
S3150802295000213020FFF7E2F85D4B0C221A6043E1B2
S31508022960FFF738FE0346002B40F040814FF408700B
S31508022970FFF78AFE3AE1FFF72DFE0346002B40F0E9
S31508022980378140F22120FFF77FFE31E1FFF722FE71
S315080229900346002B40F02E814FF40970FFF774FEB0
S315080229A028E1FFF717FE0346002B40F0258140F287
S315080229B02520FFF769FE1FE1FFF70CFE0346002BF1
S315080229C040F01C81444B5B681846FDF7F1FE3CA3B8
S315080229D0D3E90023FEF76EF802460B46144683F047
S315080229E000454FF000023D4B20462946FDF780FD83
S315080229F002460B46104619464FF00002384BFDF7C1
S31508022A002FFF02460B4610461946FEF721FA0346E1
S31508022A107B60D7ED017AFDEEE77A17EE903A3B60D6
S31508022A203B68012219460020FFF778F8284B112245
S31508022A301A60E3E0FFF7CEFD0346002B40F0E08084
S31508022A40254B1B691846FDF7B3FE1FA3D3E90023DE
S31508022A50FEF730F802460B46104619464FF00002BA
S31508022A601E4BFDF745FD02460B46104619464FF02A
S31508022A7000021B4BFDF7F4FE02460B4610461946AA
S31508022A80FEF7E6F903467B60D7ED017AFDEEE77AB3
S31508022A9017EE903A3B603B68012219460220FFF77F
S31508022AA03DF80B4B12221A600E4B1B78002B00F0D6
S31508022AB0A7800C4B00221A70A2E000BFAFF3008079
S31508022AC00000000000349A40000000008031CA402D
S31508022AD014CE002064CE002030CE00200000F03F45
S31508022AE00000A041DCD30020FFF774FD0346002B4B
S31508022AF040F088804D4B1B68002B03D04C4B0022BC
S31508022B001A607FE040F20320FFF7BEFD7AE0FFF786
S31508022B1061FD0346002B77D140F20220FFF7B4FD90
S31508022B2072E0FFF757FD0346002B6FD14FF4017091
S31508022B30FFF7AAFD6AE0FFF74DFD0346002B67D1B2
S31508022B4040F29F30FFF7A0FD62E0FFF743FD034620
S31508022B50002B5FD140F29E30FFF796FD5AE0354BC7
S31508022B601B685A1C33490A60092B55D9304B122265
S31508022B701A60304B00221A604EE0012209214FF4F6
S31508022B809660FEF773FF2A4B19221A6049E0FFF78F
S31508022B9021FD0346002B41D140F29F30FFF774FD19
S31508022BA03CE0FFF717FD0346002B39D1012201212C
S31508022BB04FF49660FEF75AFF1D4B14221A602FE057
S31508022BC000BF2EE000BF2CE000BF2AE000BF28E0CD
S31508022BD000BF26E000BF24E000BF22E000BF20E0DD
S31508022BE000BF1EE000BF1CE000BF1AE000BF18E0ED
S31508022BF000BF16E000BF14E000BF12E000BF10E0FD
S31508022C0000BF0EE000BF0CE000BF0AE000BF08E00C
S31508022C1000BF06E000BF04E000BF02E000BF00E01C
S31508022C2000BF00BF0837BD46B0BD00BF0CCE0020AE
S31508022C3014CE002064CE0020B0B592B002AF786000
S31508022C400B467B800023FB604FF000024FF0000327
S31508022C50C7E90E23FFF7BEFC0346002B00F07A8273
S31508022C60FFF7D6FC034640F29F32934200F0FD81FD
S31508022C70B3F5687F80F2508240F24222934200F313
S31508022C808F8040F202229342C0F24682A3F20223C6
S31508022C90402B00F2418201A252F823F0992E020833
S31508022CA0E72D02081D3002081931020819310208F7
S31508022CB019310208193102081931020819310208B4
S31508022CC019310208193102081931020819310208A4
S31508022CD01931020819310208193102081931020894
S31508022CE01931020819310208193102081931020884
S31508022CF01931020819310208193102081931020874
S31508022D001931020819310208193102081931020863
S31508022D10193102085D2F0208972F02081931020895
S31508022D2019310208BD2F0208F72F020819310208C5
S31508022D301931020819310208193102081931020833
S31508022D401931020819310208193102081931020823
S31508022D501931020819310208193102081931020813
S31508022D601931020819310208193102081931020803
S31508022D7019310208193102081931020819310208F3
S31508022D8019310208193102081931020819310208E3
S31508022D9019310208132F020819310208AD2D02084B
S31508022DA040F29E32934200F09081B5E107F10C039E
S31508022DB019467868FEF744FBFB681946CA481EF0AE
S31508022DC0AFFBCA4B1B68002B09D0C9481EF0A8FBEB
S31508022DD00220FFF7A7FBC54B00221A60ACE11220BE
S31508022DE0FFF7A0FBA8E107F10C0319467868FEF77E
S31508022DF027FB16F0FBFD0346184618F0A7FFFB68EB
S31508022E001846FFF78BF810EE103A1846FDF7D0FC75
S31508022E1002460B46C7E90E2316F0E8FD0346184696
S31508022E2019F013F9B0EE407AF0EE607A07F1100065
S31508022E308DED007BD7E90E23AE4935F0A3FC16F0DB
S31508022E40D5FD0346184619F0DCF851EC100BD7E904
S31508022E500E23FDF74DFB02460B46144623F00045AA
S31508022E604FF000024FF0804320462946FDF77EFFC9
S31508022E700346002B04D007F1100318461EF07CFA0D
S31508022E8016F0B4FD034697ED0E0B184619F0CBF86B
S31508022E901320FFF747FB4FE107F10C031946786841
S31508022EA0FEF7CEFA16F0A2FD0346184618F04EFFB4
S31508022EB0FB681846FFF750F810EE103A1846FDF769
S31508022EC077FC02460B46C7E90E2316F08FFD03462A
S31508022ED0184619F096F855EC104B07F11000D7E989
S31508022EE00E23CDE9002322462B46824935F04AFCB9
S31508022EF007F1100318461EF03FFA16F077FD03464F
S31508022F0097ED0E0B184619F0B2F81420FFF70AFBD4
S31508022F1012E107F10C0319467868FEF791FAFB6885
S31508022F2003F00103002B0CD1FFF7F0FA0346072B37
S31508022F3003D10820FFF7F6FAFEE00320FFF7F2FABC
S31508022F40FAE0FFF7E3FA0346072B03D10920FFF756
S31508022F50E9FAF1E00420FFF7E5FAEDE007F10C03E0
S31508022F6019467868FEF76CFAFB681A46624B1A60CD
S31508022F70FB68DB0A07EE903AF8EE677A5E4BC3ED1A
S31508022F80017AFB68DB0A19465C481EF0C9FA0D206D
S31508022F90FFF7C8FAD0E007F10C0319467868FEF77E
S31508022FA04FFAFB681A46544B9A60FB68194654480E
S31508022FB01EF0B6FA0E20FFF7B5FABDE007F10C03CC
S31508022FC019467868FEF73CFAFB681A464A4BDA60F5
S31508022FD0FB68DB0A07EE903AF8EE677A464BC3EDD2
S31508022FE0047AFB68DB0A194646481EF099FA0F204E
S31508022FF0FFF798FAA0E007F10C0319467868FEF77E
S315080230001FFAFB681A463C4B5A61FB6819463E484A
S315080230101EF086FA1020FFF785FA8DE007F10C03F9
S3150802302019467868FEF70CFAFC68FB681846FEF73C
S31508023030B1FF10EE103A1846FDF7BAFB02460B46E8
S31508023040214632481EF06CFAFB681846FEF7A2FFC4
S3150802305010EE103A1846FDF7ABFB02460B46C7E9D7
S315080230600E231620FFF75EFA66E007F10C031946EF
S315080230707868FEF7E5F9FC68FB681846FDF776FB03
S3150802308002460B4643EC102BFEF7A2FF53EC102B1D
S3150802309021461F481EF044FAFB681846FDF766FBF0
S315080230A002460B4643EC102BFEF792FF87ED0E0BFA
S315080230B0FFF72CFA0346192B03D11A20FFF732FA27
S315080230C03AE01420FFF72EFA36E007F10C03194608
S315080230D07868FEF7B5F9FB6819460E481EF020FA1D
S315080230E01420FFF71FFA27E098C0050828CE00200B
S315080230F0B4C00508D0C0050848CE0020E4C00508BB
S31508023100F8C0050810C1050824C105083CC1050810
S315080231105CC1050884C1050807F10C0319467868DD
S31508023120FEF78EF9FFF774FA03461946FB681A4644
S315080231300A481EF0F5F900BF0020FFF757FA0020EB
S31508023140FFF772FA0020FFF78DFAFFF735FA044BFC
S3150802315000221A7000BF4037BD46B0BDA4C105089B
S3150802316024CE002080B582B000AF16F03FFC03469D
S31508023170184616F0C9FC78604FF488720021786800
S3150802318035F094FB1522514901201EF057FC7B6845
S315080231904F4A1A607B684FF47A621A817B6840F656
S315080231A0AC525A817B687F221A737B684FF6FF728C
S315080231B0DA817B684FF6FF721A827B68454A9A6102
S315080231C07B68444A5A617B6800229A837B6800229C
S315080231D0DA837B68002283F820207B6800225A84DF
S315080231E07B68002283F824207B68002283F8252046
S315080231F07B68002283F826207B68002283F8272032
S315080232007B68002283F828207B68334ADA627B6867
S3150802321000221A860121786816F046FF002178688E
S3150802322016F0F3FF7B684FF6FF725A877B68002217
S3150802323083F83C207B6800221A647B6844330B229D
S315080232403021184635F032FB7B684F33382200218D
S31508023250184635F02BFB7B6887331822002118465F
S3150802326035F024FB7B68012283F89F207B680022C5
S3150802327083F8A1207B68002283F8A0207B68164A7F
S31508023280C3F8A4207B68002283F8A8207B68002262
S3150802329083F8A9207B68114AC3F8AC207B684FF0F3
S315080232A00002C3F8B0207B68002283F8B4207B684A
S315080232B0002283F8B52016F099FB03460121184629
S315080232C019F0DBFA00BF0837BD4680BDC0C1050844
S315080232D02345434900007F43CDCC2C40333333404A
S315080232E080B588B000AFF860B9601346FB71002359
S315080232F0FB6100233B61BB687B617B69BB61002381
S31508023300FB6110E0FA69FB681344184632F094F838
S3150802331003463B613A69BB691A60BB690433BB6100
S31508023320FB690433FB61FB79FA699A42EADB0123FA
S3150802333018462037BD4680BD90B5C7B000AF16F017
S3150802334055FB0346184616F0DFFBC7F814014FF47F
S3150802335088720021D7F8140135F0A8FA3B1D4FF4FC
S3150802336088720021184635F0A1FA3B1D102219462B
S31508023370D748FFF7B5FF07F58C73A3F58A731B6861
S31508023380D44A934200F0B48107F58C73A3F58A7385
S315080233901B68D14A93426BD907F58C73A3F58A73D6
S315080233A01B68CE4A934263D8D7F81431C94A1A60C1
S315080233B007F58C73A3F58A735A68D7F814315A60DD
S315080233C0D7F814314FF47A621A81D7F8143140F6D5
S315080233D0AC525A81D7F814317F221A73D7F81431AE
S315080233E0BF4A9A61D7F81431BD4A5A61D7F81431DF
S315080233F000229A83D7F814310022DA83D7F81431D7
S31508023400002283F82020D7F8143100225A84D7F8EC
S315080234101431002283F82420D7F81431002283F8C5
S315080234202520D7F81431002283F82620D7F814313C
S31508023430002283F82720D7F81431002283F828209F
S3150802344007F58C73A3F58A73DA6AD7F81431DA6248
S315080234500121D7F8140116F027FE0021D7F8140126
S3150802346016F0D3FED7F814314FF6FF725A875AE18F
S3150802347007F58C73A3F58A731B68984A934240F240
S31508023480248107F58C73A3F58A731B68954A9342C0
S3150802349000F21B81D7F814318E4A1A6007F58C732D
S315080234A0A3F58A735A68D7F814315A60D7F81431D3
S315080234B04FF47A621A81D7F8143140F6AC525A811F
S315080234C0D7F814317F221A7307F58C73A3F58A731A
S315080234D09A69D7F814319A6107F58C73A3F58A733A
S315080234E05A69D7F814315A6107F58C73A3F58A73AA
S315080234F09A8BD7F814319A8307F58C73A3F58A73D6
S31508023500DA8BD7F81431DA8307F58C73A3F58A7345
S3150802351093F82020D7F8143183F8202007F58C7306
S31508023520A3F58A735A8CD7F814315A8407F58C7323
S31508023530A3F58A7393F82420D7F8143183F8242044
S3150802354007F58C73A3F58A7393F82520D7F81431F7
S3150802355083F8252007F58C73A3F58A7393F826203A
S31508023560D7F8143183F8262007F58C73A3F58A73E6
S3150802357093F82720D7F8143183F8272007F58C7398
S31508023580A3F58A7393F82820D7F8143183F82820EC
S3150802359007F58C73A3F58A73DA6AD7F81431DA62F7
S315080235A007F58C73A3F58A731A8ED7F814311A861F
S315080235B007F58C73A3F58A735A8ED7F814315A868F
S315080235C007F58C73A3F58A7393F83520D7F8143167
S315080235D083F8352007F58C73A3F58A7393F8372099
S315080235E0D7F8143183F83720D7F8143193F83530E1
S315080235F01946D7F8140116F057FDD7F8143193F87F
S3150802360037301946D7F8140116F0FFFDD7F81431EA
S315080236104FF6FF725A87D7F81431002283F83C20F6
S31508023620D7F8143100221A64D7F8143144330B221E
S315080236303021184635F03AF9D7F814314F33382283
S315080236400021184635F032F9D7F814318733182293
S315080236500021184635F02AF907F58C73A3F58A7303
S3150802366093F89F20D7F8143183F89F20D7F814319E
S31508023670002283F8A120D7F81431002283F8A0206B
S31508023680D7F81431184AC3F8A420D7F814310022FF
S3150802369083F8A820D7F81431002283F8A920D7F88E
S315080236A01431124AC3F8AC20D7F814314FF000028D
S315080236B0C3F8B020D7F81431002283F8B420D7F81B
S315080236C01431002283F8B5202DE0FFF74BFD2AE0DE
S315080236D000C01F0823454349004543490845434955
S315080236E000007F4322454349CDCC2C403333334037
S315080236F03B1D4FF488721946D7F8140135F073F951
S315080237000F22374901201EF099F9D7F814311B8A7E
S315080237104FF6FF72934206D116F068F90346012165
S31508023720184619F0AAF8D7F8143193F8263019462C
S31508023730D7F8140116F093FBD7F8143193F83530FD
S315080237401946D7F8140116F0AFFCD7F8143193F8D6
S3150802375037301946D7F8140116F057FD16F046F910
S315080237600346184619F0F2F90346002B0BD116F058
S315080237703DF90446D7F8140116F05AFC03461946D1
S31508023780204619F0F0F916F031F90446D7F8140173
S3150802379016F0A4FD03461946204619F0A5FAD7F8ED
S315080237A0140116F084FE10EE103A1846FDF700F8DA
S315080237B009A3D3E90023FDF7C5FA0346002B05D072
S315080237C09FED080AD7F8140116F060FE0023184682
S315080237D007F58E77BD4690BD333333333333034013
S315080237E0D4C105083333334090B589B000AF0023FE
S315080237F0FB6116F0FBF80346184616F085F9786160
S315080238007B69BB61FE2031F046FE0023FB611CE0AA
S315080238103B1D10220021184635F048F8BB693C1DAD
S31508023820186859689A68DB680FC4FB6903F1016373
S3150802383003F57C233A1D1146184631F011FEBB6981
S315080238401033BB61FB691033FB61FB69B3F5887FF3
S31508023850DED3012318462437BD4690BD80B400AF97
S31508023860034B1B681846BD465DF8047B704700BFCC
S3150802387068CE002080B483B000AF7860044A7B68C3
S31508023880136000BF0C37BD465DF8047B704700BF66
S3150802389068CE002080B400AF034B1B781846BD469D
S315080238A05DF8047B704700BF6CCF002080B582B0FC
S315080238B000AF78601A4B1B78042B26D801A252F85F
S315080238C023F000BFD9380208E3380208ED380208A7
S315080238D0F7380208013902081249786834F052FFAB
S315080238E018E01149786834F04DFF13E00F497868FB
S315080238F034F048FF0EE00E49786834F043FF09E0D9
S315080239000C49786834F03EFF04E00B49786834F0D5
S3150802391039FF00BF7B6818460837BD4680BD00BF21
S315080239206CCF0020E0C10508ECC10508F4C1050802
S3150802393004C2050814C2050824C2050880B400AFEB
S31508023940034B1B781846BD465DF8047B704700BFDB
S315080239506DCF002080B483B000AF0346FB71054AE1
S31508023960FB791370012318460C37BD465DF8047BB4
S31508023970704700BF6DCF002080B582B000AF786077
S31508023980374B1B780D2B60D801A252F823F000BFE3
S31508023990C9390208D3390208DD390208E7390208AB
S315080239A0F1390208FB390208053A02080F3A0208F9
S315080239B0193A02082D3A0208233A02084B3A020833
S315080239C0373A0208413A02082649786834F0DAFE9C
S315080239D040E02549786834F0D5FE3BE0234978680B
S315080239E034F0D0FE36E02249786834F0CBFE31E076
S315080239F02049786834F0C6FE2CE01F49786834F00E
S31508023A00C1FE27E01D49786834F0BCFE22E01C4955
S31508023A10786834F0B7FE1DE01A49786834F0B2FEC9
S31508023A2018E01949786834F0ADFE13E0174978684A
S31508023A3034F0A8FE0EE01649786834F0A3FE09E0D1
S31508023A401449786834F09EFE04E01349786834F025
S31508023A5099FE00BF7B6818460837BD4680BD00BF81
S31508023A606DCF002030C205083CC2050848C20508C9
S31508023A7058C2050864C2050874C2050884C2050846
S31508023A8094C20508A8C20508BCC20508C8C205082A
S31508023A90D8C20508ECC2050800C3050880B400AF01
S31508023AA0034B1B681846BD465DF8047B704700BF8A
S31508023AB0E4CF002080B483B000AF7860044A7B6804
S31508023AC01360012318460C37BD465DF8047B704720
S31508023AD0E4CF002080B58CB008AF78607B68FB60C5
S31508023AE040221A491A480EF05FF94FF496710120DE
S31508023AF00CF0BCFD07F1080100234FF48052F86868
S31508023B002EF07EFE0346002B01D002231AE0BB6884
S31508023B10B022069201220592002204920A220392F8
S31508023B200A2202924FF48052019200930023094A14
S31508023B3009490A482FF0AAF80346002B01D00E239A
S31508023B4000E0002318461037BD4680BD7CCE002013
S31508023B506CCE0020FD9102080CC30508BCCE0020DD
S31508023B6080B582B000AF78600B467B807B881A46A8
S31508023B70796804480EF02DFB034618460837BD46F9
S31508023B8080BD00BF6CCE002080B582B000AF7860E1
S31508023B90796804480EF02EFB03469BB2184608378E
S31508023BA0BD4680BD6CCE002080B582B000AF002332
S31508023BB0FB7115F01BFF3860386817F011FC0346D5
S31508023BC0002B18D01D4B1B68643B1C4A13601B4B09
S31508023BD01B68002B2CD11A481DF0CEFB142138681D
S31508023BE017F0FDF8386817F00EF90346134A136002
S31508023BF00123FB711CE0386818F0D3F80346B3F5C5
S31508023C00FA7F06D3386818F0CCF80346B3F52F6F57
S31508023C1004D31421386817F0E2F803E00A21386859
S31508023C2017F0DDF8386817F0EEF80346034A136012
S31508023C30FB7918460837BD4680BD00BF0000002044
S31508023C4020C30508F0B597B004AFBA607B60034697
S31508023C50FB730B46BB73012387F83430FB7B87F86B
S31508023C603530BB7B87F83630BB68BB637B68FB6342
S31508023C7097F8603087F8403097F8643087F8413013
S31508023C8097F8683087F8423097F86C3087F84630EC
S31508023C9097F835301D4697F836301E46BB6BFA6BD9
S31508023CA097F8401097F84200044607F1100003946B
S31508023CB002910192009333462A46114934F062FD75
S31508023CC007F1100318461DF057FB15F08FFE034641
S31508023CD0184619F001F90346012B06D115F086FE9E
S31508023CE003460021184619F005F907F13403142191
S31508023CF01846FFF735FF00BF4C37BD46F0BD00BF7B
S31508023D0044C30508F0B599B006AFBA607B600346AE
S31508023D10FB730B46BB73062387F83430FB7B87F8A5
S31508023D203530BB7B87F83630BB68BB637B68FB6381
S31508023D3097F8603087F8403097F8643087F8413052
S31508023D4097F8683087F84230B7F86C30A7F84430ED
S31508023D5097F835301E4697F836309C46BB6BFA6B99
S31508023D6097F8401097F842000446B7F8440005460B
S31508023D7007F1100004950394029101920093634699
S31508023D803246114934F0FEFC07F1100318461DF0BD
S31508023D90F3FA15F02BFE0346184619F09DF803466A
S31508023DA0012B06D115F022FE03460021184619F00A
S31508023DB0A1F807F1340314211846FFF7D1FE00BF14
S31508023DC04C37BD46F0BD00BF60C3050880B588B054
S31508023DD000AF0346FB7102233B73FB797B73002317
S31508023DE03B6100237B6107F10C0314211846FFF798
S31508023DF0B7FE00BF2037BD4680BD80B588B000AF8C
S31508023E0003460A46FB711346BB710B233B73FB79C8
S31508023E107B73BB79BB7607F10C0314211846FFF7AF
S31508023E209FFE00BF2037BD4680BD80B58AB000AF71
S31508023E300346B9607A60FB7303233B75FB7B7B758C
S31508023E40BB68BB617B68FB6115F0D0FD034618466B
S31508023E5019F042F80346012B06D115F0C7FD0346B1
S31508023E600021184619F046F807F1140314211846DA
S31508023E70FFF776FE00BF2837BD4680BD80B588B0FD
S31508023E8000AF0346FB7104233B73FB797B73002364
S31508023E903B6100237B6107F10C0314211846FFF7E7
S31508023EA05FFE00BF2037BD4680BD80B588B000AF33
S31508023EB003463960FB7105233B73FB797B73002349
S31508023EC03B613B687B6107F10C0314211846FFF737
S31508023ED047FE00BF2037BD4680BD000080B590B0C2
S31508023EE000AF03460A46FB711346BB71072387F8E0
S31508023EF02C30FB7987F82D30BB793B6300237B6333
S31508023F0097F82D301A463B6B07F10C00084934F036
S31508023F1039FC07F10C0318461DF02EFA07F12C039B
S31508023F2014211846FFF71CFE00BF4037BD4680BD68
S31508023F3080C3050890B593B002AF044608461146F9
S31508023F401A462346FB710346BB710B467B71134621
S31508023F507B80092387F82C30FB7987F82D300023DC
S31508023F603B6300237B63BB7987F838307B7987F814
S31508023F702E307B88BB8797F82D30194697F838304C
S31508023F801C4697F82E30BA8F07F10C00019200935F
S31508023F9023460A46084934F0F5FB07F10C0318468E
S31508023FA01DF0EAF907F12C0314211846FFF7D8FD8C
S31508023FB000BF4437BD4690BD90C3050880B590B092
S31508023FC000AF03460A46FB711346BB710A2387F8FC
S31508023FD02C30FB7987F82D3000233B6300237B6363
S31508023FE0002387F83830BB7987F82E3097F82D30BA
S31508023FF01A4697F82E3007F10C00094934F0C2FB2D
S3150802400007F10C0318461DF0B7F907F12C03142122
S315080240101846FFF7A5FD00BF4037BD4680BD00BF65
S31508024020A4C3050880B588B000AF03460A46FB71EB
S315080240301346BB7108233B73FB797B73BB793B61E0
S3150802404000237B6107F10C0314211846FFF788FD4C
S3150802405000BF2037BD4680BD80B400AF00BFBD4655
S315080240605DF8047B7047000080B582B000AF15F09A
S31508024070BDFC7860194B1B78043B092B20D801A29A
S3150802408052F823F0AD400208AD400208AD400208DE
S31508024090AD400208C1400208B7400208AD40020816
S315080240A0C1400208AD400208AD4002080121786805
S315080240B017F086FB09E00021786817F081FB04E017
S315080240C00021786817F07CFB00BF054B1B78022B92
S315080240D000BF00BF0837BD4680BD00BF6DCF0020B8
S315080240E06CCF002080B483B000AF0346FB71054A4B
S315080240F0FB791370012318460C37BD465DF8047B1D
S31508024100704700BFF3CF002080B483B000AF0346E8
S31508024110FB71054AFB791370012318460C37BD4615
S315080241205DF8047B704700BFF2CF002080B582B0ED
S3150802413000AF0023FB71B14B1B78052B00F27B8184
S3150802414001A252F823F000BF614102088B4102081E
S315080241509D420208C7420208EB42020815440208B9
S31508024160A7481DF0DDF9A7481DF0DAF9A64B40F677
S31508024170C4121A600023FB7114F0A0F89F4B1B7837
S315080241800133DAB29D4B1A706BE19F4B1B68002B09
S3150802419069DD9D4B1B68C3F51C630433B3F5487F81
S315080241A01EDB15F023FC0346184615F0ADFC034644
S315080241B0184616F040F90346002B03D15A2014F08C
S315080241C093F80DE015F012FC0346184615F09CFC10
S315080241D00346184616F02FF90346184614F084F8D3
S315080241E0894B1B68643B884A136014F049FE0346F0
S315080241F0FB71FB79032B36D801A252F823F000BFD4
S3150802420011420208234202082F4202083B420208D0
S3150802421064202DF05FFD7C4B1B68643B7A4A136071
S3150802422021E0794B1B68643B774A13601BE0764BA7
S315080242301B68C83B744A136015E0734B00221A6068
S315080242406E4B1B780133DAB26C4B1A7014F076F89F
S315080242504FF4FA702DF03EFD14F062F86A4B40F600
S31508024260C4121A6000BF684B1B68002B00F3F0806B
S3150802427066481DF055F9614BFF221A7014F05EF874
S315080242804FF4FA702DF026FD14F04AF815F0AEFB3D
S3150802429003460021184618F00DFAD9E05A4B1B6856
S315080242A0002B04DD584B1B68643B574A1360564B78
S315080242B01B68002B40F0CE80504B1B780133DAB2D4
S315080242C04E4B1A70C6E052481DF02AF913F0C4FF85
S315080242D04D4B40F6C4121A600023FB71474B1B78FC
S315080242E00133DAB2454B1A70BBE0474B1B68002B09
S315080242F069DD454B1B68C3F51C630433B3F52F7F91
S315080243001EDB15F073FB0346184615F0FDFB034644
S31508024310184616F090F80346002B03D15A2013F0DC
S31508024320B1FF0DE015F062FB0346184615F0ECFBEB
S315080243300346184616F07FF80346184613F0A2FFFE
S31508024340314B1B68643B304A136014F0CDFE0346BA
S31508024350FB71FB79032B36D801A252F823F000BF72
S3150802436071430208834302088F4302089B430208EB
S315080243700A202DF0AFFC244B1B680A3B224A136025
S3150802438021E0214B1B680A3B1F4A13601BE01E4BA8
S315080243901B68143B1C4A136015E01B4B00221A606B
S315080243A0164B1B780133DAB2144B1A7013F0C6FF98
S315080243B04FF4FA702DF08EFC13F0B2FF124B40F652
S315080243C0C4121A6000BF104B1B68002B44DC0F484E
S315080243D01DF0A6F8094BFF221A7013F0AFFF4FF42F
S315080243E0FA702DF077FC13F09BFF15F0FFFA0346DF
S315080243F00021184618F05EF92EE000BFF2CF002021
S31508024400B0C30508C0C3050804000020D0C30508C8
S31508024410DCC30508154B1B68002B04DD134B1B6810
S31508024420643B124A1360114B1B68002B16D1104BC2
S3150802443000221A7012E015F0D9FA0346184618F047
S315080244402CF90346002B0BD0094B00221A7007E001
S3150802445000BF06E000BF04E000BF02E000BF00E0C4
S3150802446000BF00BF0837BD4680BD00BF040000205C
S31508024470F2CF002090B5B3B000AFF860B96011462C
S315080244801A460B46FB711346BB710023C7F8C430A4
S315080244900023C7F8A8300023C7F8C0300023C7F89E
S315080244A0BC300023C7F8B8300023C7F8A43001236C
S315080244B087F89730BB684FF47A7202FB03F3C7F8A2
S315080244C0B43015F093FAC7F8A000DC4B00221A6044
S315080244D0002387F8B3300023C7F8AC300021D7F899
S315080244E0A00018F0BEFCFFF7B7FD64202DF0F2FB22
S315080244F097F8DC30002B24D1D14B00221A70D14B0D
S3150802450001221A7007F15403022118462FF006FBFE
S3150802451007F1100207F15403114618462FF069FBFA
S3150802452007F1100318462FF017FB044607F110038C
S3150802453018462FF01DFB03461A462146C24831F09B
S31508024540B1FD14F09DFC0346032B15D013F0B6FEFD
S31508024550002014F0D3FC0346002B05D1BB481CF0FF
S315080245600BFF012387F8B33013F0E8FE4FF4FA7015
S315080245702DF0B0FB13F0D4FE97F8B330002B2FD0F2
S3150802458013F06AFE002014F0EDFD0346002B02D15B
S31508024590AF481CF0F1FE13F0D1FE4FF4FA702DF07D
S315080245A099FB13F0BDFE13F089FE012014F0A6FC58
S315080245B00346002B0CD1A5481CF0DEFE0B2387F818
S315080245C0973015F013FA03460A21184617F098FD94
S315080245D013F0B4FE4FF4FA702DF07CFB13F0A0FE34
S315080245E097F897300B2B04D1FFF73EFD97F89730D3
S315080245F0BAE30CF06FF964202DF06CFB07F1970310
S31508024600184603F029FA0CF091F9F0EE407AFDEE1D
S31508024610E77A17EE903AC7F8C430D7F8C43013F1E0
S31508024620050F03DBD7F8C430052B7DDD89481CF05E
S3150802463077FF64202DF04EFB0CF04CF94FF4FA701C
S315080246402DF048FB0CF072F9F0EE407AFDEEE77AAF
S3150802465017EE903AC7F8C430D7F8C43013F1050FED
S3150802466003DBD7F8C430052B5EDD64202DF032FB60
S315080246700CF030F94FF4FA702DF02CFB0CF056F9C9
S31508024680F0EE407AFDEEE77A17EE903AC7F8C430B4
S31508024690D7F8C43013F1050F03DBD7F8C430052B5E
S315080246A042DD13F0D9FD002014F05CFD0346002B11
S315080246B002D169481CF060FE13F040FE4FF4FA700E
S315080246C02DF008FB13F02CFE13F0F8FD002014F071
S315080246D015FC0346002B0CD160481CF04DFE0B233B
S315080246E087F8973015F082F903460A21184617F01B
S315080246F007FD13F023FE4FF4FA702DF0EBFA13F0D0
S315080247000FFE64202DF0E6FA0CF0E4F84FF4FA7086
S315080247102DF0E0FA0CF00AF9F0EE407AFDEEE77AAF
S3150802472017EE903AC7F8C43097F897300B2B04D196
S31508024730FFF79AFC97F8973016E307F15803D7F86C
S31508024740C4204749184634F01DF807F1580318469D
S315080247501CF012FED7F8A00018F094FB0446FFF7E7
S315080247607DF80346E31A002BB8BF5B4242F22732B2
S31508024770934213DDD7F8A00018F084FB0346002BFA
S315080247800CD0FB684FF47A7202FB03F3354A82FBBC
S3150802479003125211DB17D31AC7F8AC3013F0CEFD49
S315080247A00121D7F8A00017F019F90121D7F8A000BE
S315080247B017F006F80023C7F89C30D7F8AC30002B60
S315080247C00BD002E001202DF085FAD7F8AC305A1E3C
S315080247D0C7F8AC20022BF5D8A0E00A202DF07AFA09
S315080247E00CF0A4F8F0EE407AFDEEE77A17EE903A6E
S315080247F0C7F8A830D7F8A820D7F8C430D31AC7F80C
S31508024800C030D7F8A00017F0F5FE03461A46FB6833
S315080248101344C7F89C30D7F8C020D7F89C309A4280
S3150802482024DBD7F8C030002B20DDFB68D7F89C20A4
S31508024830D7F8C0100C481CF073FE28E0F4CF00200D
S31508024840721F0120701F01200700080014C4050802
S315080248502CC4050844C4050858C4050874C40508C8
S3150802486090C4050867666666A0C40508FB68D7F89B
S315080248709C20D7F8C010B8481CF052FED7F8B430BE
S31508024880643BC7F8B430D7F8B430002BA5DCD7F8A8
S31508024890B430002B42DCD7F8C0309BB21946D7F8A1
S315080248A0A00017F096FE14F0EBFA0346032B0BD082
S315080248B0AA481CF061FD0C21D7F8A00017F020FCCD
S315080248C0022387F8973029E0D7F8A00017F069FA8B
S315080248D00346B3F5C87F0BD2A1481CF04DFD0B2148
S315080248E0D7F8A00017F00CFC022387F8973015E0DA
S315080248F097F8D830002B06D09A481CF03DFD1323B2
S3150802490087F897300AE098481CF036FD0D21D7F84B
S31508024910A00017F0F5FB022387F8973013F000FD85
S315080249200021D7F8A00017F059F84FF4FA702DF0C5
S31508024930D1F90023C7F8BC300023C7F8B83040F6CF
S31508024940B833C7F8B4300A202DF0C4F90BF0EEFFDD
S31508024950F0EE407AFDEEE77A17EE903AC7F8A830FD
S31508024960D7F8A81081481CF0DBFDD7F8A820D7F89D
S31508024970C430D31AC7F8C030D7F8C0107C481CF028
S31508024980CFFDD7F8BC20D7F8C0309A4209D1D7F85C
S31508024990B8300133C7F8B830D7F8B830012B07DD7D
S315080249A00FE0D7F8C030C7F8BC300023C7F8B830D4
S315080249B0D7F8B430643BC7F8B430D7F8B430002B14
S315080249C0C1DCD7F8AC30002B05D0FB68C7F8C0307D
S315080249D00023C7F8AC30D7F8C0309BB21946D7F8CF
S315080249E0A00017F0F6FDD7F8C0309BB21946D7F8E3
S315080249F0A00017F02CFAD7F8C00002F0F5F90BF070
S31508024A0035FFC7F8A400D7F8A430002B05D0D7F88D
S31508024A10A4306FF07F42934204D11C21D7F8A0003C
S31508024A2017F06EFB07F15800D7F8A430D7F8C02064
S31508024A30504933F0A7FE07F1580318461CF09CFCB0
S31508024A40D7F8A00017F0ADF903461A4607F158033E
S31508024A504949184633F096FE07F1580318461CF0E2
S31508024A608BFCD7F8C030002B06DD444B1A68D7F802
S31508024A70C0301344414A1360FEF760FF0346052B14
S31508024A802CD10023C7F89830D7F8A00015F03CF8C7
S31508024A900346184615F0A8F803461A46D7F8C03052
S31508024AA093FBF2F3C7F89830D7F89810D7F8A00016
S31508024AB016F090FAD7F8A00016F06BFA0346304AB9
S31508024AC0A2FB03239A0B07F158032E49184633F023
S31508024AD059FE07F1580318461CF04EFC2A4B1A6871
S31508024AE0D7F8C0301344284A136097F8DC30002BF5
S31508024AF050D147F23053C7F8B43012E0D7F8B43081
S31508024B00643BC7F8B430D7F8B430002B06DC1F482C
S31508024B101CF032FC0E2387F8973006E064202DF04D
S31508024B20D9F81B4B1B78002BE8D097F897300E2B39
S31508024B3004D10F21D7F8A00017F0E2FA97F89730B8
S31508024B400E2B03D097F897300D2B23D1FFF78CFA4B
S31508024B5097F8973008E100BFB8C40508D4C4050819
S31508024B60ECC405080CC5050824C5050838C505089A
S31508024B704CC5050860C5050874C50508E4CF0020BC
S31508024B8073B2E74580C50508F4CF002098C5050825
S31508024B90721F012064202DF09DF8002387F8B33098
S31508024BA013F05AFB002014F0DDFA0346002B05D158
S31508024BB0012387F8B3306E481CF0DEFB13F0BEFB08
S31508024BC04FF4FA702DF086F813F0AAFB97F8B33073
S31508024BD0002B2DD013F072FB002014F08FF9034638
S31508024BE0002B02D163481CF0C7FB13F0A7FB4FF456
S31508024BF0FA702DF06FF813F093FB13F02DFB0120DA
S31508024C0014F0B0FA0346002B0AD159481CF0B4FB3B
S31508024C100B2387F897300A21D7F8A00017F070FA05
S31508024C2013F08CFB4FF4FA702DF054F813F078FB5E
S31508024C300BF01CFEC7F8A400D7F8A410D7F8A000FA
S31508024C4018F02DF9D7F8A430002B05D0D7F8A430E0
S31508024C506FF07F42934204D11C21D7F8A00017F0C7
S31508024C604FFA07F15803D7F8A4204349184633F0F8
S31508024C7089FD07F1580318461CF07EFB97F8DC30CD
S31508024C80002B52D13D4B00221A703D4B01221A705D
S31508024C9007F15403012118462EF040FF07F11002CE
S31508024CA007F15403114618462EF0A3FF07F1100325
S31508024CB018462EF051FF044607F1100318462EF047
S31508024CC057FF03461A4621462E4831F0EBF947F2BA
S31508024CD03053C7F8B43017E0D7F8B430643BC7F896
S31508024CE0B430D7F8B430002B0BDC27481CF044FB51
S31508024CF00E2387F897300E21D7F8A00017F000FA8E
S31508024D0006E064202CF0E6FF1C4B1B78002BE3D050
S31508024D1097F897300E2B03D097F897300D2B04D1BE
S31508024D20FFF7A2F997F897301EE013F0C7FA0020AA
S31508024D3014F0E4F80346002B0AD10E481CF01CFBBB
S31508024D400A21D7F8A00017F0DBF90B2387F897306A
S31508024D5013F0F4FA4FF4FA702CF0BCFF13F0E0FAF1
S31508024D60FFF782F997F897301846CC37BD4690BDBB
S31508024D7058C4050874C40508BCC50508731F012074
S31508024D80711F01200700080098C5050800000000E9
S31508024D90B0B5B4B000AFF860B96011461A460B4612
S31508024DA0FB711346BB710023C7F8CC300023C7F842
S31508024DB0AC300023C7F8C8300023C7F8C430002334
S31508024DC087F8AB30002387F8C3300023C7F8BC3016
S31508024DD00023C7F8B830002387F8B7300023C7F88E
S31508024DE0A430012387F89730BB684FF47A7202FB26
S31508024DF003F3C7F8B03014F0F9FDC7F8A000B54BB5
S31508024E0000221A600023C7F89C30B34B00221A709E
S31508024E100021D7F8A00018F024F8B04B00221A6037
S31508024E20AF4B00221A60AF4B00221A60AE4B00222B
S31508024E301A70FB68B3F5B47F02DD022301F06FB87E
S31508024E40FFF70AF90A202CF045FFA64AFB68136009
S31508024E50A64B00221A70A64B01221A7007F15403B8
S31508024E60022118462EF05AFE07F1100207F15403E2
S31508024E70114618462EF0BDFE07F1100318462EF00D
S31508024E806BFE044607F1100318462EF071FE034620
S31508024E901A462146974831F005F9FB68962B06DC37
S31508024EA08E4AFB6813608C4B01221A7010E0FB686D
S31508024EB0962B06DDFB68FA2B03DC884B64221A6004
S31508024EC006E0FB68DA0F13445B101A46834B1A6036
S31508024ED013F0D6FF034687F8AB3097F8AB30032BAF
S31508024EE015D013F0EBF9002014F008F80346002B4E
S31508024EF005D181481CF040FA012387F8B73013F030
S31508024F001DFA4FF4FA702CF0E5FE13F009FA97F839
S31508024F10B730002B2ED013F09FF9002014F022F997
S31508024F200346002B02D175481CF026FA13F006FA3E
S31508024F3064202CF0CFFE13F0F3F913F0BFF9012029
S31508024F4013F0DCFF0346002B0CD16D481CF014FA53
S31508024F500B2387F8973014F049FD03460A211846B1
S31508024F6017F0CEF813F0EAF94FF4FA702CF0B2FE05
S31508024F7013F0D6F997F897300B2B05D1FFF774F88B
S31508024F8097F8973000F0CBBF0BF0A4FC64202CF006
S31508024F90A1FE07F19703184602F05EFD0BF0C6FC68
S31508024FA0F0EE407AFDEEE77A17EE903AC7F8CC3083
S31508024FB0D7F8CC3013F1050F03DBD7F8CC30052B25
S31508024FC07DDD50481CF0ACFA64202CF083FE0BF011
S31508024FD081FC4FF4FA702CF07DFE0BF0A7FCF0EE84
S31508024FE0407AFDEEE77A17EE903AC7F8CC30D7F852
S31508024FF0CC3013F1050F03DBD7F8CC30052B5EDD79
S3150802500064202CF067FE0BF065FC4FF4FA702CF066
S3150802501061FE0BF08BFCF0EE407AFDEEE77A17EEB6
S31508025020903AC7F8CC30D7F8CC3013F1050F03DB2A
S31508025030D7F8CC30052B42DD13F00EF9002014F018
S3150802504091F80346002B02D12C481CF095F913F06F
S3150802505075F94FF4FA702CF03DFE13F061F913F06E
S315080250602DF9002013F04AFF0346002B0CD12448E1
S315080250701CF082F90B2387F8973014F0B7FC034625
S315080250800A21184617F03CF813F058F94FF4FA704B
S315080250902CF020FE13F044F964202CF01BFE0BF0D2
S315080250A019FC4FF4FA702CF015FE0BF03FFCF0EEEB
S315080250B0407AFDEEE77A17EE903AC7F8CC3097F8C1
S315080250C097300B2B20D1FEF7CFFF97F8973000F0D9
S315080250D026BF00BFF8CF0020FCCF002000D000205A
S315080250E004D0002008D000200CD00020721F012016
S315080250F0701F012007000800CCC5050858C405081A
S3150802510074C4050844C4050807F15803D7F8CC2027
S315080251108F49184633F036FB07F1580318461CF038
S315080251202BF9D7F8A00017F0ADFE0446FEF796FB5A
S315080251300346E31A002BB8BF5B4242F22732934278
S3150802514014DDD7F8A00017F09DFE0346002B0DD0FC
S31508025150804B1B684FF47A7202FB03F37E4A82FB8A
S3150802516003125211DB17D31AC7F8BC3013F0E6F84C
S315080251700121D7F8A00016F031FC0121D7F8A000CA
S3150802518016F01EFB0023C7F89830D7F8BC30002B60
S315080251900BD002E001202CF09DFDD7F8BC305A1E38
S315080251A0C7F8BC20022BF5D88FE00A202CF092FD16
S315080251B00BF0BCFBF0EE407AFDEEE77A17EE903A7A
S315080251C0C7F8AC30D7F8AC20D7F8CC30D31AC7F822
S315080251D0B830D7F8A00017F00DFA03461A465D4B09
S315080251E01B681344C7F89830D7F8B820D7F8983010
S315080251F09A420CDBD7F8B830002B08DDFB68D7F8E3
S315080252009820D7F8B81055481CF08AF910E0FB68C0
S31508025210D7F89820D7F8B81051481CF081F9D7F872
S31508025220B030643BC7F8B030D7F8B030002BBCDCDE
S31508025230D7F8B030002B48DCD7F8B8309BB21946FD
S31508025240D7F8A00017F0C5F913F01AFE0346032B88
S315080252500DD044481CF090F814F0C8FB03460C2104
S31508025260184616F04DFF022387F897302DE0D7F837
S31508025270A00016F096FD0346B3F5C87F0DD23A484C
S315080252801CF07AF814F0B2FB03460B21184616F006
S3150802529037FF022387F8973017E097F8E030002B9C
S315080252A006D032481CF068F8132387F897300CE0CA
S315080252B02F481CF061F814F099FB03460D21184695
S315080252C016F01EFF022387F8973013F029F80021FB
S315080252D0D7F8A00016F082FB4FF4FA702CF0FAFC0D
S315080252E00023C7F8C8300023C7F8C43041F2883310
S315080252F0C7F8B0300A202CF0EDFC0BF017FBF0EEE5
S31508025300407AFDEEE77A17EE903AC7F8AC30D7F84E
S31508025310AC1018481CF004F9D7F8AC20D7F8CC30F2
S31508025320D31AC7F8B830D7F8B81013481CF0F8F8EB
S31508025330D7F8C820D7F8B8309A421FD1D7F8C43060
S315080253400133C7F8C430D7F8C430032B1DDD25E076
S31508025350F4C5050800D0002067666666A0C405087D
S31508025360B8C4050804C605081CC605083CC60508CF
S3150802537054C6050838C505084CC50508D7F8B83017
S31508025380C7F8C8300023C7F8C430D7F8B030643B32
S31508025390C7F8B030D7F8B030002BABDCD7F8BC3042
S315080253A0002B0CD0B64B1B68C7F8B8300023C7F8D9
S315080253B0BC30B44B1B780133DAB2B24B1A70D7F849
S315080253C0B8309BB21946D7F8A00017F002F9D7F8F9
S315080253D0B8309BB21946D7F8A00016F038FDD7F8B0
S315080253E0B80001F001FD0BF041FAC7F8A400D7F89E
S315080253F0A430002B05D0D7F8A4306FF07F42934231
S3150802540004D11C21D7F8A00016F07AFE07F158003D
S31508025410D7F8A430D7F8B8209B4933F0B3F907F187
S31508025420580318461BF0A8FFD7F8A00016F0B9FCD7
S3150802543003461A4607F158039449184633F0A2F967
S3150802544007F1580318461BF097FFFEF777FA03464B
S31508025450052B2CD10023C7F89C30D7F8A00014F0EE
S3150802546053FB0346184614F0BFFB03461A46D7F801
S31508025470B83093FBF2F3C7F89C30D7F89C10D7F8EC
S31508025480A00015F0A7FDD7F8A00015F082FD034687
S315080254907F4AA2FB03239A0B07F158037D49184654
S315080254A033F070F907F1580318461BF065FFD7F871
S315080254B0B830002B06DD784B1A68D7F8B830134493
S315080254C0754A1360754B1A68D7F8B8301344734A8D
S315080254D0136047F23053C7F8B03012E0D7F8B0304D
S315080254E0643BC7F8B030D7F8B030002B06DC6C48FE
S315080254F01BF042FF0E2387F8973006E064202CF053
S31508025500E9FB684B1B78002BE8D097F897300E2BEF
S3150802551004D10F21D7F8A00016F0F2FD97F89730BC
S315080255200E2B03D097F897300D2B05D1FEF79CFD6D
S3150802553097F8973000F0F3BC002387F8B73013F0DA
S31508025540D3FD0346032B14D012F086FE002013F077
S3150802555009FE0346002B05D1012387F8B7305248C6
S315080255601BF00AFF12F0EAFE64202CF0B3FB12F0DD
S31508025570D7FE002387F8C330A9E097F8B730002B87
S3150802558000F0A08012F09AFE002013F0B7FC034642
S31508025590002B02D145481BF0EFFE12F0CFFE4FF466
S315080255A0FA702CF097FB12F0BBFE12F055FE0120A2
S315080255B013F0D8FD0346002B7AD13B481BF0DCFEDC
S315080255C097F8C330022B76D1D7F8A00014F09CFACC
S315080255D00346184614F065FE03461A464FF6FF734D
S315080255E09A4208D10B2387F897300A21D7F8A000E8
S315080255F016F086FD5FE0D7F8A00017F025FC0346F3
S315080256001C46D7F8A00014F07FFA0346184614F091
S3150802561048FE034603F5FA739C4223DCD7F8A0003A
S3150802562017F012FC03461846FBF7B0F804460D4677
S31508025630D7F8A00014F068FA0346184614F031FEAB
S3150802564003461846FBF7A2F80BA3D3E90023FBF798
S3150802565007F902460B4620462946FBF787FB03460F
S31508025660002B28D10B2387F897300A21D7F8A000F8
S3150802567016F046FD1FE000BF666666666666E63F8A
S3150802568000D000200CD0002060C5050874C50508A6
S3150802569073B2E74580C50508E4CF0020F8CF00209D
S315080256A098C50508721F012058C4050874C4050860
S315080256B0002387F8B73012F041FE64202CF00AFB6B
S315080256C012F02EFE97F8C330013387F8C33097F8E5
S315080256D0C330022B7FF651AF0BF0C8F8C7F8A40007
S315080256E0D7F8A410D7F8A00017F0D9FBD7F8A4303A
S315080256F0002B05D0D7F8A4306FF07F42934204D12D
S315080257001C21D7F8A00016F0FBFC07F15803D7F8BE
S31508025710A420C849184633F035F807F15803184645
S315080257201BF02AFE97F897300B2B04D1FEF79CFC48
S3150802573097F89730F3E397F89730022B03D097F848
S315080257409730132B04D1FEF78FFC97F89730E6E3D0
S31508025750FB68962B40F39E83FA68D7F8B830D31ABB
S31508025760B54A1360BB684FF47A7202FB03F3C7F8B3
S31508025770B030002387F8B730002387F8AB3013F030
S315080257807FFB034687F8AB3097F8AB30032B15D06F
S3150802579012F094FD002013F0B1FB0346002B05D14D
S315080257A0012387F8B730A5481BF0E6FD12F0C6FDBF
S315080257B04FF4FA702CF08EFA12F0B2FD97F8B73061
S315080257C0002B2ED012F048FD002013F0CBFC034626
S315080257D0002B02D19A481BF0CFFD12F0AFFD6420D0
S315080257E02CF078FA12F09CFD12F068FD012013F0F5
S315080257F085FB0346002B0CD190481BF0BDFD0B23FD
S3150802580087F8973014F0F2F803460A21184616F07C
S3150802581077FC12F093FD4FF4FA702CF05BFA12F053
S315080258207FFD97F897300B2B04D1FEF71DFC97F8EE
S31508025830973074E30BF04EF864202CF04BFA07F11C
S315080258409703184602F008F90BF070F8F0EE407A62
S31508025850FDEEE77A17EE903AC7F8CC30D7F8CC3097
S3150802586013F1050F03DBD7F8CC30052B7DDD754820
S315080258701BF056FE64202CF02DFA0BF02BF84FF491
S31508025880FA702CF027FA0BF051F8F0EE407AFDEE9A
S31508025890E77A17EE903AC7F8CC30D7F8CC3013F13E
S315080258A0050F03DBD7F8CC30052B5EDD64202CF020
S315080258B011FA0BF00FF84FF4FA702CF00BFA0BF002
S315080258C035F8F0EE407AFDEEE77A17EE903AC7F829
S315080258D0CC30D7F8CC3013F1050F03DBD7F8CC3030
S315080258E0052B42DD12F0B8FC002013F03BFC034600
S315080258F0002B02D152481BF03FFD12F01FFD4FF458
S31508025900FA702CF0E7F912F00BFD12F0D7FC002022
S3150802591013F0F4FA0346002B0CD148481BF02CFD71
S315080259200B2387F8973014F061F803460A211846C4
S3150802593016F0E6FB12F002FD4FF4FA702CF0CAF9E3
S3150802594012F0EEFC64202CF0C5F90AF0C3FF4FF4FE
S31508025950FA702CF0BFF90AF0E9FFF0EE407AFDEE94
S31508025960E77A17EE903AC7F8CC3097F897300B2BB0
S3150802597004D1FEF779FB97F89730D0E207F158037E
S31508025980D7F8CC203049184632F0FCFE07F1580306
S3150802599018461BF0F1FCD7F8A00017F073FA044674
S315080259A0FDF75CFF0346E31A002BB8BF5B4242F2DF
S315080259B02732934214DDD7F8A00017F063FA03469C
S315080259C0002B0DD0214B1B684FF47A7202FB03F3AE
S315080259D01F4A82FB03125211DB17D31AC7F8BC30CF
S315080259E012F0ACFC0121D7F8A00015F0F7FFD7F8A2
S315080259F0A00015F011FF0346002B02D164202CF0FB
S31508025A0069F90121D7F8A00015F0DAFE0023C7F8D4
S31508025A109830D7F8BC30002B1CD002E001202CF0BD
S31508025A2059F9D7F8BC305A1EC7F8BC20022BF5D84C
S31508025A30A0E000BFBCC5050804D0002074C4050850
S31508025A4058C4050844C4050890C4050800D00020B7
S31508025A50676666660A202CF03DF90AF067FFF0EEE3
S31508025A60407AFDEEE77A17EE903AC7F8AC30D7F8E7
S31508025A70AC20D7F8CC30D31AC7F8B830D7F8A0007C
S31508025A8016F0B8FD03461A46C84B1B681344C7F8F6
S31508025A909830D7F8B820D7F898309A420CDBD7F85E
S31508025AA0B830002B08DDFB68D7F89820D7F8B8106D
S31508025AB0BF481BF035FD10E0FB68D7F89820D7F8E9
S31508025AC0B810BC481BF02CFDD7F8B030643BC7F8B9
S31508025AD0B030D7F8B030002BBCDCD7F8B030002B8A
S31508025AE048DCD7F8B8309BB21946D7F8A00016F0AA
S31508025AF070FD13F0C5F90346032B0DD0AE481BF013
S31508025B003BFC13F073FF03460C21184616F0F8FA0D
S31508025B10022387F897302DE0D7F8A00016F041F94E
S31508025B200346B3F5C87F0DD2A4481BF025FC13F033
S31508025B305DFF03460B21184616F0E2FA022387F8A0
S31508025B40973017E097F8E030002B06D09C481BF0F8
S31508025B5013FC132387F897300CE09A481BF00CFCC9
S31508025B6013F044FF03460D21184616F0C9FA02231C
S31508025B7087F8973012F0D4FB0021D7F8A00015F069
S31508025B802DFF4FF4FA702CF0A5F80023C7F8C83099
S31508025B900023C7F8C43040F6B833C7F8B0300A2035
S31508025BA02CF098F80AF0C2FEF0EE407AFDEEE77A9B
S31508025BB017EE903AC7F8AC30D7F8AC1082481BF00B
S31508025BC0AFFCD7F8AC20D7F8CC30D31AC7F8B83020
S31508025BD0D7F8B8107D481BF0A3FCD7F8C820D7F829
S31508025BE0B8309A4209D1D7F8C4300133C7F8C4305D
S31508025BF0D7F8C430012B07DD0FE0D7F8B830C7F85D
S31508025C00C8300023C7F8C430D7F8B030643BC7F8A9
S31508025C10B030D7F8B030002BC1DCD7F8BC30002B37
S31508025C200CD0624B1B68C7F8B8300023C7F8BC30E3
S31508025C30674B1B780233DAB2654B1A70D7F8B8305D
S31508025C409BB21946D7F8A00016F0C3FCD7F8B830AD
S31508025C509BB21946D7F8A00016F0F9F8D7F8B8009B
S31508025C6001F0C2F80AF002FEC7F8A400D7F8A43079
S31508025C70002B05D0D7F8A4306FF07F42934204D1A7
S31508025C801C21D7F8A00016F03BFA07F15800D7F8FE
S31508025C90A430D7F8B8204F4932F074FD07F15803FB
S31508025CA018461BF069FBD7F8A00016F07AF80346E7
S31508025CB01A4607F158034849184632F063FD07F1B8
S31508025CC0580318461BF058FBD7F8B830002B06DDE8
S31508025CD0424B1A68D7F8B8301344404A1360404B0F
S31508025CE01A68D7F8B83013443D4A1360002387F878
S31508025CF0B73013F0F9F90346032B14D012F0ACFAB5
S31508025D00002013F02FFA0346002B05D1012387F84A
S31508025D10B73034481BF030FB12F010FB64202BF02E
S31508025D20D9FF12F0FDFA002387F8C330ADE097F8E1
S31508025D30B730002B00F0A48012F0C0FA002013F04E
S31508025D40DDF80346002B02D127481BF015FB12F09B
S31508025D50F5FA4FF4FA702BF0BDFF12F0E1FA12F0E1
S31508025D607BFA012013F0FEF90346002B7ED11D486B
S31508025D701BF002FB97F8C330022B7AD1D7F8A000A2
S31508025D8013F0C2FE0346184614F08BFA03461A4667
S31508025D904FF6FF739A4229D10B2387F897300A21C7
S31508025DA0D7F8A00016F0ACF963E000BF04D00020D3
S31508025DB0A0C40508B8C4050804C605081CC6050813
S31508025DC03CC6050854C6050838C505084CC5050865
S31508025DD00CD0002060C5050874C50508E4CF00206C
S31508025DE0F8CF002058C4050874C40508D7F8A000DF
S31508025DF017F02AF803461C46D7F8A00013F084FECB
S31508025E000346184614F04DFA034603F5FA739C4204
S31508025E1023DCD7F8A00017F017F803461846FAF756
S31508025E20B5FC04460D46D7F8A00013F06DFE0346EE
S31508025E30184614F036FA03461846FAF7A7FC3DA3A5
S31508025E40D3E90023FAF70CFD02460B4620462946FB
S31508025E50FAF78CFF0346002B0BD10B2387F89730F2
S31508025E600A21D7F8A00016F04BF902E0002387F8BA
S31508025E70B73012F063FA64202BF02CFF12F050FAB6
S31508025E8097F8C330013387F8C33097F8C330022B2B
S31508025E907FF64DAFFDF752FD0346052B2CD10023A5
S31508025EA0C7F89C30D7F8A00013F02EFE0346184612
S31508025EB013F09AFE03461A46D7F8B83093FBF2F364
S31508025EC0C7F89C30D7F89C10D7F8A00015F082F8CE
S31508025ED0D7F8A00015F05DF80346134AA2FB032380
S31508025EE09A0B07F158031149184632F04BFC07F191
S31508025EF0580318461BF040FA97F89730022B0AD037
S31508025F0097F89730132B06D0094B1B78002B02D033
S31508025F10152387F89730FEF7A7F897F897301846AB
S31508025F20D037BD46B0BD00BF73B2E74580C5050888
S31508025F300CD00020666666666666E63F00000000CC
S31508025F40B0B59CB000AF786039600023FB660023C9
S31508025F50FB650023BB660023BB65012387F84B302C
S31508025F603B684FF47A7202FB03F37B6613F03EFD3D
S31508025F707865002387F85330002387F86330C74BC8
S31508025F8000221A60002387F862300021786D16F025
S31508025F9068FFFEF761F80A202BF09CFE7B68002B4F
S31508025FA04EDD97F85330032B15D012F087F90020EF
S31508025FB012F0A4FF0346002B05D1B9481BF0DCF901
S31508025FC0012387F8633012F0B9F94FF4FA702BF00F
S31508025FD081FE12F0A5F997F86330002B32D012F041
S31508025FE03BF9002013F0BEF80346002B02D1AD4858
S31508025FF01BF0C2F912F0A2F94FF4FA702BF06AFEFE
S3150802600012F08EF912F05AF9012012F077FF0346C0
S31508026010002B0CD1A4481BF0AFF90B2387F84B30A1
S3150802602013F0E4FC03460A21184616F069F812F042
S3150802603085F94FF4FA702BF04DFE12F071F901E072
S3150802604012F00AF997F84B300B2B04D1FEF70CF82D
S3150802605097F84B3074E297F84B300E2B03D097F82B
S315080260604B300D2B04D1FDF7FFFF97F84B3067E253
S315080260707B68002B40F3A9800AF02CFC64202BF0E5
S3150802608029FE07F14B03184601F0E6FC0AF04EFC1E
S31508026090F0EE407AFDEEE77A17EE903AFB66FB6E73
S315080260A013F1050F02DBFB6E052B76DD7F481BF02D
S315080260B037FA64202BF00EFE0AF00CFC4FF4FA7045
S315080260C02BF008FE0AF032FCF0EE407AFDEEE77A93
S315080260D017EE903AFB66FB6E13F1050F02DBFB6EB9
S315080260E0052B5ADD64202BF0F5FD0AF0F3FB4FF47D
S315080260F0FA702BF0EFFD0AF019FCF0EE407AFDEE8D
S31508026100E77A17EE903AFB66FB6E13F1050F02DB90
S31508026110FB6E052B41DD12F09FF8002013F022F8E2
S315080261200346002B02D15F481BF026F912F006F946
S315080261304FF4FA702BF0CEFD12F0F2F812F0BEF818
S31508026140002012F0DBFE0346002B0CD156481BF04A
S3150802615013F90B2387F84B3013F048FC03460A2140
S31508026160184615F0CDFF12F0E9F84FF4FA702BF045
S31508026170B1FD12F0D5F864202BF0ACFD0AF0AAFBAB
S315080261804FF4FA702BF0A6FD0AF0D0FBF0EE407A37
S31508026190FDEEE77A17EE903AFB6697F84B300B2B33
S315080261A004D1FDF761FF97F84B30C9E107F10C03FB
S315080261B0FA6E3F49184632F0E5FA07F10C0318461B
S315080261C01BF0DAF844F620637B6612F0B7F8012171
S315080261D0786D15F003FC0121786D15F0F1FA7B68EC
S315080261E0002B1DDD0A202BF075FD0AF09FFBF0EE51
S315080261F0407AFDEEE77A17EE903AFB65FA6DFB6E8A
S31508026200D31ABB66786D16F0F5F903461A467B680B
S315080262101344BA6E9A4206DBBB6E002B03DD08E016
S3150802622064202BF057FD7B6E643B7B667B6E002BEE
S31508026230D5DC7B6E002B4EDC7B68002B4BDDBB6E00
S315080262409BB21946786D16F0C4F912F019FE034688
S31508026250032B0DD017481BF08FF813F0C7FB034624
S315080262600C21184615F04CFF022387F84B3032E012
S31508026270786D15F096FD0346B3F5C87F1ED20E4813
S315080262801BF07AF813F0B2FB03460B21184615F0F9
S3150802629037FF022387F84B301DE000BFF4CF0020FA
S315080262A0CCC5050858C4050874C4050844C40508BD
S315080262B090C4050804C605081CC60508A4481BF0B0
S315080262C05BF813F093FB03460D21184615F018FFE9
S315080262D0022387F84B3012F023F80021786D15F067
S315080262E07DFB4FF4C8702BF0F5FC7B68002B57DD5D
S315080262F0BB6E9BB21946786D16F06BF9BB6E9BB2F4
S315080263001946786D15F0A3FDB86E00F06DFD0AF01A
S31508026310ADFAB865BB6D002B04D0BB6D6FF07F423A
S31508026320934203D11C21786D15F0EAFE07F10C00A1
S31508026330BB6DBA6E874932F025FA07F10C03184687
S315080263401BF01AF8786D15F02CFD03461A4607F16C
S315080263500C038149184632F015FA07F10C03184660
S315080263601BF00AF87D4B1A68BB6E13447B4A13600E
S31508026370FDF7E4FA0346052B12D10023FB64786D78
S3150802638013F0C2FB0346184613F02EFC03461A46C0
S31508026390BB6E93FBF2F3FB64F96C786D14F01AFE8C
S315080263A0002387F8633012F09FFE0346032B15D0AD
S315080263B011F052FF002012F0D5FE0346002B05D13C
S315080263C0012387F8633066481AF0D6FF11F0B6FF44
S315080263D04FF4FA702BF07EFC11F0A2FF002387F827
S315080263E0623085E097F86330002B7CD011F066FFA7
S315080263F0002012F083FD0346002B02D159481AF0F9
S31508026400BBFF11F09BFF4FF4FA702BF063FC11F0FF
S3150802641087FF11F021FF012012F0A4FE0346002B8C
S3150802642056D14F481AF0A8FF97F86230022B52D17C
S31508026430786D13F069FB0346184613F032FF0346DC
S315080264401A464FF6FF739A4207D10B2387F84B3049
S315080264500A21786D15F054FE3DE0786D16F0F4FCCD
S3150802646003461C46786D13F04FFB0346184613F095
S3150802647018FF034603F5FA739C4221DC786D16F081
S31508026480E3FC03461846FAF781F904460D46786D89
S3150802649013F03AFB0346184613F003FF0346184661
S315080264A0FAF774F928A3D3E90023FAF7D9F90246C9
S315080264B00B4620462946FAF759FC0346002B0AD111
S315080264C00B2387F84B300A21786D15F019FE02E086
S315080264D0002387F8633011F031FF4FF4FA702BF07E
S315080264E0F9FB11F01DFF97F86230013387F8623025
S315080264F097F86230022B7FF675AF0AF0B7F9B865DE
S31508026500B96D786D16F0CBFCBB6D002B04D0BB6D54
S315080265106FF07F42934203D11C21786D15F0F0FD8E
S3150802652007F10C03BA6D1049184632F02BF907F138
S315080265300C0318461AF020FFFDF796FD97F84B3024
S3150802654018467037BD46B0BD666666666666E63F3D
S3150802655054C6050860C5050874C50508F4CF0020A9
S3150802656058C4050874C40508BCC5050880B586B0B4
S3150802657000AF0023BB750023FB750023FB7513F0E0
S3150802658035FA0346184613F0BFFA0346184613F0BF
S3150802659052FF0346BB7513F029FA0346184613F051
S315080265A0B3FA0246BB7D0A33DBB21946104613F02C
S315080265B031FF11F051FE002012F0D4FD0346002BE4
S315080265C005D145481AF0D8FEFB7D0133FB7511F05B
S315080265D0B5FE4FF4FA702BF07DFB11F06FFE00202A
S315080265E012F08CFC0346002B05D13C481AF0C4FE77
S315080265F0FB7D0233FB7511F0A1FE4FF4FA702BF006
S3150802660069FB11F029FE002012F0ACFD0346002BAF
S3150802661005D131481AF0B0FEFB7D0133FB7511F046
S315080266208DFE4FF4FA702BF055FB11F079FEFB7DC7
S31508026630002B0CD013F0DAF90346184613F064FA65
S315080266400346184613F0F7FE0346632B95D9FB7DDE
S31508026650002B3CD113F0CAF90346184613F054FA34
S315080266600346184613F0E7FE0346BB75BB7D4F2B60
S315080266700ED913F0BBF90346184613F045FA03463A
S315080266806421184613F0C6FE15481AF075FE19E07D
S3150802669013F0ACF90346184613F036FA0246BB7DE8
S315080266A01433DBB21946104613F0B4FEBB7D03F170
S315080266B014023B460B49184632F064F83B46184624
S315080266C01AF05AFEFDF790F807481AF055FE00BF71
S315080266D01837BD4680BD00BF68C605088CC60508C2
S315080266E0B0C60508C0C60508D0C6050880B582B07A
S315080266F000AF0346FB71FB79012B05D0FB79042B0E
S3150802670002D0FB79052B2DD111F0D8FD002012F00D
S31508026710F5FB0346002B02D144481AF02DFE11F070
S315080267200DFE4FF4FA702BF0D5FA11F0F9FD11F0BF
S3150802673093FD012012F016FD0346002B09D13C48B1
S315080267401AF01AFE13F052F903460A21184615F0F2
S31508026750D7FC11F0F3FD4FF4FA702BF0BBFA11F0E7
S31508026760DFFD5EE0FB79022B1AD111F0A7FD0120AD
S3150802677012F0C4FB0346002B09D12C481AF0FCFD83
S3150802678013F034F903460A21184615F0B9FC11F03C
S31508026790D5FD4FF4FA702BF09DFA11F0C1FD40E0D9
S315080267A013F024F90346184613F0AEF903460021FE
S315080267B0184613F02FFEFFF7D9FE11F04DFD002003
S315080267C012F0D0FC0346002B09D119481AF0D4FD61
S315080267D013F00CF903460A21184615F091FC11F03C
S315080267E0ADFD4FF4FA702BF075FA11F099FD11F020
S315080267F065FD002012F082FB0346002B09D10B48E7
S315080268001AF0BAFD13F0F2F803460A21184615F0F3
S3150802681077FC11F093FD4FF4FA702BF05BFA11F046
S315080268207FFD00BF0837BD4680BD00BF74C405089A
S3150802683058C4050880B588B000AF0023FB7700234B
S31508026840BB6113F0D3F80346184613F05DF9034605
S31508026850184613F0F0FD0346002B03D0954B1B7820
S31508026860002B75D012F00CFB0346032B1CD011F03B
S3150802687025FDFF2012F042FB0346002B0CD18E4861
S315080268801AF07AFD13F0B2F803460A21184615F0F3
S3150802689037FCFB7F0233FB7711F050FD4FF4FA7099
S315080268A02BF018FA11F03CFD12F01EFC0346032BDE
S315080268B01AD011F0D1FCFF2012F054FC0346002B2B
S315080268C00CD17E481AF058FD13F090F803460A21B7
S315080268D0184615F015FCFB7F0133FB7711F02EFDE8
S315080268E04FF4FA702BF0F6F911F0E8FCFF2012F0DB
S315080268F005FB0346002B0CD16F481AF03DFD13F039
S3150802690075F803460A21184615F0FAFBFB7F02338F
S31508026910FB7711F013FD4FF4FA702BF0DBF911F047
S31508026920FFFCFB7F002B13D1624B1B78002B0AD08E
S3150802693013F05CF80346184613F0E6F803460021FE
S31508026940184613F067FDFFF711FE5A4B00221A701C
S3150802695012F0CAFB0346032B13D011F07DFC00206C
S3150802696012F000FC0346002B05D154481AF004FD28
S31508026970FB7F0133FB7711F0E1FC4FF4FA702BF041
S31508026980A9F9FB7F002B12D113F030F803461846FB
S3150802699013F0BAF80346184613F083FC03461A4660
S315080269A04FF6FF739A4202D1454B01221A7011F033
S315080269B085FC002012F0A2FA0346002B05D13E48B8
S315080269C01AF0DAFCFB7F0233FB7711F0B7FC4FF4BF
S315080269D0FA702BF07FF911F0A3FC11F03DFC0020B0
S315080269E012F0C0FB0346002B05D134481AF0C4FC4A
S315080269F0FB7F0433FB7711F0A1FC4FF4FA702BF0FE
S31508026A0069F911F08DFCFB7F002B03D0FB7F18463A
S31508026A10FFF76CFE12F0EAFF0346184613F074F805
S31508026A200346184613F007FD03461A463B1D254939
S31508026A30184631F0A7FE3B1D18461AF09DFC09F0D0
S31508026A4015FFB861BB69002B04D0BB696FF07F42A2
S31508026A50934209D112F0CAFF03461C21184615F0C3
S31508026A604FFBFB7F0A33FB773B1DBA69164918466B
S31508026A7031F088FE3B1D18461AF07EFCFCF75EFFD5
S31508026A800346002B04D0FCF759FF0346012B0CD111
S31508026A9012F0ACFF03460121184614F091FE42F2A9
S31508026AA010702BF017F9FDF7DFFAFB7F184620372F
S31508026AB0BD4680BDDDD3002074C4050858C4050848
S31508026AC0E8CF0020C0C60508BCC5050880B584B055
S31508026AD000AF0346FB710023FB73FB79012B02D03F
S31508026AE0022B23D048E012F0FFFA0346032B40D0CC
S31508026AF011F0B2FB002012F035FB0346002B0CD135
S31508026B0020481AF039FC12F071FF03460A2118468A
S31508026B1015F0F6FAFB7B0133FB7311F00FFC4FF409
S31508026B20FA702BF0D7F811F0FBFB22E012F0A8F965
S31508026B300346032B1FD011F0C1FB002012F0DEF929
S31508026B400346002B0CD110481AF016FC12F04EFF21
S31508026B5003460A21184615F0D3FAFB7B0133FB7369
S31508026B6011F0ECFB4FF4FA702BF0B4F811F0D8FBE5
S31508026B7001E000BF00E000BFFB7B18461037BD46A8
S31508026B8080BD00BF58C4050874C4050890B5A7B0EF
S31508026B9002AF03460A46FB711346BB71012387F807
S31508026BA08F304FF00003C7F888304FF00003C7F85C
S31508026BB080300023C7F8843012F018FF03460021FC
S31508026BC0184616F04EF9002387F87F3012F00EFFAA
S31508026BD00246FB791946104615F01BFE87ED200A78
S31508026BE0FB79002B09D0FB79042B06D8012387F8F9
S31508026BF07F30D7F88030C7F88830D7F88800F9F799
S31508026C00D7FD02460B4607F15400654931F0BAFD35
S31508026C1007F1540318461AF0AFFB624B00221A70AA
S31508026C20614B01221A7007F15003012118462CF014
S31508026C3075FF07F10C0207F15003114618462CF0AE
S31508026C40D8FF07F10C0318462CF086FF044607F115
S31508026C500C0318462CF08CFF03461A462146534865
S31508026C602FF020FA47F23053C7F8843012E0D7F8EB
S31508026C708430643BC7F88430D7F88430002B06DCAE
S31508026C804B481AF079FB0D2387F88F3006E064200B
S31508026C902BF020F8434B1B78002BE8D097F88F305F
S31508026CA0012B02D097F88F3076E012F09FFE02464B
S31508026CB0FB791946104615F0ACFD87ED200A97EDCB
S31508026CC0207AD7ED227A77EE677A17EE900AF9F7E5
S31508026CD06FFD02460B463749096807F154000091D1
S31508026CE0354931F04FFD07F1540318461AF044FBB3
S31508026CF040F2DC502AF0EEFF304B00221A70304B7D
S31508026D0001221A7007F15003022118462CF006FFD9
S31508026D1007F10C0207F15003114618462CF069FFD9
S31508026D2007F10C0318462CF017FF044607F10C036B
S31508026D3018462CF01DFF03461A4621461B482FF01B
S31508026D40B1F947F23053C7F8843012E0D7F88430E5
S31508026D50643BC7F88430D7F88430002B06DC194820
S31508026D601AF00AFB0E2387F88F3006E064202AF011
S31508026D70B1FF124B1B78002BE8D097F88F30012B06
S31508026D8002D097F88F3007E00F4B00221A700F4B8C
S31508026D9000221A6097F88F3018469437BD4690BD80
S31508026DA0E0C60508731F0120711F012007000800AD
S31508026DB0F0C6050800D0002014C70508721F012076
S31508026DC0701F012098C50508FCCF0020F8CF0020C7
S31508026DD080B483B000AF0123FB71FB7918460C37E8
S31508026DE0BD465DF8047B704780B483B000AF786017
S31508026DF00C4B1B68002B0EDD0A4B1B687A689A42FD
S31508026E0003DD084B00221A6005E0064B1A687B6808
S31508026E10D31A044A136000BF0C37BD465DF8047BDB
S31508026E20704700BFECCF002080B582B000AF0346A2
S31508026E30FB8012F0DBFD0346184614F03FFA0346C0
S31508026E40002B26D0FA88164B1B681344144A136083
S31508026E50134B1B68194613481AF062FB104B1B6842
S31508026E60B3F5C87F18DD104B01221A702EF082F88E
S31508026E7003462222612118462EF0BAF80346002B51
S31508026E800AD112F0B3FD03462221184615F038F945
S31508026E9002E0034B00221A6000BF0837BD4680BDD8
S31508026EA0ECCF002028C70508F0CF002090B52DEDBD
S31508026EB0028B93B000AF4FF000037B6412F096FD8D
S31508026EC07863984B1B78002B00F07082FCF736FD2E
S31508026ED00346052B40F09980934B1B685A1C92492E
S31508026EE00A6040F6B832934240F29A808F4B93ED8D
S31508026EF0007A8F4BD3ED007AB4EE677AF1EE10FA88
S31508026F004ED08A4BD3ED007AF5EE407AF1EE10FABE
S31508026F1003D1874B4FF07E521A60854B1B68834A12
S31508026F201360844B1B68002B3AD0824B1B6807EE12
S31508026F30903AF8EE677AC7ED117A97ED117AF2EE82
S31508026F40046AC7EE267AC7ED117A784BD3ED006A42
S31508026F5097ED117AC6EE877AC7ED117AD7ED117ACF
S31508026F609FED757A67EE877AC7ED117AD7ED117AB2
S31508026F70FCEEE77A17EE903A9BB21946786B15F053
S31508026F80F2FDD7ED117AFCEEE77A3B4617EE902A28
S31508026F906A49184631F0F6FB3B4618461AF0ECF9F0
S31508026FA0614B1B6842F22832934220D9D7ED117AF7
S31508026FB0FCEEE77A17EE904A786B12F0A5FD0346C7
S31508026FC0184612F011FF03469C4210D9786B12F04C
S31508026FD09BFD0246D7ED117AFCEEE77A17EE903A58
S31508026FE09BB21946104612F0EFFEFCF7FDFB4F4B1B
S31508026FF0D3ED007AF5EEC07AF1EE10FA10DD4D4BBC
S315080270001B6801334B4A13600AE0484B4FF00002F3
S315080270101A60474B4FF000021A60464B00221A606C
S31508027020474B1B78042B00F2C38101A252F823F0C6
S3150802703045700208A1700208E97002085772020830
S31508027040B1730208786B14F0CBF90346002B40F0B3
S31508027050B18112F0CBFC0346184615F09BFF034696
S3150802706018462CF0DBFE0346022B00F0A3812EF015
S315080270707FFA034618462EF091FA0346002118466F
S315080270802CF0BDFE2F4B00221A600121786B14F0FA
S315080270906FFC2D481AF070F9294B01221A7089E102
S315080270A0284B1B685A1C27490A60284A12689342C9
S315080270B0C0F08281264B00221A6011F00FFB234B87
S315080270C002221A602EF054FA034618462EF066FA81
S315080270D00346022118462CF092FE1E481AF04CF975
S315080270E0174B02221A7067E1786B14F079F9034696
S315080270F0002B35D011F0FEFA174B184A1A60104BBE
S3150802710003221A702EF034FA034618462EF046FA6F
S315080271100346012118462CF072FE0A4B00221A6019
S315080271204CE100BFBCCF0020DCCF002010D00020ED
S3150802713014D0002018D000200000614534C7050885
S315080271406CCF00201CD000203CC705080800002090
S315080271508021012048C705080C0000207011010093
S315080271609A4B1B68643B994A1360984B1B68002B21
S3150802717040F0248111F006FB0121786B13F059FBCC
S315080271800021786B13F06EFA1221786B14F0B8FFAF
S315080271902EF0EEF9034618462EF000FA03460021B1
S315080271A018462CF02CFE8A481AF0E6F8894B042277
S315080271B01A70894B1A683B468849184631F0E2FA32
S315080271C03B4618461AF0D8F84FF000033B64824B48
S315080271D01B68022B13D9804B1B68023B07EE903AB9
S315080271E0B8EE678A786B12F08FFC0346184612F0DF
S315080271F0DFFEB0EE407AC8EE077AC7ED107A764B14
S315080272001B68092B40F2DA80786B12F07DFC034684
S31508027210184612F0CCFD0346002B09D1786B12F002
S3150802722073FC03460121184612F0B0FDFCF7DCFA9E
S315080272300121786B15F079FCD7ED107AB2EE047A53
S3150802724067EE877AFCEEE77A17EE903A9BB2184613
S3150802725010F02EFDB2E0624B1B685A1C60490A60A8
S31508027260092B40F2AD805B4B00221A704FF00003E7
S31508027270FB6300237B87584B1B68022B13D9564B9B
S315080272801B68023B07EE903AB8EE678A786B12F0F3
S315080272903BFC0346184612F08BFEB0EE407AC8EE67
S315080272A0077AC7ED0F7A4C4B1B68092B02D84B237A
S315080272B07B873CE0786B12F027FC0346184612F0EF
S315080272C076FD0346002B09D1786B12F01DFC0346A6
S315080272D00121184612F05AFDFCF786FA0121786B4D
S315080272E015F023FCD7ED0F7AFCEEE77A17EE903A03
S315080272F07B873C4B1B6840F6B832934209D93A4B16
S3150802730093ED007AD7ED0F7A77EE277A364BC3EDEF
S31508027310007AD7ED0F7AB2EE047A67EE877AFCEE38
S31508027320E77A17EE903A9BB2184610F0C1FCFCF7C2
S3150802733005FB0346052B0ED0FCF700FB0346062B7E
S3150802734009D0FCF7FBFA0346082B04D0FCF7F6FA39
S315080273500346072B0CD1254B00221A707B8F194640
S31508027360786B14F053FD7B8F1846FFF75DFD05E039
S315080273701E4B1B780133DAB21C4B1A701B4B1B7857
S31508027380022B03D90921786B14F0BAFE786B14F034
S3150802739008FD03461A46104B1B683846144931F055
S315080273A0F1F93B46184619F0E7FF09E000BF08E085
S315080273B000BF06E000BF04E000BF02E000BF00E035
S315080273C000BF4C37BD46BDEC028B90BD0C000020B9
S315080273D054C705086CCF00208021012064C7050820
S315080273E01CD00020DCCF002014D0002020D00020A2
S315080273F070C7050880B500AF12F0F8FA03461846BA
S3150802740014F03CFA0346002B11D00C4B1B88643B44
S315080274109AB20A4B1A80094B1B88002B0BD112F021
S31508027420E5FA03460021184614F004FA03E0034B72
S315080274304FF4FA521A8000BF80BD00BF1000002028
S3150802744080B582B000AF0023FB7112F0CFFA034673
S31508027450184614F013FA0346002B02D05023FB7188
S3150802746001E02823FB71FB7918460837BD4680BD23
S31508027470B0B582B000AF12F0B9FA78609A4B1B78B1
S31508027480002B40F08982994B1B78032B00F27F82EE
S3150802749001A252F823F000BFA97402085375020824
S315080274A0D57802087F790208786813F0BEFB03468E
S315080274B08F4A1360786813F0EDFB03468C4A5360D3
S315080274C0786813F01CFC0346894A9360786813F0BF
S315080274D037FC0346864AD360786813F052FC0346A3
S315080274E0834A1361786813F06DFC0346804A536138
S315080274F0786813F0BEFC03467D4A1362786813F077
S315080275000AFD03467A4A9362786813F07BFD0346BE
S31508027510774A5363786813F096FD0346744A936371
S31508027520786813F0B1FD0346714AD363714819F0BE
S3150802753023FF0121786814F043F9786813F050FFA5
S315080275400346002B01D111F0C9F8684B01221A70C3
S3150802755022E2674B1B69643B654A1361644B1B69EC
S31508027560002B09D1644819F007FF0021786814F046
S3150802757027F95E4B02221A70786813F031FF034628
S31508027580002B0CD011F0B6F85C4B1B685A1C5B49F1
S315080275900A60632B08D9564B64221A6104E011F07B
S315080275A09DF8564B00221A602DF0E4FC034605228C
S315080275B0612118462DF01CFD0346002B63D178681D
S315080275C014F08FFC55EC104B786814F0F6FC53EC6B
S315080275D0102B20462946F9F7C9FB0346002B4FD044
S315080275E0474B1B680133464A1360FFF729FF0346D8
S315080275F01A46434B1B689A4245D20021786814F012
S31508027600DFF804F003FB0346022B12D004F0FEFA5D
S315080276100346032B0DD004F0F9FA0346052B08D0CE
S3150802762004F0F4FA0346062B03D00021786813F017
S31508027630E3FF11F05FF8786813F026FD03462C4A3B
S31508027640D363304819F098FE0521786814F058FD7E
S315080276502D4B09221A702A4B00221A602B4B1B78D3
S31508027660002B09D0214B03221A70294B01221A70CA
S31508027670284B01221A7006E01B4B01221A7002E0FF
S315080276801F4B00221A60786814F0C6F80346002BCE
S3150802769000F016812DF06EFC034620226121184661
S315080276A02DF0A6FC0346002B40F0B080786814F053
S315080276B018FC51EC100B0AA3D3E90023F9F756FB81
S315080276C00346002B2AD0144B1B6803F00103002B38
S315080276D03CD1114B1B6801330F4A136036E000BFD9
S315080276E09A9999999999F13FBCCF002021D0002007
S315080276F070CF002084C7050894C7050824D0002047
S31508027700C0CF0020A8C705086DCF0020DCD3002013
S315080277100CCE002028CE0020CCCF0020786814F0AA
S31508027720E0FB51EC100BAFA3D3E90023F9F714FBE6
S315080277300346002B0AD09C4B1B6803F00103002B5F
S3150802774004D0994B1B680133974A1360964B1B6802
S31508027750002B04D0954B1B680133944A1360924B55
S315080277601B68032B48D9914B1B68C72B44D80021A9
S31508027770786814F025F804F049FA0346022B12D069
S3150802778004F044FA0346032B0DD004F03FFA0346ED
S31508027790052B08D004F03AFA0346062B03D000213B
S315080277A0786813F029FF10F0A5FF786813F06CFCCF
S315080277B003467F4AD3637F4819F0DEFD20217868A5
S315080277C014F09EFC7C4B09221A70774B00221A6031
S315080277D0764B00221A60794B1B78002B09D0784B1E
S315080277E003221A70774B01221A70774B01221A70FC
S315080277F002E0764B01221A706C4B1B68C72B05D91F
S31508027800694B00221A60694B00221A602DF0B2FBFE
S3150802781003461522612118462DF0EAFB0346002B82
S3150802782040F0B780786814F05CFB51EC100B5CA34F
S31508027830D3E90023F9F790FA0346002B3CD0644BB0
S315080278401B680133624A1360FFF7FAFD03461A46BC
S315080278505F4B1B689A4280F09C800021786813F07F
S31508027860AFFF0021786813F0C7FE10F043FF78686F
S3150802787013F00AFC03464E4AD363564819F07CFDB8
S315080278801521786814F03CFC4B4B09221A70504BB0
S3150802789000221A60494B1B78002B09D0484B032259
S315080278A01A70484B01221A70474B01221A7070E06F
S315080278B0464B01221A706CE0454B00221A6068E0BA
S315080278C0434B00221A60384B00221A60374B0022BB
S315080278D01A605EE0786813F083FD0346002B28D011
S315080278E010F008FF3C4819F047FD786813F0B6FC1B
S315080278F00346002B0BD0786812F006F903461846A1
S3150802790012F056F903461946786814F057FA2B4BC3
S315080279101B78002B09D02A4B03221A70294B012205
S315080279201A70294B01221A7036E0284B01221A7066
S3150802793032E010F027FF0121786812F07AFF002161
S31508027940786812F08FFE1221786814F0D9FB234862
S3150802795019F012FD224B04221A70184B1B78002BC1
S3150802796009D0174B03221A70164B01221A70164BAE
S3150802797001221A7010E0154B01221A700CE00F4B07
S315080279801B78002B07D1114B01221A7003E000BFA6
S3150802799002E000BF00E000BF00BF0837BD46B0BD29
S315080279A0333333333333C33FCCCF0020D0CF002019
S315080279B070CF0020C0C705086DCF0020DCD3002099
S315080279C021D000200CCE002028CE0020BCCF0020DB
S315080279D0C8CF0020D8C70508E8C7050854C7050850
S315080279E06CCF0020666666666666E63F80B500AFBF
S315080279F0174B5B6B632B29D9154B5A6B154BA3FB9C
S31508027A0002139B0B4EF6602101FB03F3D31A002BDC
S31508027A1017D111F0EBFF0346184615F05DFA034637
S31508027A20012B07D111F0E2FF03460321184614F091
S31508027A300EFA06E011F0DAFF03460421184614F09E
S31508027A4006FA034B5B6B643B014A536300BF80BD76
S31508027A5070CF002073B2E74580B58EB000AF78606C
S31508027A6011F0C4FF0346184615F00CFA38630023D2
S31508027A7087F83730002387F82F307B681B7887F81A
S31508027A802F30002387F82E300023BB62002387F8A5
S31508027A9037307FE011F0AAFF0346184615F0F2F9CF
S31508027AA03863FBF7DBFE02463B6B9B1A002BB8BF1B
S31508027AB05B4242F22732934202DD3B6B002B03D133
S31508027AC07B681B780B2B5DD141F288302AF002F9CC
S31508027AD010F0C2FB002011F045FB034687F82E3052
S31508027AE097F82E30002B02D12F4819F045FC10F0DA
S31508027AF025FC4FF4FA702AF0EDF810F011FC97F80D
S31508027B002E30002B15D008F0B1FEB86211F06EFFC8
S31508027B100346B96A184615F0C2F907F10C03BA6AA0
S31508027B202249184630F02EFE07F10C03184619F0C2
S31508027B3023FC10F0C3FB002011F0E0F90346002BEA
S31508027B4011D11B4819F018FC7B680B221A7097F89A
S31508027B503730022B0BD111F049FF03460A2118468A
S31508027B6014F0CEFA03E07B6897F82F201A7010F00B
S31508027B70E5FB4FF4FA702AF0ADF810F0D1FB08F0E5
S31508027B80A9FE02E0032387F8373097F83730013326
S31508027B9087F8373097F83730022B7FF67BAF00BF6E
S31508027BA000BF3837BD4680BD58C40508BCC50508A0
S31508027BB074C4050880B500AFFBF7F6FF0346002B31
S31508027BC032D010F0DFFD11F011FF0346184614F00B
S31508027BD083FE0346012B06D011F008FF0346002157
S31508027BE0184613F0EDFD11F001FF0346042118466D
S31508027BF014F086FA11F0FAFE0346184611F084FFCD
S31508027C0003460021184612F003FA084819F0B4FB95
S31508027C1011F0ECFE0346184613F036FA0346044AF8
S31508027C20D363044B09221A7000BF80BDF8C7050842
S31508027C3070CF00206DCF0020B0B52DED028B96B027
S31508027C4000AF11F0D3FEF864A14B1B78002B01F0AC
S31508027C5001802DF08FF903460522612118462DF081
S31508027C60C7F90346002B50D1F86C14F03AF955ECD3
S31508027C70104BF86C14F0A1F953EC102B2046294648
S31508027C80F9F774F80346002B3CD0924B1B68013374
S31508027C90904A1360FFF7D4FB03461A468D4B1B68BE
S31508027CA09A4232D20021F86C13F08AFD03F0AEFF35
S31508027CB00346022B12D003F0A9FF0346032B0DD06D
S31508027CC003F0A4FF0346052B08D003F09FFF0346E3
S31508027CD0062B03D00021F86C13F08EFCF86C13F017
S31508027CE0D3F903467C4AD3637C4819F045FB052140
S31508027CF0F86C14F005FA7A4B09221A70754B0022B1
S31508027D001A6002E0734B00221A60F86C13F084FDC5
S31508027D100346002B00F0EC802DF02CF903462022B6
S31508027D20612118462DF064F90346002B7DD1F86CC3
S31508027D3014F0D7F851EC100B5FA3D3E90023F9F737
S31508027D4015F80346002B0BD0664B1B6803F001039C
S31508027D50002B1DD1634B1B680133624A136017E07F
S31508027D60F86C14F0BEF851EC100B55A3D3E90023B6
S31508027D70F8F7F2FF0346002B0AD05A4B1B6803F0AA
S31508027D800103002B04D0574B1B680133554A136075
S31508027D90544B1B68002B04D0534B1B680133524AC1
S31508027DA01360504B1B68032B35D94F4B1B68C72BE7
S31508027DB031D80021F86C13F003FD03F027FF0346C0
S31508027DC0022B12D003F022FF0346032B0DD003F039
S31508027DD01DFF0346052B08D003F018FF0346062BA2
S31508027DE003D00021F86C13F007FCF86C13F04CF979
S31508027DF00346394AD363394819F0BEFA2021F86C8A
S31508027E0014F07EF9364B09221A70364B00221A6094
S31508027E10354B00221A60344B1B68C72B05D9314BE8
S31508027E2000221A60304B00221A602DF0A3F803468E
S31508027E301522612118462DF0DBF80346002B60D186
S31508027E40F86C14F04EF851EC100B1FA3D3E900237B
S31508027E50F8F782FF0346002B28D0244B1B68013310
S31508027E60224A1360FFF7ECFA03461A461F4B1B68B1
S31508027E709A4246D20021F86C13F0A2FC0021F86C53
S31508027E8013F0BAFBF86C13F0FFF80346124AD363F1
S31508027E90124819F071FA1521F86C14F031F9104BE1
S31508027EA009221A70114B00221A602AE00F4B00228F
S31508027EB01A6026E0AFF300809A9999999999F13F49
S31508027EC0666666666666E63F333333333333C33FE5
S31508027ED0BCCF0020C0CF002070CF0020D8C705082D
S31508027EE06DCF0020CCCF0020D0CF0020C8CF0020F5
S31508027EF0AB4B00221A60AB4B00221A60AA4B002237
S31508027F001A60AA4B1B780D2B00F2A68601A252F81C
S31508027F1023F000BF4D7F020841800208EF80020865
S31508027F206B81020829820208DF840208AD870208EB
S31508027F30CF8802081F890208358A0208E18A0208E0
S31508027F40598C02088B8B0208058C0208F86C13F010
S31508027F5085F90346002B05D1F86C13F0AFF90346F1
S31508027F60002B29D0F86C12F095FE0346904A53600E
S31508027F70F86C13F016FF03461A463B468D49184617
S31508027F8030F000FC3B46184619F0F6F9F86C13F087
S31508027F9008FF0346B3F5166F06D811F027FD034608
S31508027FA00821184614F0ACF8834819F0E5F97F4B16
S31508027FB001221A7000F067BEF86C13F0F2FE03464F
S31508027FC01C46F86C14F0C8FF03469C421CD80021D4
S31508027FD0F86C13F07DFBF86C14F07EFC0346012B5B
S31508027FE003D00021F86C13F0EBFB0021F86C13F0B8
S31508027FF003FB724B02221A70714819F0BDF96B4BDA
S3150802800003221A7000F03FBEF86C12F043FE0346D4
S31508028010674A5360F86C13F0C4FE03461A463B4699
S315080280206449184630F0AEFB3B46184619F0A4F9E7
S31508028030614819F0A1F95D4B01221A7000F023BEBE
S31508028040F86C13F00BF90346002B05D1F86C13F004
S3150802805035F90346002B19D0554B5B68643B544AE5
S315080280605360534B5B68002B3FD10121F86C13F028
S31508028070A7FBF86C12F0D9FD03464D4A1360514826
S3150802808019F07AF9494B02221A702EE0F86C13F0AD
S3150802809088FE03461C46F86C14F05EFF03469C42B3
S315080280A007D8494819F068F9404B00221A7000F0BF
S315080280B0D5BD3F4B5B68643B3D4A53603C4B5B68AE
S315080280C0002B40F0CB850121F86C13F079FBF86C94
S315080280D012F0ABFD0346364A13603A4819F04CF9DA
S315080280E0324B02221A7000F0B9BD00F0B7BD304B10
S315080280F01B68643B2E4A13602D4B1B68002B0FD15D
S31508028100F86C14F0E9FB0346012B03D00021F86C46
S3150802811013F056FB2C4819F02FF9244B00221A703B
S31508028120F86C13F03EFE03461C46F86C14F014FF76
S3150802813003469C4200F29485F86C13F001F9034653
S31508028140002B00F08D85F86C14F0C6FB0346012B54
S3150802815003D00021F86C13F033FB1B4819F00CF915
S31508028160124B00221A7000F07BBDF86C13F076F8F9
S315080281700346002B05D1F86C13F0A0F80346002B32
S3150802818024D0F86C12F0BBFD0346094A93600E48E8
S3150802819019F0F2F8054B00221A7000F063BD00BF11
S315080281A0C8CF0020CCCF0020D0CF00206DCF002032
S315080281B070CF002074C5050818C80508E0CF00204E
S315080281C024C8050830C8050840C80508B44B9B688A
S315080281D0643BB34A9360B24B9B68002B04D0B14B05
S315080281E01B78012B40F23E850121F86C13F0E8FA60
S315080281F00121F86C13F000FA0121F86C13F0B8FBB0
S31508028200F86C12F09DFD0346A54AD360F86C12F08D
S3150802821076FD0346A24A9360A34819F0ADF8A34B2C
S3150802822004221A7000F01EBDF86C13F017F8034604
S31508028230002B05D1F86C13F041F80346002B31D018
S31508028240974B5A699A4BA3FB02139B094FF47A710F
S3150802825001FB03F3D31A002B05D1914B5B6919462F
S31508028260944819F05DF98E4B5B69643B8C4A5361FD
S315080282708B4B5B69002B40F03181F86C14F02CFBB8
S315080282800346012B03D00021F86C13F099FA00215A
S31508028290F86C13F0B1F9884819F06EF8834B00228E
S315080282A01A701BE1F86C12F08DFD03467C4A536185
S315080282B07B4BDB68643B7A4AD36011F097FB034633
S315080282C0184613F043FD0346022B02D1744B0022D3
S315080282D0DA60734BDB68002B04D0724B1B78032BD6
S315080282E040F0C2846F4B00221A700121F86C13F019
S315080282F067FA0121F86C13F0EBF92DF039F9034608
S3150802830018462DF056F90346012118462BF008FDAA
S315080283106A4B00221A60F86C13F0ADFF03461A4640
S315080283203B466749184630F02DFA3B46184619F07F
S3150802833023F85E4B05221A70624B00221A6000214E
S31508028340F86C12F002FE1421F86C12F048FDF86C73
S3150802835012F059FD03465C4A13604FF000024FF0D3
S315080283600003C7E910234FF000024FF00003C7E9E4
S315080283701423F86C11F0C8FB0346184611F018FCD2
S315080283800346FB87FB8F1846F8F7F0F904460D46B5
S31508028390F86C13F006FD03461846F8F7E7F90246A5
S315080283A00B4620462946F8F7A3F802460B46C7E9C4
S315080283B010234FF00002454BC7E914234FF0000281
S315080283C04FF00003D7E91001F8F7DAFC0346002B51
S315080283D023D0FB8F1846F8F7C9F902460B46D7E9A8
S315080283E01401F8F767FB02460B46C7E91423D7E9D7
S315080283F01023D7E91401F8F733FA02460B46C7E900
S3150802840014234FF00002324BD7E91401F8F772F839
S3150802841002460B46C7E914232AE0F86C13F0C1FC9E
S315080284200346B3F57A6F23D3FB8F1846F8F79EF9FE
S3150802843002460B46D7E91401F8F73CFB02460B46FF
S31508028440C7E914234FF00002224BD7E91401F8F7C3
S3150802845007FA02460B46C7E914234FF000021C4BE3
S31508028460D7E91401F8F746F802460B46C7E914237A
S31508028470D7E91401F8F7CCFC03461946F86C12F052
S3150802848095FDD7E91401F8F7C3FC02463B461249A3
S31508028490184630F077F93B46184618F06DFFE3E3C5
S315080284A070CF0020E0CF00204CC805086DCF002011
S315080284B0D34D62105CC8050840C80508D4CF002011
S315080284C068C80508DCCF002000000020008056405E
S315080284D00000244000408F4080C80508C4E3F86CB9
S315080284E012F0BCFE0346002B08D1A04B1B78002BCA
S315080284F004D19F4B1B78002B00F081809D4B5B6952
S31508028500643B9C4A53619B4B5B69002B74D1974B26
S315080285101B78002B4ED1F86C11F0F6FA0346184672
S3150802852011F046FB03461946F86C13F047FCF86C43
S3150802853012F09FFC03468F4A1362F86C12F062FD32
S3150802854003468C4A5363F86C11F0DEFA0346184662
S3150802855011F0F4FB03461A46874B1B689A420CD263
S31508028560F86C11F0D1FA0246834B1B689BB2194686
S31508028570104611F0D3FBFBF737F9F86C11F0C4FA81
S315080285800346184611F054FD03461C46F86C14F0CF
S31508028590DDFA03469C420DD0F86C11F0B5FA044692
S315080285A0F86C14F0D3FA03461946204611F030FD4A
S315080285B0FBF71AF90021F86C13F01EF86B4B1B78BF
S315080285C0002B12D16A4B1B78002B03D06B4818F08C
S315080285D0D3FE02E06A4818F0CFFE0621F86C12F0C4
S315080285E09EFD684B06221A7097E0674818F0C4FE8B
S315080285F0644B0D221A7090E0FFF7DCFA8DE0F86CF6
S3150802860012F0E0FB03465B4A5361FFF7D3FA642193
S31508028610F86C12F0AAFCF86C13F063FC55EC104BDC
S31508028620F86C13F0A6FC53EC102B20462946F8F7F3
S315080286309DFB0346002B12D0544B1B680133534A49
S315080286401360524B1B68282B0CD9484B01221A700F
S315080286504F4818F091FE4D4B00221A6002E04B4B30
S3150802866000221A60F86C13F006FE03461C46F86CE4
S3150802867014F0CCFB03469C4228DA464818F07CFEE6
S315080286800321F86C13F03CFD434B01221A70F86C77
S3150802869012F0D9FC0346374A9363F86C13F0EBFDE4
S315080286A003461A463B463D49184630F06BF83B46A8
S315080286B0184618F061FE0021F86C12F09DFF384842
S315080286C018F05AFE2F4B07221A7009E0F86C13F0BD
S315080286D068FB0346B3F5486F02D9F86C12F012FD2F
S315080286E0F86C12F025FC0446F86C12F052FC0346AC
S315080286F09C4212D92B4B1B6803F40033002B0CD176
S31508028700294818F039FE1121F86C13F0F9FC254BAB
S315080287101B6843F40033234A1360F86C11F0F4F92A
S315080287200346184611F0CCFAB0EE408AF86C13F0FC
S31508028730C0FDF0EE407AB4EEE78AF1EE10FA0FDDEC
S31508028740F86C11F0E1F90446F86C13F0B2FDF0EE9C
S31508028750407AB0EE670A204611F0A2FAFBF744F80F
S31508028760054B1B680133044A13608CE2E0CF0020F4
S31508028770F0CF002070CF0020D4CF002098C805087B
S31508028780C0C805086DCF0020D8C80508C4CF002088
S31508028790F8C8050814C90508F1CF00202CC9050830
S315080287A044C90508D8CF002058C90508B54B1B6A25
S315080287B0643BB44A1362B34B1B6A002B50D1F86C64
S315080287C014F08AF80346012B03D00021F86C12F044
S315080287D0F7FFF86C13F05CFA0346002B05D0AA4B98
S315080287E000221A70A94B00221A70F86C13F043FD86
S315080287F003461A463B46A64918462FF0C3FF3B4690
S31508028800184618F0B9FDF86C11F07EF903461846B9
S3150802881011F0EAFA03461A463B469E4918462FF0D5
S31508028820B1FF3B46184618F0A7FDF86C12F030F86F
S315080288300346002B09D1F86C13F0C2F80346002B45
S3150802884003D00021F86C13F093F8934B00221A70A8
S315080288500321F86C12F092FC8C4B00221A7005E286
S31508028860F86C13F09EFA03461C46F86C14F074FB77
S3150802887003469C4200F2FA81F86C12F07FFD034629
S31508028880002B40F0F381F86C13F0F5FC03461A4608
S315080288903B467F4918462FF075FF3B46184618F0A7
S315080288A06BFDF86C11F030F90346184611F09CFA84
S315080288B003461A463B46774918462FF063FF3B465E
S315080288C0184618F059FD714B00221A70CEE16D4B0D
S315080288D09B6B643B6B4A93636A4B9B6B002B40F022
S315080288E0C781F86C12F08FFA03466C4A13606C481B
S315080288F018F042FDF86C13F0BEFC03461A463B46D6
S31508028900634918462FF03EFF3B46184618F034FDD9
S315080289105E4B00221A70634B00221A60A8E1594B7B
S315080289201B69643B574A1361564B1B69002B65D179
S31508028930F86C12F09EFA0346524A13620121F86C49
S3150802894012F024FE0021F86C12F056FE564B1B78E4
S31508028950002B06D0554818F00FFD4C4B0D221A7005
S3150802896013E0534B1B78002B09D0514B00221A7087
S31508028970504818F001FD454B07221A7005E04E488B
S3150802898018F0FAFC414B06221A704C4B00221A6068
S315080289904B4B00221A604B4B00221A60F86C14F0FB
S315080289A0F3F80346002B1FD00021F86C13F063FE80
S315080289B00446F86C14F006F903469C4214D30121C6
S315080289C0F86C13F058FE0446F86C14F019F90346CD
S315080289D09C4209D33C4818F0CFFC3C4B3C4A1A60EF
S315080289E0062003F001F905E03A4818F0C5FC022012
S315080289F003F0FAF80121F86C12F0BAFFF86C11F0DC
S31508028A0047FF0346002B40F03581F86C12F031FA25
S31508028A1003461C4A13620021F86C12F0EDFD002190
S31508028A20F86C12F0B3FD244818F0A6FC174B062280
S31508028A301A701FE1134BDB6B643B124AD363114B6B
S31508028A40DB6B002B40F018810121F86C12F0B8FE9E
S31508028A502CF090FA03461522612118462CF0C8FA22
S31508028A600346002B06D01C4818F086FC074B0C223E
S31508028A701A7001E1194818F07FFC044B0A221A7091
S31508028A80FAE000BF70CF00206CCF00206DCF002027
S31508028A9078C905088CC90508F0CF00200000002017
S31508028AA098C90508DCCF0020E0CF0020ACC905082C
S31508028AB0F1CF002044C90508BCC905087CD10020AD
S31508028AC080D1002084D10020CCC9050824000020CA
S31508028AD040771B00E0C90508F0C9050804CA05085D
S31508028AE0F86C13F0FEF955EC104BF86C13F01DFAFE
S31508028AF053EC102B20462946F8F724F90346002B97
S31508028B0022D0654B1B680133634A1360624B1B68AC
S31508028B10B3F5167F40F2B280F86C13F0DDFE034619
S31508028B20002B04D15C4B00221A6007F0D1FD5A4B88
S31508028B301B6840F6B832934240F2A080564B002298
S31508028B401A6007F0C5FD99E0534B00221A60534B91
S31508028B501B680133514A1360504B1B68322B40F293
S31508028B608D804E4B00221A600021F86C12F028FE06
S31508028B70F86C12F089FA0346494AD363494818F051
S31508028B80FBFB494B09221A7078E0F86C13F0A9F935
S31508028B9051EC100B3EA3D3E90023F8F7F1F803468C
S31508028BA0002B0FD03C4B1B6801333B4A13603A4BF0
S31508028BB01B68B3F5167F63D9374B00221A6007F094
S31508028BC087FD5DE0344B00221A60384B1B6801337F
S31508028BD0364A1360354B1B68322B51D9334B002268
S31508028BE01A600021F86C12F0EBFDF86C12F04CFAE0
S31508028BF003462B4AD3632B4818F0BEFB2A4B09229D
S31508028C001A703DE0F86C13F06CF955EC104BF86CE1
S31508028C1013F08BF953EC102B20462946F8F792F8F5
S31508028C200346002B12D01C4B1B6801331A4A1360E9
S31508028C30194B1B68642B25D91D4818F09DFB1A4B46
S31508028C4000221A70144B00221A601BE0124B0022F3
S31508028C501A6017E000BF16E000BF14E000BF12E07A
S31508028C6000BF10E000BF0EE000BF0CE000BF0AE044
S31508028C7000BF08E000BF06E000BF04E000BF02E054
S31508028C8000BF00E000BF5837BD46BDEC028BB0BD41
S31508028C90333333333333C33F28D00020C0CF0020C9
S31508028CA070CF0020D8C705086DCF0020C8CF002096
S31508028CB040C8050880B582B000AF10F097FE78600C
S31508028CC0786810F021FF0346184611F0BBF80346F0
S31508028CD0012B3DD10FF03EFD0346002B12D10FF0BA
S31508028CE045FD0346002B0DD1A14B1B7803F001036A
S31508028CF0DAB29F4B1A709F4B00221A709E4B0022C3
S31508028D001A7062E00FF026FD0346002B04D00FF01E
S31508028D102DFD0346002B0DD1954B00221A70954B5B
S31508028D2000221A70944B1B7803F00103DAB2924BB5
S31508028D301A704AE08E4B00221A708E4B1B7803F08B
S31508028D400103DAB28B4B1A708B4B00221A703CE085
S31508028D500FF000FD0346012B12D10FF007FD034663
S31508028D60012B0DD1824B1B7803F00103DAB2804B3B
S31508028D701A70804B00221A707F4B00221A7024E068
S31508028D800FF0E8FC0346012B04D00FF0EFFC034674
S31508028D90012B0DD1764B00221A70764B00221A70DF
S31508028DA0754B1B7803F00103DAB2734B1A700CE0A9
S31508028DB06F4B00221A706F4B1B7803F00103DAB26D
S31508028DC06C4B1A706C4B00221A700FF0B7FC0346F4
S31508028DD0002B07D1694B1B7803F00103DAB2674B04
S31508028DE01A7002E0654B00221A7010F03DF803462D
S31508028DF0012B04D10221786813F01CFF03E002213B
S31508028E00786813F02FFF10F063F90346012B04D19B
S31508028E100121786813F00EFF03E00121786813F048
S31508028E2021FF10F0BFFD0346002B07D1544B1B78D8
S31508028E3003F00103DAB2524B1A7002E0504B0022D9
S31508028E401A7010F0BBFD0346002B07D14D4B1B7859
S31508028E5003F00103DAB24B4B1A7002E0494B0022C7
S31508028E601A70494B1B785A1CD1B2474A1170022B09
S31508028E7026D93F4B1B781946786812F0A1F93E4B62
S31508028E801B781946786812F0F7F93A4B1B78194697
S31508028E90786812F021FA394B1B781946786812F06D
S31508028EA07BFA394B00221A70344B01221A70304B66
S31508028EB001221A702F4B01221A702F4B01221A70A7
S31508028EC0324B1B785A1CD1B2304A1170312B40F200
S31508028ED04B812C4B1B78002B62D0786810F014FE5D
S31508028EE00346184611F089FA0346012B31D12CF0B4
S31508028EF041F803460922622118462CF079F80346FE
S31508028F00002B22D1224818F037FA0921786813F083
S31508028F1075F90021786812F039FB0021786812F099
S31508028F20A1FB0021786812F011FC0021786812F082
S31508028F30C1FD10F0D0FC10F0EBFC0021786811F0AE
S31508028F40B5FC0021786811F0A1FD124B3C221A608B
S31508028F506EE0114B1B78002B6AD10D4818F00CFAFB
S31508028F600D4B01221A700D4B01221A7060E000BFE8
S31508028F701200002013000020140000201500002013
S31508028F8016000020170000202CD000202DD000202B
S31508028F9010CA0508180000200ED00020EACF0020CB
S31508028FA0786810F0B1FD0346184611F026FA034612
S31508028FB0012B1DD12BF0DEFF03460922622118463A
S31508028FC02CF016F80346002B32D0694B1B683C2B53
S31508028FD002D1684818F0D0F9654B1B68013B644A10
S31508028FE01360634B1B68002B22D107F071FB1FE04D
S31508028FF0614B1B78002B1BD02BF0BCFF03460922C2
S31508029000622118462BF0F4FF0346002B0AD00021F2
S31508029010786813F0F3F82BF0ADFF002309226221DA
S315080290202CF085F8554818F0A7F9534B00221A7008
S31508029030534B1B78002B46D0786810F065FD034623
S31508029040184611F0DAF90346012B2ED12BF092FFBE
S3150802905003462122612118462BF0CAFF0346002B3C
S315080290601FD1484818F088F92121786813F048F882
S315080290700FF088FB0021786812F02AFB0021786835
S3150802908012F0E2FC2CF074FA034618462CF091FA18
S315080290900346002118462AF043FE0021786811F09B
S315080290A0E1FA394B3C221A6055E0384B1B78002B03
S315080290B051D1344818F060F9344B01221A70344BF6
S315080290C001221A7047E0786810F01EFD034618461A
S315080290D011F093F90346012B1DD12BF04BFF0346E2
S315080290E02122612118462BF083FF0346002B32D03A
S315080290F0254B1B683C2B02D1264818F03DF9224B1A
S315080291001B68013B204A13601F4B1B68002B22D1A8
S3150802911007F0DEFA1FE01D4B1B78002B1BD02BF045
S3150802912029FF03462122612118462BF061FF0346D7
S31508029130002B0AD00021786812F0E2FF2BF01AFF02
S315080291400023212261212BF0F2FF134818F014F9AB
S315080291500E4B00221A70114B00221A70084B01227C
S315080291601A700F4B01221A7000BF0837BD4680BD20
S315080291701800002034CA05080ED0002058CA05086F
S315080291801600002080CA05081C0000200DD0002009
S31508029190E9CF0020A0CA0508C0CA05082DD00020BC
S315080291A01700002080B500AF2BF0E4FE03460B2221
S315080291B0612118462BF01CFF0346002B1AD010F02B
S315080291C015FC0346184612F0ECFD0346B3F5C87FB4
S315080291D010D3094818F0D0F810F008FC034600210D
S315080291E0184612F08DFF2BF0C5FE00230B226121D3
S315080291F02BF09DFF00BF80BDE0CA0508B0B59CB044
S3150802920002AF786010F0F2FB38660023A7F85E30EA
S31508029210002387F85D3000237B660EF0DCFEC94822
S3150802922008F04CFE034683F00103DBB2002B00F084
S315080292305A86C548FAF7A8FC0346A7F85E30B7F877
S315080292405E30002B00F05786BF4B1B78013B0A2B7A
S3150802925000F22F8601A252F823F000BF8992020873
S31508029260A79802087B9A0208819B0208A19B02081A
S3150802927061950208CF9B0208B79C0208BF9C0208A8
S315080292807B9D0208CF9D02080021386E13F012FA60
S315080292900020FAF739FFAC4B5B68AB4A926819466D
S315080292A0AA4818F03DF9A84B5B78002B04D0A64BC8
S315080292B05B78022B40F0F2802BF05CFE03460A2212
S315080292C0612118462BF094FE0346002B31D0A048A4
S315080292D018F052F89C4B5B78002B07D19A4B9B7877
S315080292E00B2118460EF0F0FB00F0FDBD964B9B785D
S315080292F087F854300B2387F8553007F1100207F127
S315080293005403114618462BF0D4F907F110031846F0
S315080293102AF035FE044607F1100318462AF03BFEEA
S3150802932003461A46214640F209402CF0BBFE00F0DD
S31508029330DABD2BF01FFE03460B22612118462BF0DD
S3150802934057FE0346002B31D0824818F015F87E4B9B
S315080293505B78002B07D17C4B9B780C2118460EF0C4
S31508029360B3FB00F0C0BD784B9B7887F854300C23CA
S3150802937087F8553007F1100207F1540311461846CB
S315080293802BF097F907F1100318462AF0F8FD044660
S3150802939007F1100318462AF0FEFD03461A4621462F
S315080293A040F209402CF07EFE00F09DBD2BF0E2FD56
S315080293B003460C22612118462BF01AFE0346002B9F
S315080293C00AD12BF0D7FD03460D22612118462BF050
S315080293D00FFE0346002B31D05F4817F0CDFF5A4BDC
S315080293E05B78002B07D1584B9B78022118460EF062
S315080293F06BFB00F078BD544B9B7887F854300223F8
S3150802940087F8553007F1100207F15403114618463A
S315080294102BF04FF907F1100318462AF0B0FD04465F
S3150802942007F1100318462AF0B6FD03461A462146E6
S3150802943040F209402CF036FE00F055BD0121386E87
S3150802944013F057FA404B5B78002B06D13E4B9B78BC
S31508029450092118460EF038FB20E03B4B9B7887F82B
S315080294605430092387F8553007F1100207F15403DF
S31508029470114618462BF01DF907F1100318462AF073
S315080294807EFD044607F1100318462AF084FD0346BA
S315080294901A46214640F209402CF004FE2A4B586827
S315080294A0294B9968284B1C7B274B5D7B264B9B7B5C
S315080294B0254A927C019200932B462246FAF7DAFF56
S315080294C0034687F85D30204B5B78002B08D11E4B8C
S315080294D09B7897F85D20114618460EF0F5FA2AE0B1
S315080294E0194B5B78022B26D1174B9B7887F8543099
S315080294F097F85D3087F85530184B1B689BB2A7F86A
S31508029500563007F1100207F15403114618462BF09C
S31508029510D0F807F1100318462AF031FD044607F180
S31508029520100318462AF037FD03461A46214640F22A
S3150802953009402CF0B7FD0021386E13F0DAF900F075
S31508029540D2BC00BF6CCE002030D0002000CB05086C
S3150802955010CB050828CB050840CB0508F4CF002018
S315080295600021386E13F0A6F80020FAF7CDFDAB4BB2
S315080295705B68AA4A92681946A94817F0D1FFA74B11
S315080295805B78002B08D0A54B5B78022B04D0A34B43
S315080295905B78032B40F024812BF0ECFC03460A226D
S315080295A0612118462BF024FD0346002B3ED09D4828
S315080295B017F0E2FE994B5B78002B07D1974B9B7805
S315080295C00B2118460EF080FA00F08DBC934B9B785F
S315080295D087F854300B2387F85530904B1B8AA7F827
S315080295E0583007F1100207F15403114618462BF0BA
S315080295F060F88A4B5B78022B03D140F209437B66FB
S3150802960001E0894B7B6607F1100318462AF0B7FC7E
S31508029610044607F1100318462AF0BDFC03461A460B
S315080296202146786E2CF03EFD00F05DBC2BF0A2FCC4
S3150802963003460B22612118462BF0DAFC0346002B5F
S315080296403ED07A4817F098FE744B5B78002B07D108
S31508029650724B9B780C2118460EF036FA00F043BC82
S315080296606E4B9B7887F854300C2387F855306B4B32
S315080296701B8AA7F8583007F1100207F1540311465E
S3150802968018462BF016F8654B5B78022B03D140F28D
S3150802969009437B6601E0644B7B6607F110031846B3
S315080296A02AF06DFC044607F1100318462AF073FCEB
S315080296B003461A462146786E2CF0F4FC00F013BCD9
S315080296C02BF058FC03460C22612118462BF090FC1D
S315080296D00346002B0AD12BF04DFC03460D226121CD
S315080296E018462BF085FC0346002B3CD0504817F051
S315080296F043FE4A4B5B78002B06D1484B9B780221E6
S3150802970018460EF0E1F9EEE3444B9B7887F854309D
S31508029710022387F85530414B1B8AA7F8583007F1C0
S31508029720100207F15403114618462AF0C2FF3B4BB2
S315080297305B78022B03D140F209437B6601E03A4B80
S315080297407B6607F1100318462AF019FC044607F14E
S31508029750100318462AF01FFC03461A462146786E5D
S315080297602CF0A0FCBFE30121386E13F0C2F82B4B94
S315080297705B78002B06D1294B9B78092118460EF0F7
S31508029780A3F92DE0254B9B7887F85430092387F8EF
S315080297905530224B1B8AA7F8583007F1100207F1F9
S315080297A05403114618462AF084FF1C4B5B78022B99
S315080297B003D140F209437B6601E01B4B7B6607F146
S315080297C0100318462AF0DBFB044607F11003184675
S315080297D02AF0E1FB03461A462146786E2CF062FC13
S315080297E00E4B58680D4B99680C4B1A7B0B4B5C7BDE
S315080297F00A4B9B7B00932346FBF7CAFA034687F874
S315080298005D30064B5B78002B14D1044B9B7897F896
S315080298105D20114618460EF057F93FE030D0002079
S3150802982000CB050854CB05080600100028CB05080E
S3150802983040CB0508CC4B9B7887F8543097F85D30B7
S3150802984087F85530C94B1B689BB2A7F85630C64BEA
S315080298501B8AA7F8583007F1100207F1540311467C
S3150802986018462AF026FFC04B5B78022B03D140F23A
S3150802987009437B6601E0BE4B7B6607F11003184677
S315080298802AF07DFB044607F1100318462AF083FBEB
S3150802989003461A462146786E2CF004FC0221386EDD
S315080298A013F027F81FE3B34817F066FD2BF060FEA6
S315080298B0034618462BF072FE0346002118462AF084
S315080298C0FCF9FCF7B7FF0346002B40F0AC802BF0FF
S315080298D051FB03462522662118462BF089FB0346CF
S315080298E0002B20D12BF046FB03462422662118467C
S315080298F02BF07EFB0346002B15D12BF03BFB0346D0
S315080299000A22612118462BF073FB0346002B0AD163
S315080299102BF030FB03461C22612118462BF068FB0C
S315080299200346002B1BD02BF025FB0023252266219C
S315080299302BF0FDFB2BF01EFB0023242266212BF0C5
S31508029940F6FB2BF017FB00230A2261212BF0EFFB13
S315080299502BF010FB00231C2261212BF0E8FB2BF0D5
S3150802996009FB03460122612118462BF041FB0346F7
S31508029970002B0AD12BF0FEFA034612226121184661
S315080299802BF036FB0346002B18D02BF0F3FA0023F4
S31508029990252261212BF0CBFB2BF0ECFA00231222B5
S315080299A061212BF0C4FB0021386E10F042FF002023
S315080299B0F9F7D0FF0121386E10F054FE6E4817F001
S315080299C0DBFC694B5B78002B07D101200EF0E6F928
S315080299D00021386E12F08DFF6DE2634B5B78022B25
S315080299E040F069820021386E12F083FF01233B732F
S315080299F007F1100207F10C03114618462AF09FFDDB
S31508029A0007F1100318462AF0BAFA044607F11003BA
S31508029A1018462AF0C0FA03461A46214640F2094079
S31508029A202CF040FB47E2504B5B78002B03D1022017
S31508029A300EF0B4F93FE24C4B5B78022B40F03B82C6
S31508029A4002233B7207F1100207F108031146184672
S31508029A502AF075FD07F1100318462AF090FA044613
S31508029A6007F1100318462AF096FA03461A462146C3
S31508029A7040F209402CF016FB1DE23B4B5B78002BAB
S31508029A8003D109200EF0DEF924E0374B5B78022B6E
S31508029A9020D1354B9B7887F85430092387F85530FF
S31508029AA007F1100207F15403114618462AF001FE7F
S31508029AB007F1100318462AF062FA044607F1100362
S31508029AC018462AF068FA03461A46214640F2094021
S31508029AD02CF0E8FA0121386E12F00BFF224B5B6874
S31508029AE0214A926811461846FCF72AFA034687F86D
S31508029AF05D301D4B5B78002B05D197F85D30184613
S31508029B000EF0A0F92AE0184B5B78022B26D1164BE9
S31508029B109B7887F8543097F85D3087F85530174B9D
S31508029B201B689BB2A7F8563007F1100207F15403D7
S31508029B30114618462AF0BDFD07F1100318462AF009
S31508029B401EFA044607F1100318462AF024FA0346B9
S31508029B501A46214640F209402CF0A4FA0021386E32
S31508029B6012F0C7FEBFE100BF30D00020F8CF0020B8
S31508029B70060010006CCB05087CCB0508F4CF002044
S31508029B8006F026FFF9F730FECD4817F0F5FBCD4B68
S31508029B905B78002B40F0918101200EF07DF98CE173
S31508029BA00FF024FF03460121184611F017FFC54B93
S31508029BB09B68642202FB03F3184628F08BF80FF021
S31508029BC015FF03460021184611F008FF8BE10FF036
S31508029BD00DFF0346184612F07FFE0346002B41D1BD
S31508029BE0B84B5B68DBB21846FCF770FF034687F88A
S31508029BF05D30B44B5B78002B0BD197F85D30002BA8
S31508029C0003D101200DF0FFFF68E102200DF0FBFFF2
S31508029C1064E1AC4B5B78022B40F0608197F85D30CB
S31508029C20002B06D107F11003194601202AF070FD10
S31508029C3005E007F11003194602202AF069FD07F12B
S31508029C40100318462AF09BF9044607F11003184632
S31508029C502AF0A1F903461A46214640F209402CF099
S31508029C6021FA3BE1984817F087FB964B5B78002B65
S31508029C7003D101200DF0C7FF30E1924B5B78022B2E
S31508029C8040F02C8107F11003194601202AF040FD05
S31508029C9007F1100318462AF072F9044607F1100371
S31508029CA018462AF078F903461A46214640F2094030
S31508029CB02CF0F8F912E1854817F032FC13E1814BD2
S31508029CC01B7B804A927811461846FCF75FFF0346CB
S31508029CD087F85D307B4B5B78002B05D197F85D30B2
S31508029CE018460DF0BAFF43E0764B5B78022B1AD181
S31508029CF007F1100297F85D30114618462AF025FD3D
S31508029D0007F1100318462AF03AF9044607F1100338
S31508029D1018462AF040F903461A46214640F20940F7
S31508029D202CF0C0F924E0674B5B78032B20D197F817
S31508029D305D3087F85530634B1B8AA7F8583007F110
S31508029D40100207F15403114618462AF01BFD07F1C3
S31508029D50100318462AF013F9044607F110031846A9
S31508029D602AF019F903461A46214659482CF09AF957
S31508029D700021386E12F0BDFDB5E0FDF729F803465D
S31508029D8087F85D304F4B5B78002B00F0A9804D4B6E
S31508029D905B78022B40F0A48007F1100297F85D3039
S31508029DA0114618462AF011FD07F1100318462AF043
S31508029DB0E6F8044607F1100318462AF0ECF80346BB
S31508029DC01A46214640F209402CF06CF988E04148CF
S31508029DD017F0A6FB2BF0CCFB034618462BF0DEFB4E
S31508029DE003460021184629F068FFFCF723FD0346BF
S31508029DF0002B56D12BF0BEF80346252266211846BB
S31508029E002BF0F6F80346002B20D12BF0B3F80346C5
S31508029E102422662118462BF0EBF80346002B15D1AF
S31508029E202BF0A8F803460A22612118462BF0E0F81F
S31508029E300346002B0AD12BF09DF803461C2261210A
S31508029E4018462BF0D5F80346002B1BD02BF092F8B8
S31508029E500023252266212BF06AF92BF08BF80023C2
S31508029E60242266212BF063F92BF084F800230A22B8
S31508029E7061212BF05CF92BF07DF800231C2261216D
S31508029E802BF055F9144817F04BFB0E4B5B78002B59
S31508029E9028D101200DF0ACFF0021386E12F029FD01
S31508029EA020E0084B5B78002B1CD102200DF0A0FFA6
S31508029EB018E000BF17E000BF15E000BF13E000BFBF
S31508029EC088CB050830D000209CCB0508ACCB05080A
S31508029ED006001000CCCB05087CCB050800BF02E0C3
S31508029EE000BF00E000BF012006F0DAFB642027F07D
S31508029EF0F1FEFFF794B900BF6837BD46B0BD00BF93
S31508029F0080B582B000AF0FF071FD7860FEF7D2FE21
S31508029F10FDF7AEFAFFF746F9FDF76CFA786810F026
S31508029F2093FB0346002B14D02A4B1B78002B10D028
S31508029F30FCF7BCFF786810F051FC0346012B44D0AD
S31508029F40786810F069FC0346012B3ED0FDF774FED3
S31508029F503BE0214B1B78002B38D0786810F0BAFF0B
S31508029F6003461E4A13601D4B1B68642B0FD91B4BF5
S31508029F701B681B4A93420AD8164B00221A70174BC3
S31508029F801B68643B1946786810F094FF1EE0134B71
S31508029F901B68002B0FD0114B1B68642B0BD80021B2
S31508029FA0786811F00DFC0D4B1B68643B19467868FE
S31508029FB010F080FF0AE0074B01221A70094B0022B3
S31508029FC01A70094B00221A7000E000BF00BF08375A
S31508029FD0BD4680BD20000020BCCF002044D0002012
S31508029FE0C0D401006CCF00206DCF002080B483B0AE
S31508029FF000AF0346FB71054AFB7913700123184625
S3150802A0000C37BD465DF8047B704700BF210000206F
S3150802A01080B400AF034B1B781846BD465DF8047B37
S3150802A020704700BF2100002080B582B000AF78607B
S3150802A030214B1B78062B34D801A252F823F000BF15
S3150802A0405DA0020867A0020871A002087BA00208A8
S3150802A05085A002088FA0020899A002081749786805
S3150802A0602EF090FB22E0164978682EF08BFB1DE055
S3150802A070144978682EF086FB18E0134978682EF0A2
S3150802A08081FB13E0114978682EF07CFB0EE010493B
S3150802A09078682EF077FB09E00E4978682EF072FB95
S3150802A0A004E00D4978682EF06DFB00BF7B68184600
S3150802A0B00837BD4680BD00BF21000020D4CB050865
S3150802A0C0E8CB0508F4CB050804CC050814CC05082A
S3150802A0D030CC050840CC050850CC050880B582B0BE
S3150802A0E000AF7860114B1B78022B10D0022B13DCC1
S3150802A0F0002B02D0012B05D00EE00D4978682EF010
S3150802A10041FB0EE00B4978682EF03CFB09E00A4950
S3150802A11078682EF037FB04E0084978682EF032FB9F
S3150802A12000BF7B6818460837BD4680BDF8D00020B8
S3150802A13060CC05086CCC05087CCC050898CC0508CB
S3150802A14080B582B000AF78600B467B807B881A4662
S3150802A1507968044808F03DF8034618460837BD46AC
S3150802A16080BD00BF04D1002080B582B000AF786000
S3150802A1707968044808F03EF803469BB21846083741
S3150802A180BD4680BD04D1002090B591B002AF3B60B8
S3150802A1900346FB710B46BB7113467B71012387F895
S3150802A1A02830FB7987F82930BB7987F82A307B79FA
S3150802A1B087F82B303B68FB62B7F848303B6397F861
S3150802A1C04C3087F8343097F82A30194697F82B30EE
S3150802A1D01C46FB6A3A6B07F1080001920093234674
S3150802A1E00A4609492EF0CEFA07F10803184617F06F
S3150802A1F0C3F807F1280310211846FFF7A1FF00BF8D
S3150802A2003C37BD4690BD00BFA8CC050880B58EB0C8
S3150802A21000AF03460A46FB711346BB71022387F851
S3150802A2202830FB7987F82930002387F82A30BB794A
S3150802A23087F82B300023FB6200233B6397F82B3009
S3150802A2401A4607F10803094918462EF09BFA07F140
S3150802A2500803184617F090F807F128031021184644
S3150802A260FFF76EFF00BF3837BD4680BDC4CC050870
S3150802A27080B58EB000AF03460A46FB711346BB7122
S3150802A280032387F82830FB7987F82930002387F8D3
S3150802A2902A30BB7987F82B300023FB6200233B6305
S3150802A2A097F82B301A4607F10803094918462EF083
S3150802A2B069FA07F10803184617F05EF807F128034A
S3150802A2C010211846FFF73CFF00BF3837BD4680BD50
S3150802A2D0DCCC050880B58EB000AF03460A46FB7192
S3150802A2E01346BB71042387F82830FB7987F829308F
S3150802A2F0BB79FB62FA6A07F10803094918462EF088
S3150802A30041FA07F10803184617F036F807F1280349
S3150802A31010211846FFF714FF00BF3837BD4680BD27
S3150802A320F0CC050880B500AF124B1B78032B01D081
S3150802A330062B0ED10FF05AFB03460121184611F0DF
S3150802A340DDFA0FF053FB03460121184611F078FC9B
S3150802A3500EE00FF04BFB03460021184611F0CEFA29
S3150802A3600FF044FB03460021184611F069FC00BFB2
S3150802A37000BF80BD210000202DE9B0432DED028BE0
S3150802A3809CB004AF3C4684E80F000FF02FFBF8643C
S3150802A3907B68FB65012387F85B304FF000037B651A
S3150802A3A04FF000033B65BB68002B0DD0F86C12F02A
S3150802A3B023FA0246BB781946104628F0A7FF87ED0E
S3150802A3C0140A42F21073FB65386DF6F7F1F9024684
S3150802A3D00B46C54817F0A4F80121F86C11F08EFA5D
S3150802A3E00121F86C11F02CFC0EF0C4FC0346032B79
S3150802A3F029D0BE4816F0C0FF0DF0ECFE00200EF084
S3150802A400F7FC0346002B17D1062387F85B30B848BA
S3150802A41016F0B2FF2BF0ACF8034618462BF0BEF83E
S3150802A42003460521184629F020FD2AF0A3FD01233B
S3150802A430052263212AF01AFE0DF0F8FE642027F0A1
S3150802A44049FC0DF0DDFE97F85B30062B04D1FFF7C9
S3150802A45069FF97F85B30F7E10EF0CEF90346032B56
S3150802A46026D0A44816F088FF0FF0DEF900200EF079
S3150802A47051FA0346002B17D1032387F85B309E480F
S3150802A48016F07AFF2BF074F8034618462BF086F876
S3150802A49003460721184629F0E8FC2AF06BFD01233A
S3150802A4A0072263212AF0E2FD0FF0EAF90FF0FEF91E
S3150802A4B097F85B30032B6CD10EF000FB0346032B97
S3150802A4C026D08E4816F058FF0FF0C4F900200EF079
S3150802A4D083FB0346002B17D1042387F85B30884891
S3150802A4E016F04AFF2BF044F8034618462BF056F8A6
S3150802A4F003460821184629F0B8FC2AF03BFD012339
S3150802A500082263212AF0B2FD0FF0BAF90FF0CEF94C
S3150802A51097F85B30042B04D1FFF704FF97F85B30FA
S3150802A52092E10EF0A1FB0346032B29D0754816F0DB
S3150802A53023FF0DF039FE00200EF0D4FB0346002B54
S3150802A54017D1052387F85B306F4816F015FF2BF0F5
S3150802A5500FF8034618462BF021F80346062118463B
S3150802A56029F083FC2AF006FD0123062263212AF03C
S3150802A5707DFD0DF05BFE642027F0ACFB0DF040FE7E
S3150802A58097F85B30052B04D1FFF7CCFE97F85B30C2
S3150802A5905AE1BB68002B00F0C580BC68F86C0FF066
S3150802A5A0B3FA034618460FF0C4FF03469C425CD929
S3150802A5B058E0F86C12F020F90246BB7819461046A4
S3150802A5C028F0A4FE87ED150A786DF6F7F1F802462B
S3150802A5D00B464E4816F0A4FF97ED157AD7ED147A76
S3150802A5E037EE678ABC68F86C0FF08EFA034618468F
S3150802A5F00FF09FFF0346E31A07EE903AF8EE677AE2
S3150802A600B4EEE78AF1EE10FA26DB97ED157AD7ED66
S3150802A610147A77EE677A17EE900AF6F7C9F8804643
S3150802A6208946386DF6F7C4F804460D46786DF6F78E
S3150802A630BFF802460B4607F11000CDE90223CDE921
S3150802A640004542464B4632492EF09CF807F1100364
S3150802A650184616F091FE08E0642027F03BFBFB6DD6
S3150802A660643BFB65FB6D002BA3DCFB6D002B5FD106
S3150802A67097ED157AD7ED147A77EE677A17EE900A80
S3150802A680F6F796F880468946386DF6F791F8044645
S3150802A6900D46786DF6F78CF802460B4607F1100060
S3150802A6A0CDE90223CDE9004542464B4619492EF02B
S3150802A6B069F807F11003184616F05EFE2AF058FFED
S3150802A6C0034618462AF06AFF03460921184629F066
S3150802A6D0CCFB2AF04FFC0123092263212AF0C6FC8F
S3150802A6E0072387F85B3023E004CD050814CD050857
S3150802A6F028CD050848CD050860CD05087CCD050896
S3150802A70098CD0508B4CD0508C8CD0508E8CD0508D5
S3150802A710F8CD05081CCE0508642027F0DBFAFB6D88
S3150802A720643BFB65FB6D002BF6DC4B4816F024FEFA
S3150802A7300EF0C4F90346032B26D0484816F01CFE31
S3150802A7400FF088F800200EF047FA0346002B17D1BF
S3150802A750042387F85B30424816F00EFE2AF008FFFB
S3150802A760034618462AF01AFF03460821184629F016
S3150802A7707CFB2AF0FFFB0123082263212AF076FCE0
S3150802A7800FF07EF80FF092F80EF06EFA0346032BDE
S3150802A79029D0344816F0F0FD0DF006FD00200EF023
S3150802A7A0A1FA0346002B17D1052387F85B302E48FA
S3150802A7B016F0E2FD2AF0DCFE034618462AF0EEFE03
S3150802A7C003460621184629F050FB2AF0D3FB01233B
S3150802A7D0062263212AF04AFC0DF028FD642027F0A0
S3150802A7E079FA0DF00DFD40F6B83027F073FA97F8AE
S3150802A7F05B30012B0AD12AF0BBFE034618462AF023
S3150802A800CDFE03460321184629F065FBF86C11F0C4
S3150802A810F3FF0246BB781946104628F077FD87ED06
S3150802A820150A786DF5F7C4FF02460B4607F11000C4
S3150802A8300E492DF0A7FF07F11003184616F09CFDE6
S3150802A840FFF770FD97F85B3018466037BD46BDECDA
S3150802A850028BBDE8B08300BF40CE05087CCD050853
S3150802A86098CD0508B4CD0508C8CD050854CE050807
S3150802A87090B587B000AF3C4684E80F000123FB750C
S3150802A880FB78012B4CD10EF075FA0346032B1DD02B
S3150802A890474816F071FD0DF09DFC00200EF0A8FA4F
S3150802A8A00346002B0BD10623FB75424816F064FDBE
S3150802A8B02AF060FB0123052263212AF0D7FB0DF05B
S3150802A8C0B5FC642027F006FA0DF09AFCFB7D062BF0
S3150802A8D001D1FB7D68E00DF08FFF0346032B1AD0EA
S3150802A8E0354816F049FD0EF09FFF00200EF012F8CB
S3150802A8F00346002B0BD10323FB75304816F03CFDAB
S3150802A9002AF038FB0123072263212AF0AFFB0EF057
S3150802A910B7FF0EF0CBFFFB7D032B44D1FB7D43E053
S3150802A9200EF0CCF80346032B1AD0254816F024FD60
S3150802A9300EF090FF00200EF04FF90346002B0BD1C4
S3150802A9400423FB751F4816F017FD2AF013FB012393
S3150802A950082263212AF08AFB0EF092FF0EF0A6FF68
S3150802A9600EF082F90346032B1DD0174816F004FD94
S3150802A9700DF01AFC00200EF0B5F90346002B0BD198
S3150802A9800523FB75114816F0F7FC2AF0F3FA0123A2
S3150802A990062263212AF06AFB0DF048FC642027F0A0
S3150802A9A099F90DF02DFCFB7D18461C37BD4690BD66
S3150802A9B014CD050828CD050848CD050860CD05083B
S3150802A9C07CCD050898CD0508B4CD0508C8CD05087F
S3150802A9D090B587B000AF3C4684E80F000123FB75AB
S3150802A9E0FB78002B2CD10DF007FF0346032B00F052
S3150802A9F0C180634816F0C0FC0EF016FF00200DF069
S3150802AA0089FF0346002B16D10323FB755D4816F012
S3150802AA10B3FC2AF0ADFD034618462AF0BFFD0346ED
S3150802AA200721184629F021FA2AF0A4FA0123072257
S3150802AA3063212AF01BFB0EF023FF0EF037FF99E085
S3150802AA40FB78012B5CD10EF039F80346032B2BD188
S3150802AA500EF034F80346032B26D14B4816F08CFC2D
S3150802AA600EF0F8FE00200EF0B7F80346002B16D1BA
S3150802AA700423FB75454816F07FFC2AF079FD034648
S3150802AA8018462AF08BFD03460821184629F0EDF9E7
S3150802AA902AF070FA0123082263212AF0E7FA0EF057
S3150802AAA0EFFE0EF003FF65E00EF008F80346032BEF
S3150802AAB060D0354816F060FC0EF0CCFE00200EF091
S3150802AAC08BF80346002B16D10423FB752F4816F084
S3150802AAD053FC2AF04DFD034618462AF05FFD03464D
S3150802AAE00821184629F0C1F92AF044FA0123082256
S3150802AAF063212AF0BBFA0EF0C3FE0EF0D7FE39E048
S3150802AB00FB78022B36D10DF077FE0346032B04D1D0
S3150802AB100DF0D4FF0346032B2CD01D4816F02CFC4F
S3150802AB200EF082FE00200DF081FF0346002B16D19F
S3150802AB300323FB75174816F01FFC2AF019FD034676
S3150802AB4018462AF02BFD03460721184629F08DF9E7
S3150802AB502AF010FA0123072263212AF087FA4FF412
S3150802AB602F7027F0B7F80EF08BFE642027F0B2F8A4
S3150802AB700EF09CFEFB7D18461C37BD4690BD00BFF5
S3150802AB8064CE050880CE0508A0CE0508C0CE050805
S3150802AB90E4CE050808CF050890B587B000AF3C4655
S3150802ABA084E80F000023FB750EF05EF80346032BBC
S3150802ABB01ED0874816F0E0FB0DF0F6FA00200EF0DC
S3150802ABC091F80346002B0CD1FB7D0133FB758148B6
S3150802ABD016F0D2FB2AF0CEF90123062263212AF0C7
S3150802ABE045FA0DF023FB642027F074F80DF008FBF4
S3150802ABF00DF064FF0346032B26D0774816F0BCFBFC
S3150802AC000EF028FE00200DF0E7FF0346002B17D1B1
S3150802AC10FB7D0133FB75714816F0AEFB2AF0A8FCE2
S3150802AC20034618462AF0BAFC03460821184629F0B4
S3150802AC301CF92AF09FF90123082263212AF016FA41
S3150802AC400EF01EFE0EF032FEFB7D002B01D0FB7DC0
S3150802AC50BAE00EF08FF80346032B1ED0604816F0B2
S3150802AC608BFB0DF0B7FA00200EF0C2F80346002B54
S3150802AC700CD1FB7D0133FB755A4816F07DFB2AF091
S3150802AC8079F90123052263212AF0F0F90DF0CEFAAB
S3150802AC90642027F01FF80DF0B3FA0DF0ADFD034658
S3150802ACA0032B26D0504816F067FB0EF0BDFD002098
S3150802ACB00DF030FE0346002B17D1FB7D0133FB75E1
S3150802ACC04A4816F059FB2AF053FC034618462AF05E
S3150802ACD065FC03460721184629F0C7F82AF04AF9FF
S3150802ACE00123072263212AF0C1F90EF0C9FD0EF0ED
S3150802ACF0DDFD0DF0E3FE0346032B26D0364816F09B
S3150802AD003BFB0EF0A7FD00200DF066FF0346002B65
S3150802AD1017D1FB7D0133FB75304816F02DFB2AF05F
S3150802AD2027FC034618462AF039FC0346082118462A
S3150802AD3029F09BF82AF01EF90123082263212AF03A
S3150802AD4095F90EF09DFD0EF0B1FD0DF08DFF03464F
S3150802AD50032B1ED01E4816F00FFB0DF025FA002015
S3150802AD600DF0C0FF0346002B0CD1FB7D0133FB75AA
S3150802AD70184816F001FB2AF0FDF801230622632182
S3150802AD802AF074F90DF052FA642026F0A3FF0DF0AA
S3150802AD9037FA052005F084FCFFF73AF90346012B3A
S3150802ADA004D0FFF735F90346002B0CD10EF01EFE30
S3150802ADB003460121184610F0A1FD42F2107026F052
S3150802ADC089FFFFF7AFFAFB7D18461C37BD4690BDD3
S3150802ADD0B4CD0508C8CD0508A0CE0508C0CE05081D
S3150802ADE014CD050828CD050864CE050880CE0508C9
S3150802ADF090B585B000AF78600023FB7378680FF0D2
S3150802AE0047FD0346002B32D0786810F057FB0346FD
S3150802AE10002B1BD1786811F0B7FE0346002B26D00B
S3150802AE200021786811F027FC0446786811F0CAFEFA
S3150802AE3003469C421BD30121786811F01CFC044688
S3150802AE40786811F0DDFE03469C4210D300F0DEFE60
S3150802AE500346002B0BD10221786811F020FF034626
S3150802AE6083F00103DBB2002B01D00123FB73FB7BCA
S3150802AE7018461437BD4690BDB0B582B000AF0EF085
S3150802AE80B5FD7860786810F065FD0346002B6DD035
S3150802AE90786811F0DAF851EC100B3EA3D3E90023D7
S3150802AEA0F5F750FF0346002B07D0374B1B7803F004
S3150802AEB00103DAB2344B1A7002E0334B00221A70DD
S3150802AEC0786811F0C2F855EC104B78680EF01CFE43
S3150802AED0034618460FF0EBFA10EE103A1846F5F745
S3150802AEE067FC27A3D3E90023F5F702FB02460B46C4
S3150802AEF020462946F5F744FF0346002B07D0234B85
S3150802AF001B7803F00103DAB2204B1A7002E01F4BDA
S3150802AF1000221A701E4B1B885A1C91B21C4A1180B9
S3150802AF20282B26D9184B1B78002B04D001217868C8
S3150802AF3010F0EFFA03E00021786810F0EAFA134BF2
S3150802AF401B78002B04D00121786810F0C4FA03E0BC
S3150802AF500021786810F0BFFA0B4B01221A700B4BCE
S3150802AF6001221A700A4B00221A8002E0084B0022BC
S3150802AF701A8000BF0837BD46B0BD00BFAFF30080D8
S3150802AF809A9999999999A93F55D1002054D10020A7
S3150802AF9056D10020666666666666024080B582B04D
S3150802AFA000AF0EF023FD7860264B1B78022B2CD0BF
S3150802AFB0022B3CDC002B02D0012B12D037E078683A
S3150802AFC011F0BBFA0346142B33DD1F4816F0D4F9E9
S3150802AFD01E4B00221A600DF099FB1A4B01221A70B9
S3150802AFE027E01A4B1B685A1C18490A60B3F5967F64
S3150802AFF021D9174816F0C0F9144B00221A600DF031
S3150802B00091FB104B02221A7015E0104B1B685A1C52
S3150802B0100E490A60B3F5E16F0FD90E4816F0ACF97E
S3150802B0200A4B00221A60074B00221A7005E000BF7D
S3150802B03004E000BF02E000BF00E000BF00BF08371F
S3150802B040BD4680BDF8D000202CCF050858D1002077
S3150802B0503CCF050854CF050880B500AF0EF0C6FCF4
S3150802B0600346184610F03CFC0346002B11D00C4B45
S3150802B0701B88643B9AB20A4B1A80094B1B88002B21
S3150802B0800BD10EF0B3FC03460021184610F004FC5F
S3150802B09003E0034B4FF4FA521A8000BF80BD00BF8B
S3150802B0A02200002080B582B000AF0023FB710EF0AB
S3150802B0B09DFC0346184610F013FC0346002B02D0EB
S3150802B0C05023FB7101E02823FB71FB7918460837E8
S3150802B0D0BD4680BD00000000B0B582B000AF0EF0DC
S3150802B0E085FC786029F046FF034603226321184649
S3150802B0F029F07EFF0346002B59D1786810F0A5FF88
S3150802B10051EC100B4FF00002B64BF5F72FFE034633
S3150802B110002B49D0B44B1B680133B34A1360FFF7BF
S3150802B120C1FF03461A46B04B1B689A423FD200211A
S3150802B130786810F0E3FB0021786810F081FD00F0D2
S3150802B14065FD0346022B12D000F060FD0346032B71
S3150802B1500DD000F05BFD0346052B08D000F056FD26
S3150802B1600346062B03D00021786810F07BFA9F4825
S3150802B17016F002F92AF0FCF9034618462AF00EFAE6
S3150802B18003460321184628F070FE29F0F3FE012330
S3150802B1900322632129F06AFF002178680FF076FC02
S3150802B1A0914B00221A6002E08F4B00221A607868DF
S3150802B1B010F0D0FB0346002B50D029F0DBFE0346E5
S3150802B1C004226321184629F013FF0346002B45D1B2
S3150802B1D0786810F03AFF51EC100B4FF00002844BDE
S3150802B1E0F5F7BAFD0346002B35D0824B1B680133AF
S3150802B1F0804A1360FFF756FF03461A467D4B1B68C3
S3150802B2009A422BD20021786810F078FB00217868E0
S3150802B21010F016FD0021786810F024FA764816F028
S3150802B220ABF82AF0A5F9034618462AF0B7F90346F9
S3150802B2300421184628F019FE29F09CFE012304224F
S3150802B240632129F013FF002178680FF01FFC694B70
S3150802B25000221A6002E0674B00221A60674B1B78CD
S3150802B260062B00F2DF8101A252F823F089B2020806
S3150802B270E1B2020825B6020899B3020821B4020807
S3150802B280F3B4020833B502085D4B1B68002B07D1DD
S3150802B2900121786810F032FB0121786810F0D0FCA1
S3150802B2A0574B1B685A1C56490A60962B40F2BC81BA
S3150802B2B0544816F061F8786811F00FFF0346012B1F
S3150802B2C007D00021786810F019FB0021786810F081
S3150802B2D0B7FC4B4B00221A60484B01221A70A3E1B5
S3150802B2E0786810F027F90346002B13D000F08EFC7D
S3150802B2F00346002B1AD000F089FC0346052B15D00D
S3150802B300414B1B78002B11D178680FF0C1FA03461E
S3150802B310002B0BD0786811F068FE0346002B20D06C
S3150802B320786810F0E9F80346002B1AD1374816F068
S3150802B33023F80121786810F0E1FA0121786810F003
S3150802B3407FFC0121786810F08DF90121786810F0E8
S3150802B350B1FB0121786810F0F9F9284B03221A701B
S3150802B36064E1274B1B685A1C25490A60B3F5616FCD
S3150802B37040F25C81264815F0FFFF0121786810F03B
S3150802B380BDFA0121786810F05BFC1D4B00221A6099
S3150802B3901A4B05221A7049E1786810F0ADF803468F
S3150802B3A0002B00F045817868FFF722FD0346002B43
S3150802B3B00AD0184B4FF4FA621A60174815F0DCFFE8
S3150802B3C00E4B04221A7033E1144815F0D5FF0021FA
S3150802B3D0786810F047F90A4B00221A60074B0622D2
S3150802B3E01A7025E100000C40FCD0002060CF050849
S3150802B3F00000F83F00D1002074CF05082100002084
S3150802B4005CD1002084CF050896D1002090CF05088C
S3150802B410A0CF050860D10020B0CF0508D0CF050817
S3150802B4208B4B1B68643B8A4A1360894B1B68002B4B
S3150802B43046D10121786810F0A9F80021786810F041
S3150802B44011F9844B00221A60834B00221A60834B3F
S3150802B45000221A60786811F097FB0346002B1FD06A
S3150802B4600021786811F007F90446786811F0AAFBFA
S3150802B47003469C4214D30121786811F0FCF804466D
S3150802B480786811F0BDFB03469C4209D3744815F04F
S3150802B49073FF744B744A1A60062000F0A5FB05E098
S3150802B4A0724815F069FF022000F09EFB01217868B8
S3150802B4B010F05EFA6E4815F05FFF6E4B06221A70A0
S3150802B4C078680FF0E5F90346002B40F0B3806A4B23
S3150802B4D000221A600021786810F0C4F80021786802
S3150802B4E010F054F8624815F047FF624B06221A70AC
S3150802B4F0A0E0614B1B685A1C5F490A60962B40F212
S3150802B5009B805E4815F038FF786811F0E6FD034621
S3150802B510012B07D00021786810F0F0F9002178682D
S3150802B52010F08EFB544B00221A60524B01221A70FD
S3150802B53082E0514B1B685A1C4F490A6040F2DC52A2
S3150802B54093422DD8786811F050FD0346002B19D086
S3150802B550786810F07AFD55EC104B78680EF0D4FA3C
S3150802B560034618460EF0C4FF10EE103A1846F5F7D1
S3150802B5701FF902460B4620462946F5F7E3FB034622
S3150802B580002B0DD1786810F060FD51EC100B2EA33C
S3150802B590D3E90023F5F7D6FB0346002B00D14CE08E
S3150802B5A0364815F0E9FE786811F01FFD0346002BB0
S3150802B5B01DD0786810F049FD55EC104B78680EF0EE
S3150802B5C0A3FA034618460EF093FF10EE103A1846F1
S3150802B5D0F5F7EEF802460B4620462946F5F7B2FB82
S3150802B5E00346002B03D0264815F0C6FE13E07868FA
S3150802B5F011F073FD0346012B0DD0786811F0F5FCA6
S3150802B6000346002B07D10021786810F077F900214C
S3150802B610786810F015FB184B00221A60154B0122A8
S3150802B6201A700AE000BF08E000BF06E000BF04E0A7
S3150802B63000BF02E000BF00E000BF00BF0837BD46FA
S3150802B640B0BD00BFAFF30080333333333333034027
S3150802B65060D100207CD1002080D1002084D1002036
S3150802B660E0CF05082400002040771B00F4CF050828
S3150802B670D0CF0508210000205CD1002084CF050820
S3150802B68004D0050880B500AF29F074FC03460122F0
S3150802B6906321184629F0ACFC0346002B4CD129F04D
S3150802B6A069FC034603226321184629F0A1FC0346D6
S3150802B6B0002B41D129F05EFC034604226321184679
S3150802B6C029F096FC0346002B36D129F053FC034693
S3150802B6D005226321184629F08BFC0346002B2BD141
S3150802B6E029F048FC034606226321184629F080FC05
S3150802B6F00346002B20D129F03DFC0346072263218D
S3150802B700184629F075FC0346002B15D129F032FCA0
S3150802B710034608226321184629F06AFC0346002BD1
S3150802B7200AD129F027FC034608226321184629F084
S3150802B7305FFC0346002B01D0012300E000231846D4
S3150802B74080BD00000000000080B500AFFFF79AFF39
S3150802B7500346002B14D00EF049F903460121184678
S3150802B76011F06EFC0346002B32D01D4815F004FE7C
S3150802B7700EF03CF903460121184611F091FC27E028
S3150802B7800EF034F903460121184611F059FC034616
S3150802B79083F00103DBB2002B1AD00EF027F9034619
S3150802B7A0184610F052FC51EC100B0BA3D3E90023F8
S3150802B7B0F5F7E6FA0346002B00D109E0094815F029
S3150802B7C0DBFD0EF013F903460121184611F050FC71
S3150802B7D000BF80BDAFF300803333333333330340C6
S3150802B7E020D005083CD0050880B500AF114B1B6870
S3150802B7F05A1C10490A60052B1AD90EF0F7F80346A7
S3150802B80018460FF0B5FE0346002B07D029F0B2FB07
S3150802B81000230222632129F08AFC06E029F0AAFB0A
S3150802B82002230222632129F021FC024B00221A601C
S3150802B83000BF80BD64D1002080B58CB008AF7860A7
S3150802B8407B68FB6040221A491A4806F0ADFA78214D
S3150802B850052004F00BFF07F1080100234FF480527C
S3150802B860F86826F0CDFF0346002B01D002231AE022
S3150802B870BB68B022069201220592002204920A228D
S3150802B88003920A2202924FF48052019200930023F5
S3150802B890094A0A490A4827F0F9F90346002B01D052
S3150802B8A00E2300E0002318461037BD4680BD00BFB0
S3150802B8B014D1002004D10020C5B8020854D00508C6
S3150802B8C048D00020B0B588B002AF78600EF08EF886
S3150802B8D0F86000237B810023FB754FF4E1633B612B
S3150802B8E0BC4806F0EBFA034683F00103DBB2002BF1
S3150802B8F000F06481B848FEF737FC03467B817B89F2
S3150802B900002B00F06281B44B1B78013B032B00F23B
S3150802B910528101A252F823F029B9020839BA02085B
S3150802B92057BA0208A7BA020829F022FE03461846A1
S3150802B93029F034FE03460221184628F0CCFA0121E2
S3150802B940F86811F0D7FB0121F8680FF0D7FF01213B
S3150802B950F86810F075F91FE0F86810F076FB55ECF8
S3150802B960104BF8680EF0D0F8034618460EF0C0FDE4
S3150802B97010EE103A1846F4F71BFF02460B4620460D
S3150802B9802946F5F7FDF90346002B0BD1052004F0ED
S3150802B99087FE642026F09EF93B695A1E3A61002BFF
S3150802B9A0DAD100E000BF3B69002B36D08A4B5B68D0
S3150802B9B0002B03D1884B9B68002B06D0864B0FCBF6
S3150802B9C0FEF7DAFC0346FB750AE029F0D1FD0346C9
S3150802B9D0184629F0E3FD03460321184628F07BFAA8
S3150802B9E07D4B5B78002B1BD1FB7D012B06D17A4B55
S3150802B9F01B7B012118460CF0D1F811E00321F868E7
S3150802BA0011F0E2FA0021F8680FF040F8724B1B7B3E
S3150802BA10022118460CF0C2F802E0704815F0ACFC98
S3150802BA200021F86811F0EEFA4FF4E1633B61002158
S3150802BA30F86811F05FFBC1E0674B0FCBFEF718FF02
S3150802BA400346012B03D101200CF060FBB6E002206D
S3150802BA500CF05CFBB2E0604BDB78022B08D10021CC
S3150802BA60F8680FF04BFF0021F86810F0E9F80BE0D0
S3150802BA70594BDB78012B07D10121F8680FF03EFFFD
S3150802BA800121F86810F0DCF8534B0FCBFEF7A0FF44
S3150802BA900346012B03D101200CF038FB8EE002206D
S3150802BAA00CF034FB8AE04E4815F03AFD29F062FAAA
S3150802BAB00023009300230122632129F0F1FB29F0D8
S3150802BAC059FA0023009300230222632129F0E8FB96
S3150802BAD029F050FA0023009300230322632129F058
S3150802BAE0DFFB29F047FA002300930023042263218F
S3150802BAF029F0D6FB29F03EFA0023009300230522FB
S3150802BB00632129F0CDFB29F035FA0023009300239F
S3150802BB100622632129F0C4FB29F02CFA002300939C
S3150802BB2000230722632129F0BBFB29F023FA00230D
S3150802BB30009300230822632129F0B2FB29F01AFA9E
S3150802BB400023009300230922632129F0A9FB29F087
S3150802BB500FFD0346184629F021FD03460021184623
S3150802BB6028F083F91C4B0FCBFFF716F80346002B78
S3150802BB7019D11C4815F0D4FC174B5B78002B1CD145
S3150802BB8001200CF099FA0021F86811F0B3FA29F0AD
S3150802BB90EFFC0346184629F001FD03460121184623
S3150802BBA028F099F909E00C4B5B78002B05D10220A5
S3150802BBB00CF082FA01E000BF00E000BF052004F0A5
S3150802BBC06FFD642026F086F88AE600BF1837BD4660
S3150802BBD0B0BD00BF04D1002068D100206CD0050892
S3150802BBE08CD005089CD0050880B483B000AF034604
S3150802BBF0FB71054AFB791370012318460C37BD46BB
S3150802BC005DF8047B704700BF79D1002080B400AF8D
S3150802BC10034B1B781846BD465DF8047B704700BF88
S3150802BC2079D1002080B582B000AF7860214B1B78AD
S3150802BC30062B34D801A252F823F000BF59BC0208D9
S3150802BC4063BC02086DBC020877BC020881BC020804
S3150802BC508BBC020895BC0208174978682CF092FD3D
S3150802BC6022E0164978682CF08DFD1DE014497868A3
S3150802BC702CF088FD18E0134978682CF083FD13E050
S3150802BC80114978682CF07EFD0EE0104978682CF090
S3150802BC9079FD09E00E4978682CF074FD04E00D4937
S3150802BCA078682CF06FFD00BF7B6818460837BD46DA
S3150802BCB080BD00BF79D10020B0D00508BCD00508E8
S3150802BCC0C8D00508D8D00508ECD0050800D1050863
S3150802BCD014D1050824D1050880B483B000AF034601
S3150802BCE0FB71054AFB791370012318460C37BD46CA
S3150802BCF05DF8047B704700BF78D1002080B400AF9E
S3150802BD00034B1B781846BD465DF8047B704700BF97
S3150802BD1078D1002080B582B000AF78601F4B1B78BF
S3150802BD20072B31D801A252F823F000BF4DBD0208F5
S3150802BD3057BD020861BD02086BBD020875BD02083F
S3150802BD4089BD020889BD02087FBD020814497868C0
S3150802BD502CF018FD1DE0134978682CF013FD18E045
S3150802BD60114978682CF00EFD13E0104978682CF01A
S3150802BD7009FD0EE00E4978682CF004FD09E00D492C
S3150802BD8078682CF0FFFC04E00B4978682CF0FAFC82
S3150802BD9000BF7B6818460837BD4680BD78D10020AB
S3150802BDA034D1050840D105084CD105085CD10508EF
S3150802BDB06CD1050880D1050890D1050880B483B0F6
S3150802BDC000AF0346FB71054AFB7913700123184637
S3150802BDD00C37BD465DF8047B704700BF8CD1002046
S3150802BDE080B500AF40220349034805F0DDFF00BFD6
S3150802BDF080BD00BFA8D1002098D1002080B582B0AE
S3150802BE0000AF78600B467B807B881A4679680448BF
S3150802BE1006F0DFF9034618460837BD4680BD00BF5F
S3150802BE2098D1002080B582B000AF7860796804485E
S3150802BE3006F0E0F903469BB218460837BD4680BDB0
S3150802BE4098D1002080B400AF034B1B681846BD4644
S3150802BE505DF8047B704700BF88D1002080B485B0A6
S3150802BE6000AF7860084B1A687B681340002B14BF32
S3150802BE7001230023DBB2FB60FB6818461437BD4674
S3150802BE805DF8047B704700BF88D1002080B483B078
S3150802BE9000AF7860064B1A687B681343044A13603E
S3150802BEA0012318460C37BD465DF8047B704700BF70
S3150802BEB088D1002080B483B000AF78607B68DA430B
S3150802BEC0054B1B681340044A1360012318460C37B6
S3150802BED0BD465DF8047B704788D1002080B590B0D6
S3150802BEE002AF3B600346FB710B46BB7113467B717F
S3150802BEF0012387F82C30FB7987F82D30BB7987F830
S3150802BF002E307B7987F82F303B683B63B7F8403091
S3150802BF107B6397F82F3019463A6B7B6B07F10C0057
S3150802BF20009313460A4609492CF02CFC07F10C0328
S3150802BF30184615F021FA07F12C030C211846FFF7CB
S3150802BF405DFF00BF3837BD4680BD00BFA0D10508DA
S3150802BF5080B584B000AF0023FB810023BB81002398
S3150802BF607B8100233B810DF041FD786078680DF0F6
S3150802BF70CBFD38600021786810F07DFB0346BB8153
S3150802BF800121786810F077FB03467B8102217868E5
S3150802BF9010F071FB0346FB810521786810F06BFBF4
S3150802BFA003463B81FB8940F2DB52934207D8864B14
S3150802BFB01B7803F00103DAB2834B1A7002E0824B54
S3150802BFC000221A70786810F085FD0346002B25D0EA
S3150802BFD0BB8940F6340293420CD97B8940F6340277
S3150802BFE0934207D9794B1B7803F00103DAB2774BF0
S3150802BFF01A7002E0754B00221A707B8940F2DB52F6
S3150802C000934207D8724B1B7803F00103DAB2704BDE
S3150802C0101A7095E06E4B00221A7091E0BB8940F6C1
S3150802C020340293420CD97B8940F63402934207D9EB
S3150802C030664B1B7803F00103DAB2644B1A7002E00E
S3150802C040624B00221A700DF0D1FC0346184610F016
S3150802C05043FF0346012B10D1BB8940F26B72934210
S3150802C06007D85B4B1B7803F00103DAB2584B1A70F8
S3150802C07066E0574B00221A7062E038680DF021FF1D
S3150802C0800346012B1CD17B89B3F5967F07D2504B09
S3150802C0901B7803F00103DAB24D4B1A7050E0BB89E4
S3150802C0A040F26B72934207D8494B1B7803F001039F
S3150802C0B0DAB2474B1A7043E0454B00221A703FE04A
S3150802C0C038680DF0FEFE0346022B10D1BB8940F2FA
S3150802C0D06B72934207D83E4B1B7803F00103DAB220
S3150802C0E03B4B1A702CE03A4B00221A7028E038684B
S3150802C0F00DF0E7FE0346032B0FD1BB89B3F5966F06
S3150802C10007D2334B1B7803F00103DAB2304B1A70AD
S3150802C11016E02F4B00221A7012E0BB89B3F5167F80
S3150802C1200BD27B89B3F5167F07D2294B1B7803F00E
S3150802C1300103DAB2264B1A7002E0254B00221A7066
S3150802C1403B8940F2DB52934207D8224B1B7803F015
S3150802C1500103DAB21F4B1A7002E01E4B00221A7054
S3150802C1601D4B1B785A1CD1B21B4A1170092B26D9B2
S3150802C170154B1B78194678680FF040F9134B1B7854
S3150802C180194678680FF06BF9114B1B7819467868CF
S3150802C1900FF083F90F4B1B78194678680FF0D7F919
S3150802C1A00D4B00221A70084B01221A70074B012206
S3150802C1B01A70074B01221A70064B01221A7000BF29
S3150802C1C01037BD4680BD00BF280000202900002088
S3150802C1D02A0000202B000020C8D2002080B483B099
S3150802C1E000AF7860044A7B681360012318460C374F
S3150802C1F0BD465DF8047B7047E8D1002080B500AFE4
S3150802C200204B1B68092B1AD80DF0F0FB03460021B8
S3150802C21018460FF085FC29F0ABF90346184629F0B3
S3150802C220BDF903461521184627F02CFD01210120E8
S3150802C2300BF07FFC144815F09FF8002320E00DF060
S3150802C240D5FB034618460FF093FC0346002B11D183
S3150802C2500DF0CCFB0346012118460FF061FC29F0CC
S3150802C26087F90346184629F099F903461421184610
S3150802C27027F008FD034B1B680A3B024A1360012399
S3150802C280184680BDE8D10020B8D1050880B483B02D
S3150802C29000AF7860044A7B681360012318460C379E
S3150802C2A0BD465DF8047B7047ECD1002080B500AF2F
S3150802C2B0254B1B68632B21D80DF0BAF90DF096FBB6
S3150802C2C00346002118460FF060FC29F051F903468F
S3150802C2D0184629F063F903461521184627F0D2FCB9
S3150802C2E0012102200BF025FC184815F045F86420B8
S3150802C2F025F0F0FC0DF0B2F9002322E00DF076FBF2
S3150802C300034618460FF052FC0346002B11D129F0BA
S3150802C3102FF90346184629F041F90346142118460F
S3150802C32027F0B0FC0DF062FB0346012118460FF018
S3150802C3302CFC0DF051F9044B1B68643B024A13604E
S3150802C3400123184680BD00BFECD10020C8D10508DC
S3150802C35080B500AF154B1B68632B1DD80DF068F925
S3150802C3600DF044FB0346002118460FF00EFC29F097
S3150802C370FFF80346184629F011F90346152118460F
S3150802C38027F080FC0A4814F0F7FF642025F0A2FC87
S3150802C3900DF064F9002307E00DF034F9034B1B682E
S3150802C3A0643B024A13600123184680BDECD1002083
S3150802C3B0D8D1050880B500AF164B1B780B2B18D0C1
S3150802C3C00B2B1CDC002B02D00A2B09D017E00DF030
S3150802C3D019F9104B1B780133DAB20E4B1A7015E0B5
S3150802C3E00DF026F90B4B1B780133DAB2094B1A709A
S3150802C3F00CE00DF033F9074B00221A7006E0054BE4
S3150802C4001B780133DAB2034B1A7000BF014B1B7853
S3150802C410184680BDC9D2002080B483B000AF7860C8
S3150802C420044A7B681360012318460C37BD465DF83B
S3150802C430047B7047F0D1002080B500AF254B1B68FE
S3150802C440632B21D80DF060F90DF0D0FA03460021CE
S3150802C45018460FF0B8FB29F08BF80346184629F060
S3150802C4609DF803461521184627F00CFC01210320E6
S3150802C4700BF05FFB184814F07FFF642025F02AFCB6
S3150802C4800DF058F9002322E00DF0B0FA03461846DB
S3150802C4900FF0AAFB0346002B11D129F069F80346CF
S3150802C4A0184629F07BF803461421184627F0EAFBBA
S3150802C4B00DF09CFA0346012118460FF084FB0DF095
S3150802C4C0F7F8044B1B68643B024A136001231846BB
S3150802C4D080BD00BFF0D10020ECD1050880B500AFC1
S3150802C4E0164B1B780B2B18D00B2B1CDC002B02D0FF
S3150802C4F00A2B09D017E00DF0F1F8104B1B7801331F
S3150802C500DAB20E4B1A7015E00DF0FEF80B4B1B78DB
S3150802C5100133DAB2094B1A700CE00DF00BF9074B2E
S3150802C52000221A7006E0054B1B780133DAB2034B78
S3150802C5301A7000BF014B1B78184680BDCAD200206C
S3150802C54080B500AF154B1B68632B1DD80DF0DCF8C0
S3150802C5500DF04CFA0346002118460FF034FB29F079
S3150802C56007F80346184629F019F80346152118460E
S3150802C57027F088FB0A4814F0FFFE642025F0AAFB80
S3150802C5800DF0D8F8002307E00DF0A8F8034B1B6856
S3150802C590643B024A13600123184680BDF0D100208D
S3150802C5A0FCD1050880B483B000AF7860044A7B6882
S3150802C5B01360012318460C37BD465DF8047B7047A5
S3150802C5C0F4D1002080B500AF254B1B68632B21D818
S3150802C5D00DF006F90DF00AFA0346002118460FF087
S3150802C5E010FB28F0C5FF0346184628F0D7FF034676
S3150802C5F01521184627F046FB012105200BF099FA6A
S3150802C600184814F0B9FE642025F064FB0DF0FEF814
S3150802C610002322E00DF0EAF9034618460FF002FB62
S3150802C6200346002B11D128F0A3FF0346184628F02B
S3150802C630B5FF03461421184627F024FB0DF0D6F958
S3150802C6400346012118460FF0DCFA0DF09DF8044B5B
S3150802C6501B68643B024A13600123184680BD00BF6B
S3150802C660F4D1002010D2050880B500AF1E4B1B6816
S3150802C670632B28D80CF0DCFF0DF046F80DF0B6F95E
S3150802C6800346002118460FF080FA0DF0AFF903466B
S3150802C690002118460FF097FA28F06AFF0346184653
S3150802C6A028F07CFF03461521184627F0EBFA0F48B7
S3150802C6B014F062FE642025F00DFB0CF0CFFF0DF09E
S3150802C6C039F800230EE00CF09DFF0DF007F8084B31
S3150802C6D01B68643B064A1360034B1B68643B024AA9
S3150802C6E013600123184680BDF0D1002034D2050814
S3150802C6F0ECD1002080B500AF314B1B68632B2CD8D8
S3150802C7000CF096FF0DF000F80DF070F903460021C3
S3150802C71018460FF03AFA0DF069F903460021184651
S3150802C7200FF051FA28F024FF0346184628F036FF80
S3150802C73003461521184627F0A5FA012104200BF015
S3150802C740F8F9204814F018FE642025F0C3FA0CF014
S3150802C75085FF0CF0EFFF002330E00DF047F90346A2
S3150802C76018460FF023FA0346002B18D128F000FFCB
S3150802C7700346184628F012FF03461421184627F0E6
S3150802C78081FA0DF033F90346012118460FF0FDF937
S3150802C7900DF02CF90346012118460FF014FA0CF095
S3150802C7A01BFF0CF085FF084B1B68643B064A1360A7
S3150802C7B0034B1B68643B024A13600123184680BD7B
S3150802C7C0F0D1002034D20508ECD10020F0B593B0A0
S3150802C7D004AF03460A46FB711346BB80BB8807EEC5
S3150802C7E0903AF8EE677AC7ED0D7AFB79002B00F0DE
S3150802C7F0CA80FB79042B00F2C680FB79012B19D17A
S3150802C8000DF0F4F8034618460FF076FFB0EE407ABC
S3150802C810D7ED0D7A77EE877AC7ED0D7A0DF0E6F841
S3150802C820034618460FF068FFF0EE407A584BC3ED00
S3150802C830047A55E0FB79022B19D10DF0D7F8034695
S3150802C84018460FF079FFB0EE407AD7ED0D7A77EEFB
S3150802C850877AC7ED0D7A0DF0C9F8034618460FF028
S3150802C8606BFFF0EE407A4A4BC3ED047A38E0FB7967
S3150802C870032B19D10DF0BAF8034618460FF07CFFC0
S3150802C880B0EE407AD7ED0D7A77EE877AC7ED0D7A54
S3150802C8900DF0ACF8034618460FF06EFFF0EE407A3C
S3150802C8A03B4BC3ED047A1BE0FB79042B18D10DF040
S3150802C8B09DF8034618460FF07FFFB0EE407AD7ED93
S3150802C8C00D7A77EE877AC7ED0D7A0DF08FF8034663
S3150802C8D018460FF071FFF0EE407A2D4BC3ED047A3D
S3150802C8E02B4A7B6B5360FB7907EE903AF8EE677A30
S3150802C8F0274BC3ED007A264B4FF000029A60244B71
S3150802C9000022DA60224B00225A61214B00229A61E8
S3150802C9101F4B4FF00002DA61D7ED0D7AB1EE047AB9
S3150802C92077EEC77A1A4BC3ED087A194B1B69184A70
S3150802C9305362174B01229A62154B002283F82C2068
S3150802C940134B00221A63FE79114B1B691846F3F73B
S3150802C9502FFF04460D460E4B5B681846F3F728FF71
S3150802C96002460B4607F10C00CDE90223CDE9004544
S3150802C970324608492BF006FF07F10C03184614F055
S3150802C980FBFC012300E0002318463C37BD46F0BDF8
S3150802C990F8D1002054D205082DE9B04398B004AF67
S3150802C9A04FF00003FB644FF00003BB64A44BD3EDC6
S3150802C9B0007AB7EE007AF4EE477AF1EE10FA08D169
S3150802C9C00DF014F8034618460FF096FE87ED130A83
S3150802C9D037E09B4BD3ED007AB0EE007AF4EE477A55
S3150802C9E0F1EE10FA08D10DF001F8034618460FF0D9
S3150802C9F0A3FE87ED130A24E0914BD3ED007AB0EE3D
S3150802CA00087AF4EE477AF1EE10FA08D10CF0EEFF46
S3150802CA10034618460FF0B0FE87ED130A11E0884B5D
S3150802CA20D3ED007AB1EE007AF4EE477AF1EE10FA17
S3150802CA3007D10CF0DBFF034618460FF0BDFE87ED63
S3150802CA40130AF86CF3F7B4FE04460D467C4B5B6892
S3150802CA501846F3F7ADFE02460B46CDE900232246F9
S3150802CA602B46784814F05CFD754BD3ED087A97EDA2
S3150802CA70137AB4EEE77AF1EE10FAC0F27D810CF081
S3150802CA80B5FF0346002118460FF04AF86C4B002200
S3150802CA90DA606B4BD3ED087AF5EEC07AF1EE10FA4E
S3150802CAA000F28D80664BD3ED017AB1EE047A77EE09
S3150802CAB0C77A97ED137AB4EEE77AF1EE10FA32DD19
S3150802CAC05F4BDB691846F3F773FE04460D46F86CAE
S3150802CAD0F3F76EFE02460B4607F10C00CDE900237A
S3150802CAE022462B4658492BF04DFE07F10C031846F1
S3150802CAF014F042FC28F03CFD0346184628F04EFD89
S3150802CB0003461521184627F0BDF8012101200BF02E
S3150802CB1010F84B4B4FF000025A60494B4FF0000297
S3150802CB209A60002307E3494B1B785A1CD1B2474A3D
S3150802CB301170C72B41D9424BDB691846F3F738FE09
S3150802CB40804689463E4B1B6A1846F3F731FE044671
S3150802CB500D46F86CF3F72CFE02460B4607F10C005D
S3150802CB60CDE90223CDE9004542464B4638492BF02A
S3150802CB7009FE07F10C03184614F0FEFB334B00229C
S3150802CB801A70344B01221A702D4BD3ED007AFCEE43
S3150802CB90E77AC7ED017A3B79DBB2294A92ED017A47
S3150802CBA0D7ED137A77EE677AFCEEE77A17EE902AD4
S3150802CBB092B211461846FFF709FE0123BBE2204B43
S3150802CBC0D3ED017AB1EE047A77EEC77A97ED137A46
S3150802CBD0B4EEE77AF1EE10FA3EDD194BDB69184638
S3150802CBE0F3F7E6FD04460D46F86CF3F7E1FD024657
S3150802CBF00B4607F10C00CDE9002322462B461249C3
S3150802CC002BF0C0FD07F10C03184614F0B5FB28F00B
S3150802CC10AFFC0346184628F0C1FC03461521184600
S3150802CC2027F030F8012101200AF083FF044B4FF068
S3150802CC3000025A60024B4FF000029A6000237AE221
S3150802CC40F8D1002070D2050880D2050894D10020B8
S3150802CC50A4D2050895D10020B34B93ED017AB24BC5
S3150802CC60D3ED087A77EE677AF0EEE77AB3EE0E7AC4
S3150802CC70F4EEC77AF1EE10FA49DBAC4B1B78002BBF
S3150802CC8045D1AB4B1B785A1CD1B2A94A1170C72B96
S3150802CC903BD9A54BDB691846F3F78AFD04460D46D0
S3150802CCA0A14B1B6A1846F3F783FD02460B4607F1AA
S3150802CCB00C00CDE9002322462B469E492BF062FD45
S3150802CCC007F10C03184614F057FB994B00221A7009
S3150802CCD0964B01221A70944BD3ED007AFCEEE77A52
S3150802CCE0C7ED017A3B79DBB28F4A92ED017A8E4A19
S3150802CCF0D2ED087A77EE677AFCEEE77A17EE902A93
S3150802CD0092B211461846FFF761FD012313E2864BDC
S3150802CD10DB691846F3F74CFD04460D46824B1B6A3F
S3150802CD201846F3F745FD02460B4607F10C00CDE916
S3150802CD30002322462B4680492BF024FD07F10C03DB
S3150802CD40184614F019FB28F013FC0346184628F077
S3150802CD5025FC03461521184626F094FF01210120D9
S3150802CD600AF0E7FE704B4FF000025A606E4B4FF026
S3150802CD7000029A600023DEE16B4B93F82C30002BFD
S3150802CD804CD0694B93F82C30013BDAB2664B83F8E8
S3150802CD902C20654B93F82C30002B40F086810CF042
S3150802CDA025FE0346002118460EF0BAFE5E4B002207
S3150802CDB0DA605D4BDB691846F3F7FAFC04460D4662
S3150802CDC0594B1B6A1846F3F7F3FC02460B4607F162
S3150802CDD00C00CDE9002322462B4658492BF0D2FCFB
S3150802CDE007F10C03184614F0C7FA28F0C1FB0346EC
S3150802CDF0184628F0D3FB03461521184626F042FFAB
S3150802CE00012101200AF095FE474B4FF000025A60B5
S3150802CE10454B4FF000029A6000238CE1444B0022F6
S3150802CE201A700CF0E3FD034618460EF0A1FE0346FF
S3150802CE30002B11D10CF0DAFD0346012118460EF03B
S3150802CE406FFE28F095FB0346184628F0A7FB034613
S3150802CE501421184626F016FF334BD3ED047A97EDC4
S3150802CE60137A77EE677AC7ED127AD7ED127AB0EEB1
S3150802CE70007AF4EEC77AF1EE10FA61DB2A4BD3EDAB
S3150802CE80097A97ED137A77EE677AC7ED127AD7EDB4
S3150802CE90127AB7EE007AF4EEC77AF1EE10FA3ADBB6
S3150802CEA0214B9B6A07EE903AB8EE677AD7ED126A7B
S3150802CEB0C6EE877AC7ED127A1B4B9B6901331A4A6B
S3150802CEC09361194B9B69022B21D9174B93ED077A6C
S3150802CED0154B9B69033B07EE903AF8EE677A67EEC5
S3150802CEE0277A114BC3ED077A0F4B93ED077AD7EDE5
S3150802CEF0127A77EE276A0C4B9B69023B07EE903A49
S3150802CF00B8EE677AC6EE877A074BC3ED077A064B01
S3150802CF1001229A6204E0044B9B6A0133024A936235
S3150802CF20014AFB6C536210E0F8D1002095D100202B
S3150802CF3094D10020D0D20508F4D2050814D30508E6
S3150802CF40814B5B690133804A53617F4B9C697E4BF7
S3150802CF50DB691846F3F72CFC02460B4621467B484A
S3150802CF6014F0DEFA784B1A6B531C77490B63784B2D
S3150802CF70A3FB02135B094FF4967101FB03F3D31A61
S3150802CF80002B0ED1F86CF3F713FC02460B4607F199
S3150802CF900C0070492BF0F6FB07F10C03184614F047
S3150802CFA0EBF9694B5B69952B0AD9674BD3ED017A85
S3150802CFB0B2EE007A77EEC77A634BC3ED087A2BE0B6
S3150802CFC0614B5B69012B14D95F4B93ED017A5E4B7A
S3150802CFD0D3ED076A5C4B5B69023B07EE903AF8EEC3
S3150802CFE0677A66EEA77A77EE677A574BC3ED087AC1
S3150802CFF012E0554B93ED017A534BD3ED076A524B28
S3150802D0005B6907EE903AF8EE677A66EEA77A77EEEC
S3150802D010677A4D4BC3ED087A4B4B93ED087AD7EDF9
S3150802D020137A37EE677A484BD3ED077AF2EE046A3B
S3150802D03067EEA67AB4EEE77AF1EE10FA2BD5424BF2
S3150802D04093F82C30002B26D13F4B93ED087AD7ED77
S3150802D050137A37EE677A3C4BD3ED077AC7EE276A1F
S3150802D06016EE900AF3F7A4FB35A3D3E90023F3F7E8
S3150802D07021FD02460B4610461946F3F7C9FE03463A
S3150802D080DAB2314B83F82C202F4B93F82C30194601
S3150802D090314814F045FA2C4B1B6A1846F3F788FBFD
S3150802D0A002460B462D4814F03BFA274BD3ED027A7B
S3150802D0B0B0EE087A77EE877A97ED137AB4EEE77AC6
S3150802D0C0F1EE10FA05DB204AFB6C93601E4B002238
S3150802D0D0DA601D4BDB6801331B4AD3601A4BDB68E7
S3150802D0E040F2DB52934225D90CF080FC034600211C
S3150802D0F018460EF015FD002101200AF01AFD28F047
S3150802D10037FA0346184628F049FA03461421184600
S3150802D11026F0D3FD124814F02FF90B4B0022DA60E1
S3150802D120094B4FF000025A60074B4FF000029A6013
S3150802D130002300E0012318465037BD46BDE8B083F8
S3150802D1409A9999999999F93FF8D1002038D30508FF
S3150802D150B5814E1B50D3050864D3050874D3050858
S3150802D16084D30508B0B590B002AF03460A46FB71F0
S3150802D1701346BB80BB8807EE903AF8EE677AC7ED8E
S3150802D1800D7A4FF000033B63FB79002B00F0838096
S3150802D190FB79042B7FD8FB79012B10D10CF026FCE6
S3150802D1A0034618460FF0A8FA87ED0C0A97ED0D7A92
S3150802D1B0D7ED0C7A77EE277AC7ED0D7A3AE0FB7946
S3150802D1C0022B10D10CF012FC034618460FF0B4FAE3
S3150802D1D087ED0C0A97ED0D7AD7ED0C7A77EE277A5A
S3150802D1E0C7ED0D7A26E0FB79032B10D10CF0FEFB76
S3150802D1F0034618460FF0C0FA87ED0C0A97ED0D7A2A
S3150802D200D7ED0C7A77EE277AC7ED0D7A12E0FB791D
S3150802D210042B0FD10CF0EAFB034618460FF0CCFAA2
S3150802D22087ED0C0A97ED0D7AD7ED0C7A77EE277A09
S3150802D230C7ED0D7A1A4A7B6B5360FB7907EE903A73
S3150802D240F8EE677A164BC3ED007A154B4FF00002DB
S3150802D2509A60134B0022DA60114B00221A63386B6C
S3150802D260F3F7A6FA04460D460D4B5B681846F3F724
S3150802D2709FFA02460B4607F10800CDE9002322462B
S3150802D2802B4608492BF07EFA07F10803184614F0D4
S3150802D29073F8012300E0002318463837BD46B0BDAF
S3150802D2A02CD2002094D3050880B586B000AF034679
S3150802D2B03960FB71FB7903F12D0207F10C030D4965
S3150802D2C018462BF05FFA07F10C03184614F054F8C7
S3150802D2D0FB792D33DBB218460CF062F9FB79064A64
S3150802D2E0A2FB0323DB08DAB23B681A7000BF1837C1
S3150802D2F0BD4680BDACD30508CDCCCCCCB0B58CB080
S3150802D30002AF4FF000037B620CF070FB38629E4B53
S3150802D3101B78002B11D1386A0CF0F6FB0346184627
S3150802D3200CF0EDFD03461A46974B1A70964B1B787E
S3150802D330002B02D1944B14221A70944BD3ED007A27
S3150802D340B7EE007AF4EE477AF1EE10FA05D1386AAA
S3150802D3500FF0D2F987ED090A2EE08C4BD3ED007A4D
S3150802D360B0EE007AF4EE477AF1EE10FA05D1386A91
S3150802D3700FF0E2F987ED090A1EE0844BD3ED007A35
S3150802D380B0EE087AF4EE477AF1EE10FA05D1386A69
S3150802D3900FF0F2F987ED090A0EE07C4BD3ED007A1D
S3150802D3A0B1EE007AF4EE477AF1EE10FA04D1386A51
S3150802D3B00FF002FA87ED090A786AF3F7F9F90446D3
S3150802D3C00D46724B5B681846F3F7F2F902460B46AE
S3150802D3D0CDE9002322462B466D4814F0A1F86B4B83
S3150802D3E0D3ED017AB7EE007A77EEC77A97ED097A26
S3150802D3F0B4EEE77AF1EE10FA48DB664813F0BCFFA2
S3150802D4000CF016F90CF0F2FA0346002118460EF053
S3150802D410BCFB614B00221A70604B00221A7028F07E
S3150802D420A7F80346184628F0B9F803461521184600
S3150802D43026F028FC012102200AF07BFB386A0CF050
S3150802D44063FB034618460CF05AFD0346142B0BD908
S3150802D450386A0CF059FB02464B4B1B7819461046A4
S3150802D4600CF03CFDF6F7C0F9484B0022DA60474B50
S3150802D4704FF000025A60454B4FF000029A60642052
S3150802D48024F028FC0CF0EAF800230EE10CF0AEFAC0
S3150802D490034618460EF08AFB0346002B11D128F0E4
S3150802D4A067F80346184628F079F803461421184601
S3150802D4B026F0E8FB0CF09AFA0346012118460EF00C
S3150802D4C064FB324B93ED017AD7ED097A77EE677AE8
S3150802D4D0B1EE087AF4EEC77AF1EE10FA0FDD2F4BA9
S3150802D4E01B78002B72D12E4813F046FF0CF074F805
S3150802D4F0294B01221A70294B01221A7066E0274B22
S3150802D50000221A70214BDB683B2B0AD8224B1B7868
S3150802D510012B5BD81C4B1B781F491846FFF7C4FE24
S3150802D52054E01A4BDB683B2B14D9184BDB68772B74
S3150802D53010D8194B1B78022B48D8134B1B780A3381
S3150802D540DAB2114B1A70104B1B7813491846FFF7BB
S3150802D550ABFE3BE00D4BDB68772B23D90B4BDB6825
S3150802D560B32B1FD80C4B1B78032B2FD8064B1B78D3
S3150802D5700A33DAB2044B1A70034B1B78064918466B
S3150802D580FFF792FE22E000BFCBD200202CD2002069
S3150802D59070D20508B4D30508CCD20020CDD200201B
S3150802D5A0C0D30508434BDB68B32B0FD9424B1B7814
S3150802D5B0042B0BD8414B1B780A33DAB23F4B1A704D
S3150802D5C03E4B1B783C491846FFF76EFE394B196BE2
S3150802D5D04B1C384A13633A4BA3FB01231A09134619
S3150802D5E01B019B1A5B00CA1A002A0CD1786AF3F748
S3150802D5F0DFF802460B46384632492BF0C3F83B465B
S3150802D600184613F0B9FE2B4BD3ED027AB0EE087A20
S3150802D61077EE877A97ED097AB4EEE77AF1EE10FAA1
S3150802D62005DB244A7B6A9360224B0022DA60214B8F
S3150802D630DB6801331F4AD3601E4BDB68B3F5AF7F45
S3150802D64032D3214813F098FE0BF0F2FF0CF0CEF914
S3150802D6500346002118460EF098FA174B00221A7054
S3150802D6601A4B00221A70002102200AF062FA27F0E9
S3150802D6707FFF0346184627F091FF034615211846F1
S3150802D68026F01BFB0B4B0022DA600A4B4FF0000216
S3150802D6905A60084B4FF000029A60642024F01AFB85
S3150802D6A00BF0DCFF002300E0012318462837BD46AD
S3150802D6B0B0BD00BF2CD20020CCD20020CBD2002095
S3150802D6C089888888CCD30508E0D30508CDD20020FE
S3150802D6D0B0B590B002AF03460A46FB711346BB804B
S3150802D6E0BB8807EE903AF8EE677AC7ED0D7A4FF0E7
S3150802D6F000033B63FB79002B00F08380FB79042B44
S3150802D7007FD8FB79012B10D10CF070F90346184625
S3150802D7100EF0F2FF87ED0C0A97ED0D7AD7ED0C7A2B
S3150802D72077EE277AC7ED0D7A3AE0FB79022B10D10C
S3150802D7300CF05CF9034618460EF0FEFF87ED0C0A5C
S3150802D74097ED0D7AD7ED0C7A77EE277AC7ED0D7A33
S3150802D75026E0FB79032B10D10CF048F9034618464C
S3150802D7600FF00AF887ED0C0A97ED0D7AD7ED0C7AC9
S3150802D77077EE277AC7ED0D7A12E0FB79042B0FD1E3
S3150802D7800CF034F9034618460FF016F887ED0C0A22
S3150802D79097ED0D7AD7ED0C7A77EE277AC7ED0D7AE3
S3150802D7A01A4A7B6B5360FB7907EE903AF8EE677A72
S3150802D7B0164BC3ED007A154B4FF000029A60134BD5
S3150802D7C00022DA60114B00221A63386BF2F7F0FF77
S3150802D7D004460D460D4B5B681846F2F7E9FF02460A
S3150802D7E00B4607F10800CDE9002322462B460849D5
S3150802D7F02AF0C8FF07F10803184613F0BDFD0123F6
S3150802D80000E0002318463837BD46B0BD60D2002076
S3150802D810F0D3050880B586B000AF03463960FB71C0
S3150802D820FA7907F10C030C4918462AF0ABFF07F1FF
S3150802D8300C03184613F0A0FDFB7918460BF01CFFE3
S3150802D840FB79064AA2FB0323DB08DAB23B681A70A5
S3150802D85000BF1837BD4680BD08D40508CDCCCCCC50
S3150802D860B0B58CB002AF4FF000037B620CF0BEF885
S3150802D87038629E4B1B78002B11D1386A0CF044F99A
S3150802D880034618460CF059FB03461A46974B1A707C
S3150802D890964B1B78002B02D1944B14221A70944B88
S3150802D8A0D3ED007AB7EE007AF4EE477AF1EE10FA83
S3150802D8B005D1386A0EF020FF87ED090A2EE08C4B57
S3150802D8C0D3ED007AB0EE007AF4EE477AF1EE10FA6A
S3150802D8D005D1386A0EF030FF87ED090A1EE0844B3F
S3150802D8E0D3ED007AB0EE087AF4EE477AF1EE10FA42
S3150802D8F005D1386A0EF040FF87ED090A0EE07C4B27
S3150802D900D3ED007AB1EE007AF4EE477AF1EE10FA28
S3150802D91004D1386A0EF050FF87ED090A786AF2F7E1
S3150802D92047FF04460D46724B5B681846F2F740FFFE
S3150802D93002460B46CDE9002322462B466D4813F0D4
S3150802D940EFFD6B4BD3ED017AB7EE007A77EEC77A25
S3150802D95097ED097AB4EEE77AF1EE10FA48DB6648F3
S3150802D96013F00AFD0BF0D0FE0CF040F80346002136
S3150802D97018460EF028F9614B00221A70604B0022F5
S3150802D9801A7027F0F5FD0346184627F007FE0346E8
S3150802D9901521184626F076F9012103200AF0C9F85E
S3150802D9A0386A0CF0B1F8034618460CF0C6FA034674
S3150802D9B0142B0BD9386A0CF0A7F802464B4B1B7886
S3150802D9C0194610460CF0A8FAF5F70EFF484B002246
S3150802D9D0DA60474B4FF000025A60454B4FF000029F
S3150802D9E09A60642024F076F90BF0A4FE00230EE177
S3150802D9F00BF0FCFF034618460EF0F6F80346002B1A
S3150802DA0011D127F0B5FD0346184627F0C7FD034690
S3150802DA101421184626F036F90BF0E8FF03460121D1
S3150802DA2018460EF0D0F8324B93ED017AD7ED097A03
S3150802DA3077EE677AB1EE087AF4EEC77AF1EE10FA63
S3150802DA400FDD2F4B1B78002B72D12E4813F094FC56
S3150802DA500BF02EFE294B01221A70294B01221A704D
S3150802DA6066E0274B00221A70214BDB683B2B0AD84B
S3150802DA70224B1B78012B5BD81C4B1B781F49184677
S3150802DA80FFF7C8FE54E01A4BDB683B2B14D9184B38
S3150802DA90DB68772B10D8194B1B78022B48D8134B07
S3150802DAA01B780A33DAB2114B1A70104B1B781349DA
S3150802DAB01846FFF7AFFE3BE00D4BDB68772B23D901
S3150802DAC00B4BDB68B32B1FD80C4B1B78032B2FD8B9
S3150802DAD0064B1B780A33DAB2044B1A70034B1B78CF
S3150802DAE006491846FFF796FE22E000BFCED200206E
S3150802DAF060D2002070D2050810D40508CFD20020C3
S3150802DB00D0D200201CD40508434BDB68B32B0FD9AF
S3150802DB10424B1B78042B0BD8414B1B780A33DAB2DB
S3150802DB203F4B1A703E4B1B783C491846FFF772FE6C
S3150802DB30394B196B4B1C384A13633A4BA3FB012327
S3150802DB401A0913461B019B1A5B00CA1A002A0CD132
S3150802DB50786AF2F72DFE02460B46384632492AF013
S3150802DB6011FE3B46184613F007FC2B4BD3ED027AFF
S3150802DB70B0EE087A77EE877A97ED097AB4EEE77A05
S3150802DB80F1EE10FA05DB244A7B6A9360224B0022E7
S3150802DB90DA60214BDB6801331F4AD3601E4BDB6810
S3150802DBA0B3F5AF7F32D3214813F0E6FB0BF0ACFD99
S3150802DBB00BF01CFF0346002118460EF004F8174B1B
S3150802DBC000221A701A4B00221A700021032009F04B
S3150802DBD0B0FF27F0CDFC0346184627F0DFFC0346C4
S3150802DBE01621184626F069F80B4B0022DA600A4B12
S3150802DBF04FF000025A60084B4FF000029A60642008
S3150802DC0024F068F80BF096FD002300E0012318467D
S3150802DC102837BD46B0BD00BF60D20020CFD2002053
S3150802DC20CED200208988888828D405083CD40508DD
S3150802DC30D0D20020B0B590B002AF03460A46FB71B7
S3150802DC401346BB80BB8807EE903AF8EE677AC7EDB3
S3150802DC500D7A4FF000033B63FB79002B00F08380BB
S3150802DC60FB79042B7FD8FB79012B10D10BF0BEFE72
S3150802DC70034618460EF040FD87ED0C0A97ED0D7A1D
S3150802DC80D7ED0C7A77EE277AC7ED0D7A3AE0FB796B
S3150802DC90022B10D10BF0AAFE034618460EF04CFDD5
S3150802DCA087ED0C0A97ED0D7AD7ED0C7A77EE277A7F
S3150802DCB0C7ED0D7A26E0FB79032B10D10BF096FE01
S3150802DCC0034618460EF058FD87ED0C0A97ED0D7AB5
S3150802DCD0D7ED0C7A77EE277AC7ED0D7A12E0FB7943
S3150802DCE0042B0FD10BF082FE034618460EF064FD94
S3150802DCF087ED0C0A97ED0D7AD7ED0C7A77EE277A2F
S3150802DD00C7ED0D7A1A4A7B6B5360FB7907EE903A98
S3150802DD10F8EE677A164BC3ED007A154B4FF0000200
S3150802DD209A60134B0022DA60114B00221A63386B91
S3150802DD30F2F73EFD04460D460D4B5B681846F2F7B0
S3150802DD4037FD02460B4607F10800CDE900232246B5
S3150802DD502B4608492AF016FD07F10803184613F060
S3150802DD600BFB012300E0002318463837BD46B0BD39
S3150802DD7094D200204CD4050880B586B000AF03467D
S3150802DD803960FB71FA7907F10C030C4918462AF037
S3150802DD90F9FC07F10C03184613F0EEFAFB7918465C
S3150802DDA00BF0D6FCFB79064AA2FB0323DB08DAB2A0
S3150802DDB03B681A7000BF1837BD4680BD64D4050893
S3150802DDC0CDCCCCCCB0B58CB002AF4FF000037B62A1
S3150802DDD00BF00CFE38629E4B1B78002B11D1386A69
S3150802DDE00BF092FE034618460CF0C5F803461A468F
S3150802DDF0974B1A70964B1B78002B02D1944B142220
S3150802DE001A70944BD3ED007AB7EE007AF4EE477A9D
S3150802DE10F1EE10FA05D1386A0EF06EFC87ED090AA2
S3150802DE202EE08C4BD3ED007AB0EE007AF4EE477A08
S3150802DE30F1EE10FA05D1386A0EF07EFC87ED090A72
S3150802DE401EE0844BD3ED007AB0EE087AF4EE477AF8
S3150802DE50F1EE10FA05D1386A0EF08EFC87ED090A42
S3150802DE600EE07C4BD3ED007AB1EE007AF4EE477AF7
S3150802DE70F1EE10FA04D1386A0EF09EFC87ED090A13
S3150802DE80786AF2F795FC04460D46724B5B681846AB
S3150802DE90F2F78EFC02460B46CDE9002322462B46B4
S3150802DEA06D4813F03DFB6B4BD3ED017AB7EE007A62
S3150802DEB077EEC77A97ED097AB4EEE77AF1EE10FAB9
S3150802DEC048DB664813F058FA0BF08AFC0BF08EFD15
S3150802DED00346002118460DF094FE614B00221A7083
S3150802DEE0604B00221A7027F043FB0346184627F0B8
S3150802DEF055FB03461521184625F0C4FE01210520C7
S3150802DF0009F017FE386A0BF0FFFD034618460CF0B7
S3150802DF1032F80346142B0BD9386A0BF0F5FD024684
S3150802DF204B4B1B78194610460CF014F8F5F75CFCB7
S3150802DF30484B0022DA60474B4FF000025A60454BC5
S3150802DF404FF000029A60642023F0C4FE0BF05EFCD8
S3150802DF5000230EE10BF04AFD034618460DF062FE59
S3150802DF600346002B11D127F003FB0346184627F078
S3150802DF7015FB03461421184625F084FE0BF036FDE0
S3150802DF800346012118460DF03CFE324B93ED017A09
S3150802DF90D7ED097A77EE677AB1EE087AF4EEC77AA0
S3150802DFA0F1EE10FA0FDD2F4B1B78002B72D12E489B
S3150802DFB013F0E2F90BF0E8FB294B01221A70294B00
S3150802DFC001221A7066E0274B00221A70214BDB6881
S3150802DFD03B2B0AD8224B1B78012B5BD81C4B1B7890
S3150802DFE01F491846FFF7C8FE54E01A4BDB683B2B5D
S3150802DFF014D9184BDB68772B10D8194B1B78022BD0
S3150802E00048D8134B1B780A33DAB2114B1A70104BE5
S3150802E0101B7813491846FFF7AFFE3BE00D4BDB684A
S3150802E020772B23D90B4BDB68B32B1FD80C4B1B78EA
S3150802E030032B2FD8064B1B780A33DAB2044B1A7015
S3150802E040034B1B7806491846FFF796FE22E000BFE7
S3150802E050D1D2002094D2002070D205086CD40508CB
S3150802E060D2D20020D3D2002078D40508434BDB68ED
S3150802E070B32B0FD9424B1B78042B0BD8414B1B7879
S3150802E0800A33DAB23F4B1A703E4B1B783C491846A4
S3150802E090FFF772FE394B196B4B1C384A13633A4B1E
S3150802E0A0A3FB01231A0913461B019B1A5B00CA1A12
S3150802E0B0002A0CD1786AF2F77BFB02460B463846F1
S3150802E0C032492AF05FFB3B46184613F055F92B4BAB
S3150802E0D0D3ED027AB0EE087A77EE877A97ED097A67
S3150802E0E0B4EEE77AF1EE10FA05DB244A7B6A93600E
S3150802E0F0224B0022DA60214BDB6801331F4AD360C8
S3150802E1001E4BDB68B3F5AF7F32D3214813F034F9DF
S3150802E1100BF066FB0BF06AFC0346002118460DF06D
S3150802E12070FD174B00221A701A4B00221A70002132
S3150802E130052009F0FEFC27F01BFA0346184627F0CD
S3150802E1402DFA03461721184625F0B7FD0B4B002278
S3150802E150DA600A4B4FF000025A60084B4FF0000291
S3150802E1609A60642023F0B6FD0BF050FB002300E012
S3150802E170012318462837BD46B0BD00BF94D20020F9
S3150802E180D2D20020D1D200208988888884D4050872
S3150802E19098D40508D3D2002080B500AF0BF026FC30
S3150802E1A0034618460EF0F0FC0346002B33D00BF05C
S3150802E1B01DFC0346002118460EF05DFA0346B3F528
S3150802E1C0167F28D30BF012FC0346012118460EF0DF
S3150802E1D052FA0346B3F5167F1DD326F0CBFE034645
S3150802E1E001226221184626F003FF0346002B2CD192
S3150802E1F026F0C0FE034605226221184626F0F8FEDE
S3150802E2000346002B21D10BF0F1FB034606211846E3
S3150802E2100DF0F4FF19E026F0ADFE03460622622150
S3150802E220184626F0E5FE0346002B0FD00BF0DEFB60
S3150802E2300346002118460DF0E1FF26F09BFE002357
S3150802E2400622622126F073FF00E000BF00BF80BDF0
S3150802E25090B52DED028B8FB000AF0BF0C7FBB862FD
S3150802E260B34B1B78072B00F2598301A252F823F00D
S3150802E27091E2020865E302081BE402080FE50208B8
S3150802E2809DE50208E9E50208F7E802081DE9020821
S3150802E290B86A0DF0D7F80346002B41D1F5F7FAFA1A
S3150802E2A00346002B0AD0F5F7F5FA0346042B05D0E8
S3150802E2B0B86A0CF0B1FA0346012B31D127F058F9A6
S3150802E2C00346184627F06AF903460021184625F040
S3150802E2D0B1FDB86A0EF0E0FB0346002B16D0B86A09
S3150802E2E00DF052FD0346002B3AD00121B86A0DF013
S3150802E2F03FFB904B00221A608F4B00221A608F4810
S3150802E30013F03AF88A4B01221A7029E08A4B002246
S3150802E3101A608A4813F030F8854B01221A701FE0FA
S3150802E3200121B86A0EF0BBFC0346002B0DD0B86A71
S3150802E3300DF088F80346002B07D00121012009F0C9
S3150802E34086FE0121B86A0EF00FFDB86A0EF0A4FB2C
S3150802E3500346002B00F0E482794B00221A70DFE2B2
S3150802E36000BFDDE2B86A0DF06DF80346002B32D124
S3150802E370714B1B685A1C70490A60724A12689342AA
S3150802E380C0F0D08227F0F4F80346184627F006F9BB
S3150802E39003460221184625F04DFD0BF095FA664B09
S3150802E3A000221A60684B00221A600121B86A0EF030
S3150802E3B076FC0346002B07D0614B1B78022B03D849
S3150802E3C00121B86A0DF0ACFB604812F0D5FF584B34
S3150802E3D002221A70A6E227F0CBF80346184627F05F
S3150802E3E0DDF803460121184625F024FD584812F0A7
S3150802E3F0C3FF4F4B00221A700121B86A0EF04FFC78
S3150802E4000346002B00F08E820121B86A0EF0ACFC9E
S3150802E4100121012009F01BFE84E2B86A0DF012F808
S3150802E4200346002B2FD1444B1B685A1C42490A60EB
S3150802E430484A12689342C0F077820BF053FA46486C
S3150802E44012F09AFF454B47F230521A60B86A0EF03C
S3150802E45023FB0346002B0FD0394B1B78092B01D916
S3150802E4600BF064FA344B00221A603D4812F084FF1E
S3150802E4702F4B05221A7057E23A4812F07DFF2C4BB1
S3150802E48003221A7050E227F073F80346184627F05B
S3150802E49085F803460121184625F0CCFC264B0022B6
S3150802E4A01A60B86A0EF0F8FA0346002B0FD00BF082
S3150802E4B02FFA0BF010FA0BF040FA2B4812F05CFF19
S3150802E4C02A4812F059FF1A4B06221A700AE00BF074
S3150802E4D009FA214812F050FF254812F04DFF144B55
S3150802E4E004221A700121B86A0EF0D9FB0346002BE2
S3150802E4F000F01A820021B86A0DF012FB0121B86AEF
S3150802E5000EF032FC0121012009F0A1FD0CE2B86AE5
S3150802E5100CF098FF0346002B2CD0074B00221A60FA
S3150802E520134812F029FF024B04221A70FEE100BFBB
S3150802E53078D1002090D10020D4D20020A8D4050892
S3150802E540D8D200202C00002080210120B4D405084E
S3150802E550C0D4050830000020CCD4050834000020B9
S3150802E560DCD40508F0D4050800D5050814D5050835
S3150802E57028D505089F4B1B68643B9E4A13609D4B32
S3150802E5801B68002B40F0D2810BF0D0F9994B40F66C
S3150802E590B8321A60984812F0EFFEC7E1974B1B682B
S3150802E5A05A1C96490A60964A12689342C0F0C0817C
S3150802E5B0924B00221A600BF0ABF90BF08CF99148DA
S3150802E5C012F0DAFE904812F0D7FE26F0D1FF034683
S3150802E5D0184626F0E3FF03460121184625F02AFCD1
S3150802E5E08A4B00221A70A3E1B86A0CF02BFF034685
S3150802E5F0002B72D026F0BCFF0346184626F0CEFF43
S3150802E60003460121184625F015FC814B00221A7093
S3150802E6107A4B00221A600BF07BF90BF05CF90BF0CF
S3150802E6208CF97C4812F0A8FE7B4812F0A5FE01215F
S3150802E630B86A0EF034FB0346002B0BD00021B86AE9
S3150802E6400DF06EFA0121B86A0EF08EFB0121012047
S3150802E65009F0FDFC6D4B06221A70B86A0EF058FADC
S3150802E6600346002B28D04FF000037B636B4B1B68D5
S3150802E670022B13D9694B1B68023B07EE903AB8EE98
S3150802E680678AB86A0BF040FA034618460BF090FC04
S3150802E690B0EE407AC8EE077AC7ED0D7AD7ED0D7A55
S3150802E6A0B2EE047A67EE877AFCEEE77A17EE903ACC
S3150802E6B09BB2184609F0FCFA584B1C680221B86A44
S3150802E6C00DF0D9FF03463846224655492AF05AF82C
S3150802E6D03B46184612F050FE2CE1484B1B685A1C62
S3150802E6E046490A604F4A12689342C0F02381434B57
S3150802E6F000221A60464B1B780133DAB2444B1A7071
S3150802E700434B1B78142B40F29180414B00221A701E
S3150802E7100BF013F90BF0FCF80BF0DDF80121B86ADF
S3150802E7200CF0A5F826F024FF0346184626F036FF15
S3150802E73003460021184625F07DFB2E4B47F2305240
S3150802E7401A600521B86A0DF059FD374812F014FE11
S3150802E7502E4B07221A700121B86A0EF0A0FA034658
S3150802E760002B07D00121B86A0EF0FEFA0121022019
S3150802E77009F06DFCB86A0EF0CBF90346002B28D0D7
S3150802E7804FF000033B63254B1B68022B13D9234B1F
S3150802E7901B68023B07EE903AB8EE678AB86A0BF036
S3150802E7A0B3F9034618460BF003FCB0EE407AC8EEFE
S3150802E7B0077AC7ED0C7AD7ED0C7AB2EE047A67EED1
S3150802E7C0877AFCEEE77A17EE903A9BB2184609F07A
S3150802E7D06FFA124B1C680221B86A0DF04CFF034609
S3150802E7E0384622460E4929F0CDFF3B46184612F016
S3150802E7F0C3FD9FE0340000203CD50508D4D2002092
S3150802E8003800002050D50508C0D4050878D1002064
S3150802E810D8D2002064D5050814D505088021012020
S3150802E82078D505083C0000208CD5050826F0A0FE00
S3150802E8300346184626F0B2FE03460021184625F07E
S3150802E840F9FA0BF065F80BF046F80BF076F83E4845
S3150802E85012F092FD3D4812F08FFD3D4B06221A70CA
S3150802E8600121B86A0EF01BFA0346002B03D00021D9
S3150802E870B86A0DF055F9B86A0EF04AF90346002B44
S3150802E88028D04FF00003FB62324B1B68022B13D9C8
S3150802E890304B1B68023B07EE903AB8EE678AB86AB5
S3150802E8A00BF032F9034618460BF082FBB0EE407ABB
S3150802E8B0C8EE077AC7ED0B7AD7ED0B7AB2EE047A71
S3150802E8C067EE877AFCEEE77A17EE903A9BB218461D
S3150802E8D009F0EEF91F4B1C680221B86A0DF0CBFE4F
S3150802E8E00346384622461C4929F04CFF3B46184641
S3150802E8F012F042FD1EE0194B1B685A1C17490A60A2
S3150802E900174A1268934217D3144B00221A60154805
S3150802E91012F032FD0E4B00221A700DE000BF0CE019
S3150802E92000BF0AE000BF08E000BF06E000BF04E03F
S3150802E93000BF02E000BF00E000BF00BF3C37BD4693
S3150802E940BDEC028B90BD00BF00D5050814D505089D
S3150802E95078D100208021012078D50508D4D200205C
S3150802E96040000020C0D4050890B52DED028B97B063
S3150802E97000AF0BF03BF878650023A7F85230934BAB
S3150802E9801B78072B00F2C18401A252F823F000BFBC
S3150802E990B1E90208C5EA020809EC020805F102080B
S3150802E9A063F10208BBF102083DF20208E3F102082C
S3150802E9B0786D0CF0F7FE0346002B45D1FBF728FBD2
S3150802E9C00346012B0AD0FBF723FB0346062B05D089
S3150802E9D0786D0BF0EFFF0346002B35D1786D0CF0FE
S3150802E9E06DFD0346002B1BD1786D0EF0CDF803465C
S3150802E9F0002B29D00021786D0DF03DFE0446786D76
S3150802EA000EF0E0F803469C421ED30121786D0DF004
S3150802EA1032FE0446786D0EF0F3F803469C4213D391
S3150802EA206B4B00221A700121786D0CF0A1FF694B1D
S3150802EA3000221A60684B4FF4FA621A60674812F0AD
S3150802EA409BFC624B01221A70FBF7E2FA0346012B82
S3150802EA500BD0FBF7DDFA0346062B06D0786D0BF0D2
S3150802EA60A9FF0346002B40F052840021786D0DF071
S3150802EA7002FE0346B3F5167F1ED9564B1B685A1C6F
S3150802EA8054490A6042F22732934240F24084514B7B
S3150802EA9000221A60786D0CF093FF0346002B05D00E
S3150802EAA00021786D0CF064FF00F031BC0121786D0D
S3150802EAB00CF05EFF00F02BBC0121786D0CF058FFBC
S3150802EAC000F025BC444B1B68643B434A1360FBF7C2
S3150802EAD09FFA0346012B0AD0FBF79AFA0346062B3E
S3150802EAE005D0786D0BF066FF0346002B5FD1786D73
S3150802EAF00CF058FE0346002B13D0786D0CF0DAFDA5
S3150802EB000346002B0DD00021786D0CF03FFD3448EA
S3150802EB1012F032FC334812F02FFC2C4B00221A70EA
S3150802EB2007E00121786D0CF031FD0121786D0CF0BA
S3150802EB30C1FF294B1B68002B47D10121786D0CF0C8
S3150802EB4005FE294B00221A60284B00221A60284B20
S3150802EB5000221A60786D0EF017F80346002B1FD0B4
S3150802EB600021786D0DF087FD0446786D0EF02AF8BF
S3150802EB7003469C4214D30121786D0DF07CFD0446B0
S3150802EB80786D0EF03DF803469C4209D3194812F0F7
S3150802EB90F3FB194B194A1A600C4B06221A7014E039
S3150802EBA0174812F0E9FB094B02221A700DE0002100
S3150802EBB0786D0CF0EBFC134812F0DEFB094812F0F4
S3150802EBC0DBFB024B00221A70ACE3ABE379D10020DF
S3150802EBD096D1002090D1002044000020A0D5050837
S3150802EBE0ACD50508C4D505087CD1002080D1002003
S3150802EBF084D10020D0D505082400002040771B00C8
S3150802EC00E4D50508F4D505080121786D0EF0EDF86E
S3150802EC10BC4B1B68002B6BD0786D0DF06BFB034663
S3150802EC20002B04DCB84B1B686433B74A1360B64B37
S3150802EC301B68B64A93425BD30021786D0DF01BFD23
S3150802EC400346A7F850300121786D0DF014FD0346EE
S3150802EC50A7F84E30B7F85030B3F52F6F48D2786D13
S3150802EC600AF052FF0246B7F85030194610460AF023
S3150802EC70DFFFB7F84E30B3F52F6F0AD2786D0AF078
S3150802EC8043FF0246B7F84E30194610460AF0ECFF23
S3150802EC9008E0786D0AF038FF03464FF42F611846EC
S3150802ECA00AF0E2FF786D0AF02FFF034618460AF0CB
S3150802ECB0CFFF03461C46786D0AF026FF0346184620
S3150802ECC00AF0E2FF0346381D2246914929F05AFD09
S3150802ECD03B1D184612F050FB8A4B00221A600AF0B6
S3150802ECE085FE0346002118460DF0C7FDF4F77CFDA4
S3150802ECF00121786D0DF0BFFC0346B3F5167F14D9D2
S3150802ED00844B1B68002B0CD0834B1A68814B1B68FB
S3150802ED10D31A43F69722934207D9804B01221A60E7
S3150802ED2003E07D4B1B687B4A1360786D0DF0E2FAAF
S3150802ED300346B3F1FF3F04DB784B1B68002B00F058
S3150802ED40A680704B1B68002B5ED06F4B00221A60A0
S3150802ED500021786D0DF08FFC0346A7F84830012193
S3150802ED60786D0DF088FC0346A7F84630B7F84830A8
S3150802ED70B3F52F6F48D2786D0AF0C6FE0246B7F889
S3150802ED804830194610460AF053FFB7F84630B3F52D
S3150802ED902F6F0AD2786D0AF0B7FE0246B7F84630E8
S3150802EDA0194610460AF060FF08E0786D0AF0ACFED4
S3150802EDB003464FF42F6118460AF056FF786D0AF09B
S3150802EDC0A3FE034618460AF043FF03461C46786D1F
S3150802EDD00AF09AFE034618460AF056FF0346381DFD
S3150802EDE022464F4929F0CEFC3B1D184612F0C4FABA
S3150802EDF0444B00221A600AF0F9FD03460021184620
S3150802EE000DF03BFDF4F7F0FC464B474A1A60786D65
S3150802EE100CF090FB0346002B13D0786D0BF0CAFD5D
S3150802EE200346002B0DD0FBF7F3F80346012B04D05B
S3150802EE30FBF7EEF80346062B03D13C4B01221A7068
S3150802EE40EBE03B4812F098FA3A4B00221A7000217E
S3150802EE50786D0CF09BFB786D0AF056FE0346184651
S3150802EE600AF088FF03461A462B4B1B689A4280F023
S3150802EE70D480786D0AF048FE0246274B1B689BB27F
S3150802EE80194610460AF066FFF4F7AEFCC5E0786D3F
S3150802EE900CF0F6FA0346002B00F0C080194B1B68EB
S3150802EEA0002B78D0184B00221A600021786D0DF0DD
S3150802EEB0E2FB0346A7F84C300121786D0DF0DBFB27
S3150802EEC00346A7F84A30B7F84C30B3F52F6F62D22B
S3150802EED0786D0AF019FE0246B7F84C301946104604
S3150802EEE00AF0A6FEB7F84A30B3F52F6F24D2786D2A
S3150802EEF00AF00AFE0246B7F84A30194610460AF0E0
S3150802EF00B3FE22E0DCD20020E0D20020003E490017
S3150802EF100CD6050884D100207CD1002080D100209F
S3150802EF202CD605082400002000BADB0096D1002062
S3150802EF30C4D5050879D10020786D0AF0E5FD0346A7
S3150802EF404FF42F6118460AF08FFE786D0AF0DCFD41
S3150802EF50034618460AF07CFE03461C46786D0AF0FC
S3150802EF60D3FD034618460AF08FFE0346381D22468D
S3150802EF70A64929F007FC3B1D184612F0FDF9A44BD9
S3150802EF8000221A600AF032FD0346002118460DF0E7
S3150802EF9074FCF4F729FC9F4B9F4A1A60786D0CF0B3
S3150802EFA0C9FA0346002B13D0786D0BF003FD03460E
S3150802EFB0002B0DD0FBF72CF80346012B04D0FBF7E8
S3150802EFC027F80346062B03D1944B01221A7025E033
S3150802EFD0934812F0D1F9934B00221A700021786DEA
S3150802EFE00CF0D4FA786D0AF08FFD034618460AF03B
S3150802EFF0C1FE03461A468C4B1B689A420ED2786D9E
S3150802F0000AF082FD0246884B1B689BB219461046D7
S3150802F0100AF0A0FEF4F7E8FB00E000BF786D0DF0F9
S3150802F0205BFF0346012B06D1786D0DF095FF03466B
S3150802F030A7F8523003E040F62823A7F85230786D35
S3150802F0400CF078FA0346002B12D0786D0BF0B2FC5E
S3150802F0500346002B0CD0FAF7DBFF0346012B04D03C
S3150802F060FAF7D6FF0346062B02D16C4B01221A7019
S3150802F070786D0CF097FB0346002B1AD0786D0CF0CE
S3150802F08019FB0346002B14D00021786D0CF07EFA8A
S3150802F0905F4B1B68002B02D0644B00221A60644B3C
S3150802F0A04FF4FA621A60634812F066F95D4B07225A
S3150802F0B01A70786D0AF028FD034618460AF01FFEF4
S3150802F0C0B0EE408A786D0DF033F9F0EE407AB4EE80
S3150802F0D0E78AF1EE10FA0FDD786D0AF015FD04469F
S3150802F0E0786D0DF025F9F0EE407AB0EE670A204603
S3150802F0F00AF0F5FDF4F778FB4B4B1B6801334A4AD5
S3150802F10013600FE14C4B1B68643B4B4A1360786DE6
S3150802F1100DF0E2FE0346012B06D1786D0DF01CFFB9
S3150802F1200346A7F8523003E04FF41663A7F85230A5
S3150802F130414B1B68002B06D0786D0CF0A1F90346EB
S3150802F140002B00F0E6800021786D0CF01FFA314B97
S3150802F150314A1A60324812F00FF9324B00221A70FD
S3150802F160D7E02C4B1B68643B2A4A1360786D0DF076
S3150802F170B3FE0346012B06D1786D0DF0EDFE03466C
S3150802F180A7F8523003E04FF41663A7F85230214B22
S3150802F1901B68002B07D0786D0DF0ACF8034613F107
S3150802F1A0020F80F2B8801B4B1B4A1A601C4812F0E9
S3150802F1B0E3F81C4B00221A70ADE01D4B1B68643B3A
S3150802F1C01B4A13601A4B1B68002B40F0A680134B90
S3150802F1D000221A70124812F0CFF8124B00221A7047
S3150802F1E09BE0134B1B68643B114A1360104B1B6868
S3150802F1F0002B40F09480094B00221A70084812F03E
S3150802F200BBF8084B00221A7089E000BF2CD6050805
S3150802F210DCD200202400002000BADB0096D10020B0
S3150802F220C4D5050879D100207CD10020E0D200207F
S3150802F2304400002048D60508480000200221786DBF
S3150802F2400DF0D3FD786D0DF055F80346002B2DDC35
S3150802F250374B1B68643B364A1360354B1B68002BD9
S3150802F26027D1786D0CF066F90346002B13D0786D1A
S3150802F2700BF0A0FB0346002B0DD0FAF7C9FE034696
S3150802F280012B04D0FAF7C4FE0346062B03D1294BF9
S3150802F29001221A700DE0284812F06EF8274B002258
S3150802F2A01A700021786D0CF071F902E0204B244A9D
S3150802F2B01A60786D0DF010FE0346012B06D1786DA3
S3150802F2C00DF04AFE0346A7F8523003E040F628231B
S3150802F2D0A7F85230786D0CF065FA0346002B20D059
S3150802F2E0786D0CF0E7F90346002B1AD00021786DE9
S3150802F2F00CF04CF9134B4FF4FA621A60124812F0EA
S3150802F3003BF80E4B07221A700BE000BF0AE000BF5B
S3150802F31008E000BF06E000BF04E000BF02E000BF4D
S3150802F32000E000BF00BF5C37BD46BDEC028B90BD56
S3150802F3302400002096D10020C4D5050879D10020E2
S3150802F34040771B00440000205CD6050880B500AF54
S3150802F350FCF778FD0346002B38D01D4B1B78002B93
S3150802F36034D01C4B1B685A1C1A490A60092B2DD922
S3150802F3700220FCF773FD0346002B10D0FDF71AF89E
S3150802F3800346002B0BD10220FCF794FD124811F01C
S3150802F390F3FF104B00221A600D4B00221A7004204C
S3150802F3A0FCF75CFD0346002B10D0FDF797F80346E1
S3150802F3B0002B0BD10420FCF77DFD084811F0DCFF79
S3150802F3C0044B00221A60024B00221A7000BF80BD4D
S3150802F3D08CD10020E4D2002078D6050888D6050804
S3150802F3E080B58CB000AF002387F82F303F4BD3F897
S3150802F3F0F430002B08DA062387F82F303B1D3C49E8
S3150802F400184629F0BFF954E0384BD3F8F43003F024
S3150802F4108043002B08D0052387F82F303B1D35493A
S3150802F420184629F0AFF944E0304BD3F8F43003F02C
S3150802F4300053002B08D0042387F82F303B1D2E4992
S3150802F440184629F09FF934E0284BD3F8F43003F034
S3150802F4508053002B08D0032387F82F303B1D2749FA
S3150802F460184629F08FF924E0204BD3F8F43003F03C
S3150802F4700063002B0ED0022387F82F303B1D20494C
S3150802F480184629F07FF91F4B01221A701E4B0122DA
S3150802F4901A700EE0154BD3F8F43003F08063002B94
S3150802F4A007D0012387F82F303B1D1849184629F043
S3150802F4B069F93B1D1846F1F70FF803469AB23B1D48
S3150802F4C01946012012F0BAFA3B1D184611F054FFEC
S3150802F4D0064BD3F8F430054A43F40003C2F8F43075
S3150802F4E097F82F3018463037BD4680BD000C0244C7
S3150802F4F098D60508B0D60508CCD60508F0D605086C
S3150802F50008D70508DCD30020DDD3002020D705085C
S3150802F51090B583B000AF786078680BF028F8044697
S3150802F52078680BF057F803469C4208DA0121786896
S3150802F5300BF03AF8002178680BF076F81AE078684A
S3150802F5400CF004FC0346002B14D178680BF05FF824
S3150802F5500346002B0AD1094811F0E2FF0121786817
S3150802F5600BF080F8012178680BF0A0F90121786880
S3150802F5700BF05AF800BF0C37BD4690BD34D70508C4
S3150802F58098B500AF0AF032FA034618460CF0D0F8DE
S3150802F5900346002B06D14B4B00221A704A4B002217
S3150802F5A01A604EE00AF022FA034618460CF04CF8A6
S3150802F5B00346002B42D1444B1C68631C424A136023
S3150802F5C00AF014FA034618460BF07FFD03469C42DE
S3150802F5D034D30AF00BFA0346002118460CF078F8E1
S3150802F5E00AF004FA0346002118460CF02DFA0AF02E
S3150802F5F0FDF9034618460BF0F1FF0346002B0FD11F
S3150802F6000AF0F4F9034618460CF054F80346002BA0
S3150802F61006D10AF0EBF90346002118460CF04AFA1D
S3150802F62025F0A6FF0346184625F0C3FF0346002128
S3150802F630184624F075FB244B00221A60214B00223F
S3150802F6401A700AF0D3F9034618460CF0ABF80346CB
S3150802F650002B03D11D4B00221A6030E00AF0C6F9CE
S3150802F660034618460BF0BAFF0346002B27D10AF0C9
S3150802F670BDF9034618460CF01DF80346002B1ED1A9
S3150802F680124B1C68631C114A13600AF0AFF9034651
S3150802F69018460BF01AFD03469C4210D30AF0A6F947
S3150802F6A00346002118460CF051F80AF09FF9034662
S3150802F6B0002118460CF0FEF9044B00221A6000BF1E
S3150802F6C098BD00BF4C000020E0D30020E4D3002000
S3150802F6D080B500AF0AF08AF9034618460CF09CF882
S3150802F6E00346002B02D008F023FF01E008F03AFF98
S3150802F6F00AF07CF9034618460CF01AF80346002B62
S3150802F70008D008F08BFF364B1B78002B04D109F082
S3150802F710D9FE01E008F09CFF0AF068F9034618468C
S3150802F7200BF05CFF0346002B02D009F08FFE01E0C6
S3150802F73009F0A6FE0AF05AF9034618460BF084FFAA
S3150802F7400346002B02D009F0E5FD01E009F0FCFDB5
S3150802F7500AF04CF9034618460CF068F90346002BE2
S3150802F76002D008F0A9FE01E008F0C0FE0AF03EF950
S3150802F770034618460CF0C6F90346002B02D009F0D8
S3150802F780D1FE01E009F0E8FE0AF030F90346184610
S3150802F7900CF0E0F80346002B02D008F005FF01E062
S3150802F7A008F01CFF0AF022F9034618460BF0FAFF86
S3150802F7B00346002B02D008F06BFF01E008F082FF37
S3150802F7C00AF014F9034618460BF074FF0346002B99
S3150802F7D002D009F0DBFD01E009F0F2FD00BF80BDB1
S3150802F7E0CCD3002080B582B000AF0AF0FFF80346FA
S3150802F7F018460DF053F80346FB710AF0F7F803466C
S3150802F80018460CF070FC0346002B08D10AF0EEF8F5
S3150802F810034618460CF0E5FC0346002B02D008F016
S3150802F820B7FC9BE0FB79012B02D0022B2BD063E0BD
S3150802F8304C4B1B78012B02D108F092FC87E0494B0E
S3150802F8401B78022B02D108F097FC80E0454B1B7807
S3150802F850032B02D108F084FC79E0424B1B78042B77
S3150802F86002D108F089FC72E03E4B1B78042B06D9BC
S3150802F8703C4B1B780D2B02D808F07EFC67E0394B0F
S3150802F88000221A7063E0374B1B78012B02D108F06D
S3150802F89067FC5CE0334B1B78022B02D108F06CFC48
S3150802F8A055E0304B1B78032B02D108F059FC4EE089
S3150802F8B02C4B1B78042B02D108F05EFC47E0294B3F
S3150802F8C01B78052B02D108F04BFC40E0254B1B7830
S3150802F8D0062B02D108F050FC39E0224B1B78062B86
S3150802F8E006D9204B1B780D2B02D808F045FC2EE0D2
S3150802F8F01C4B00221A702AE01A4B1B78012B02D1E4
S3150802F90008F02EFC22E0174B1B78022B02D108F0D6
S3150802F91027FC1BE0134B1B78032B02D108F020FCB3
S3150802F92014E0104B1B78042B02D108F019FC0DE0E9
S3150802F9300C4B1B78042B06D90A4B1B78072B02D8CB
S3150802F94008F01AFC02E0074B00221A7000BF054BAA
S3150802F9501B780133DAB2034B1A7000BF00BF0837AF
S3150802F960BD4680BDE8D3002080B500AF0C22002139
S3150802F970024828F09BFF00BF80BD00BFD0D30020FD
S3150802F980B0B5A2B000AF25F0F5FA0346184625F041
S3150802F99007FB0346002B36D03B1D0121184623F0F0
S3150802F9A0F3FF3B1D0121184624F009F825F0E2FA77
S3150802F9B00346184625F04EFB02463B1D11461846DD
S3150802F9C024F01DF807F144023B1D1146184624F09F
S3150802F9D059F823F0C4FF044607F14403184624F0F5
S3150802F9E01EF8054607F14403184624F024F8034690
S3150802F9F01A462946204626F055FB25F0BBFA034649
S3150802FA00184625F0E7FA0A4B1B685A1C08490A6089
S3150802FA10632B08D925F0AEFA0346184625F0CCFA28
S3150802FA20034B00221A6000BF8837BD46B0BD00BF2F
S3150802FA30ECD3002090B585B000AF0023FB81604867
S3150802FA4002F03CFA034683F00103DBB2002B00F016
S3150802FA50B4803B461846FCF7E5F90346FB81FB8969
S3150802FA60002B00F0A9803B78012B40F0A680FB789A
S3150802FA70012B1BD1BB68002B13D0524B00221A70E4
S3150802FA80BB78BA6892B211461846FCF79FFE03463F
S3150802FA90002B40F089800C2200214B4828F006FFF3
S3150802FAA082E07B681846FCF799FB7DE0FB78022B1F
S3150802FAB017D1BB68002B0FD0BB78BA6892B2114631
S3150802FAC01846FDF74FFB0346002B6DD10C22002189
S3150802FAD03D4828F0EBFE67E07B681846FCF7D6FB44
S3150802FAE062E0FB78032B1AD1BB68002B0FD0BB78D8
S3150802FAF0BA6892B211461846FDF7EAFD0346002B8C
S3150802FB0009D10C220021304828F0D0FE03E07B6898
S3150802FB101846FCF781FC0420FCF7B8F944E0FB78A8
S3150802FB20052B1AD1BB68002B0FD0BB78BA6892B2E4
S3150802FB3011461846FEF77EF80346002B09D10C2219
S3150802FB400021214828F0B2FE03E07B681846FCF73C
S3150802FB5029FD0820FCF79AF926E0FB78042B08D140
S3150802FB607B681846FCF792FB7B681846FCF754FC40
S3150802FB701AE0FB78662B04D17B681846FCF786FBED
S3150802FB8012E0FB78672B04D17B681846FCF744FC25
S3150802FB900AE0FB78682B07D17B681846FCF776FBE8
S3150802FBA07B681846FCF738FC074B1C463B4693E82D
S3150802FBB0070084E8070000E000BF1437BD4690BD81
S3150802FBC098D1002095D10020D0D3002080B500AF6F
S3150802FBD00F4BDB78012B18D10D4B9B68002B0AD0F3
S3150802FBE0FCF7DAFE0346002B0FD10C220021084847
S3150802FBF028F05CFE09E0FCF701FB0346002B04D162
S3150802FC000C220021024828F051FE00BF80BD00BF29
S3150802FC10D0D3002080B500AF594BDB78022B24D114
S3150802FC200220FCF747F9564B9B68002B0ED0FDF7CE
S3150802FC3065FB0346002B40F0A1800C2200215048A8
S3150802FC4028F034FE0220FCF721F997E0FCF72EFB98
S3150802FC500346002B40F092800C220021484828F0E7
S3150802FC6025FE0220FCF712F988E0454BDB78032BC8
S3150802FC7022D10420FCF71EF9414B9B68002B0DD0BC
S3150802FC80FDF7EEFD0346002B78D10C2200213C48F5
S3150802FC9028F00CFE0420FCF7F9F86FE0FCF7CCFB21
S3150802FCA00346002B6AD10C220021354828F0FEFDB6
S3150802FCB00420FCF7EBF861E0314BDB78052B22D107
S3150802FCC00820FCF7F7F82E4B9B68002B0DD0FEF7A1
S3150802FCD079F80346002B51D10C220021284828F036
S3150802FCE0E5FD0820FCF7D2F848E0FCF76BFC034672
S3150802FCF0002B43D10C220021214828F0D7FD0820E9
S3150802FD00FCF7C4F83AE01E4BDB78042B0AD1FCF761
S3150802FD10F1FC0346002B31D10C220021184828F0A9
S3150802FD20C5FD2BE0164BDB78662B0AD1FCF710FBD8
S3150802FD300346002B22D10C220021114828F0B6FDD9
S3150802FD401CE00F4BDB78672B0AD1FCF7F9FB03465D
S3150802FD50002B13D10C220021094828F0A7FD0DE03B
S3150802FD60074BDB78682B09D1FCF77EFC0346002B90
S3150802FD7004D10C220021024828F098FD00BF80BD5C
S3150802FD80D0D3002080B58EB008AF786000237B619F
S3150802FD907B683B6107F10C0100234FF480523869F6
S3150802FDA022F02EFD0346002B01D0022353E0FB6806
S3150802FDB0B022069201220592002204920A22039296
S3150802FDC00A2202924FF48052019200930023244A97
S3150802FDD02449254822F05AFF0346002B01D00E2358
S3150802FDE039E0342300222149214822F01DFE034628
S3150802FDF0002B01D01C232EE01421002000F036FC33
S3150802FE00FBF7EEFF7868F3F765FE7868FBF714FDF3
S3150802FE10786800F069FC78680EF044FE786801F0AC
S3150802FE20FDFE786806F09CFF342300221149124829
S3150802FE3022F0FAFD0346002B01D01C230BE03423E3
S3150802FE4000220E490E4822F0EFFD0346002B01D090
S3150802FE501C2300E07B6918461837BD4680BD00BFE3
S3150802FE6085FE02084CD70508E8D200205CD70508AB
S3150802FE7098D300206CD705089C2101207CD7050859
S3150802FE80A8D400202DE9F043D5B006AF07F59C7338
S3150802FE90A3F59A73186000F0B7FC002387F8373188
S3150802FEA00023A7F83431002387F833310023A7F853
S3150802FEB03031002387F82F31002387F82E310023AB
S3150802FEC0C7F82831002387F827310023C7F82031DD
S3150802FED0002387F81F310023C7F81831002387F853
S3150802FEE017310023C7F81031002387F80F3107F1BD
S3150802FEF0700380220021184628F0D8FCFFF770FA12
S3150802FF0007F10C03C94ACA49184628F03BFCC948F6
S3150802FF1011F032FA07F10C03184611F02DFA09F01E
S3150802FF2065FDC7F80801D7F8080109F0EDFD034693
S3150802FF30184609F03CFF0346012B04D10121D7F8E4
S3150802FF4008010CF0F2FDD7F8080109F0DDFD0346B9
S3150802FF50184609F02CFF03461A4607F10C03B64960
S3150802FF60184628F00FFC07F10C03184611F004FA9C
S3150802FF700EF046FD0121D7F808010BF0F9FCD7F877
S3150802FF8008010CF055FB0446D7F808010CF066FB8D
S3150802FF90034606221946204612F0E4F9FFF716FE32
S3150802FFA097F83731092B0DD90123A7F834310023E5
S3150802FFB087F83731D7F808010CF03AFB034618469A
S3150802FFC012F0FAFAB7F83431002B00F00681002352
S3150802FFD0A7F8343111F012FA0EF0A6FCFFF7B6F9BB
S3150802FFE0F9F78EFFF7F702FDFFF7CAFCFFF722FDC6
S3150802FFF0FFF710FED7F808010AF04AFC0346002B61
S3150803000064D0FBF7A5FFD7F808010AF0E7FB034618
S31508030010002B09D1D7F808010AF01CFC0346002B6C
S3150803002002D1FEF715F910E0D7F808010AF012FC19
S315080300300346002B09D00121D7F808010CF02FFE3F
S315080300400346002B01D0FEF703F90221D7F808016E
S315080300500CF025FE0346002B35D0FBF7D7FD0346E8
S31508030060022B09D0FBF7D2FD0346032B04D0FBF77B
S31508030070CDFD0346062B08D10021D7F808010BF05E
S3150803008085FA0020FBF7B0FD02E00020FBF7ACFD84
S315080300900321D7F808010CF0A8FED7F808010CF0DD
S315080300A029F90346052B2CDD0021D7F808010CF0A6
S315080300B09CFE0221D7F808010CF056FE0221012006
S315080300C007F0C5FF1DE0FEF74FFC1AE0FBF79EFDA0
S315080300D00346022B09D0FBF799FD0346032B04D0ED
S315080300E0FBF794FD0346062B08D10021D7F8080130
S315080300F00BF04CFA0020FBF777FD02E00020FBF734
S3150803010073FDFAF7B9FEFAF7A7FFD7F808010AF05D
S3150803011051FC0346002B0AD0484B1B78002B06D00C
S31508030120FAF73CFFFAF7D8FFFBF70EFB55E0F9F7AA
S315080301306FFF0346032B10D1404B1B78002B21D0AE
S315080301400021D7F808010BF08DFA3D4B4AF6C87221
S315080301501A603A4B00221A7014E0F9F759FF03465E
S31508030160052B04D0F9F754FF0346062B0AD1334B64
S315080301701B78002B06D0324B4FF4FA721A602F4BBA
S3150803018000221A700121D7F808010CF089FF2C4BBD
S315080301901B68002B11D02A4B1B68642B0DD8002132
S315080301A0D7F808010BF0AAFB0021D7F808010BF0D2
S315080301B047FD234B00221A600FE0214B1B68642B73
S315080301C005D91F4B1B68643B1D4A136005E00020D5
S315080301D0F9F70CFF194B01221A7097F83331312BB3
S315080301E005D90123A7F83031002387F83331B7F847
S315080301F03031002B41D0FBF709FD0346022B0ED005
S31508030200FBF704FD0346032B09D0FBF7FFFC034664
S31508030210042B04D0FBF7FAFC0346062B12D1022162
S31508030220D7F808010CF047FB1CE000BF88D7050880
S3150803023090D70508B0D70508C0D705084D00002094
S31508030240F0D30020F3F77AFB0346052B05D10121EA
S31508030250D7F808010CF02FFB04E00021D7F80801B2
S315080302600CF029FBFFF7BEFA0023A7F8303125F077
S315080302707FF90346184625F0C7F997F82F31632BFC
S3150803028005D9012387F82E31002387F82F3197F8EC
S315080302902E31002B25D0002387F82E31FFF718FAC5
S315080302A0D7F80801FFF734F9FFF76AF9FBF79CFA61
S315080302B0D7F808010BF00AFD0346002B11D0D7F82F
S315080302C008010BF0B3FB0346002B05D00021D7F832
S315080302D008010BF083FB04E00121D7F808010BF0B2
S315080302E07DFBD7F82831B3F5967F05D3012387F825
S315080302F027310023C7F8283197F82731002B00F058
S31508030300A6800421D7F808010CF0B5F903469BB279
S315080303101946D7F808010CF00BFB0021D7F808019A
S315080303200CF0A9F980460121D7F808010CF0A3F9C6
S3150803033081460221D7F808010CF09DF904460321EA
S31508030340D7F808010CF097F905460421D7F80801F0
S315080303500CF091F90646D7F808010CF0DBFA0346C8
S315080303603B600521D7F808010CF085F9034607F128
S315080303700C0004933B6803930296019500944B463D
S315080303804246B44928F0FEF907F10C03184611F062
S31508030390C7F8D7F8D830C7F804310021D7F80801C9
S315080303A00CF069F90346C7F80031D7F8DC30C7F80B
S315080303B0FC300121D7F808010CF05DF90346C7F8AC
S315080303C0F830D7F8E030C7F8F4300221D7F8080137
S315080303D00CF051F90346C7F8F030D7F80421D7F8DB
S315080303E00031D31A002BB8BF5B42C82B13DCD7F8EE
S315080303F0FC20D7F8F830D31A002BB8BF5B42C82BBA
S3150803040009DCD7F8F420D7F8F030D31A002BB8BF95
S315080304105B42C82B10DDD7F808010CF01FF901461B
S3150803042007F1700368331822184628F0DCFA07F137
S315080304300C03184610F0A0FFFDF7AEFE25F098F85A
S315080304400346184625F008F9002387F82731D7F815
S31508030450203140F2DB52934205D9012387F81F3135
S315080304600023C7F8203197F81F31002B04D0002347
S3150803047087F81F3101F086FCD7F8183147F22F5257
S31508030480934205D9012387F817310023C7F8183192
S3150803049097F81731002B12D0D7F808010AF0D4F8C9
S315080304A00346002B06D0D7F808010AF0F1F90346EC
S315080304B0002B01D107F0ADFD002387F81731D7F8D4
S315080304C01031654A934205D9012387F80F31002372
S315080304D0C7F8103197F80F31002B7ED0002387F821
S315080304E00F31D7F808010AF00DFE0346002B03D097
S315080304F0D7F808010AF023FED7F808010AF031FEF7
S315080305000346002B03D0D7F808010AF047FEF3F792
S31508030510C5FA0446D7F8080109F0F6FA0346184659
S3150803052009F0A2FD03461D46D7F808010AF0EAFDBD
S31508030530034607F10C0000932B462246474928F049
S3150803054021F907F10C03184610F016FFF3F7A6FA7C
S315080305500446D7F8080109F0D7FA0346184609F0FE
S3150803056083FD03469C420ED9D7F8080109F0CCFA55
S315080305700446F3F793FA03469BB21946204609F055
S3150803058063FDF3F731F9F3F789FA0346B3F57A7F8F
S3150803059020D2D7F8080109F0B7FA0346184609F036
S315080305A068FF0346012B15D1D7F808010CF0CEFADC
S315080305B003461A4640F6AC539A420BD9D7F80801B4
S315080305C00CF08AFC0346002B04D10121D7F8080155
S315080305D00CF090FC0020F3F76DFA97F82F310133EE
S315080305E087F82F3197F83331013387F83331D7F842
S315080305F028310133C7F82831D7F820310133C7F832
S315080306002031D7F818310133C7F8183197F837313D
S31508030610013387F83731D7F810310133C7F810316A
S31508030620002000F03DF897F83731092B0ED9D7F893
S3150803063008010BF0FDFF0446D7F808010CF00EF885
S31508030640034606221946204611F08CFE0A2021F09D
S3150803065041FBA3E4CCD705083F7E050004D805086B
S3150803066080B500AF20F0D6FB00BF80BD80B483B051
S3150803067000AF03463960FB71FB7908493A6841F8CC
S315080306803320FB79054ADB0013443A685A60012391
S3150803069018460C37BD465DF8047B704750000020AA
S315080306A080B483B000AF0346FB71FA79FB79074937
S315080306B051F832200549DB000B445A6001231846DA
S315080306C00C37BD465DF8047B704700BF5000002019
S315080306D080B400AF034B01221A7000BFBD465DF814
S315080306E0047B7047A4D4002080B58CB008AF78602B
S315080306F07B68FB6007F1080100234FF40062F86882
S3150803070022F07EF80346002B01D002231AE0BB68C9
S31508030710B022069201220592002204920A2203922B
S315080307200A2202924FF40062019200930023074AB9
S315080307300749084822F0AAFA0346002B01D00E23DC
S3150803074000E0002318461037BD4680BD5907030845
S315080307501CD80508F4D3002080B58AB000AF7860AA
S31508030760002387F82730002387F8273030E097F8E7
S315080307702730214A52F833304FF6FF7293420AD094
S3150803078097F827201C49D3000B445B68591E1A485F
S31508030790D3000344596097F82730174ADB001344FC
S315080307A05B68002B0FD197F8272007F10803134935
S315080307B0184627F0E7FF07F10803184610F0DCFD93
S315080307C00F4B01221A7097F82730013387F8273021
S315080307D097F82730052BCAD9094B1B78002B03D06A
S315080307E0084810F0C9FD01E00EF00AF94FF47A70D3
S315080307F021F070FAB7E700BF5000002028D8050893
S31508030800A4D4002040D8050880B586B004AF0023D9
S315080308107B60342300221149114822F005F909F0B7
S31508030820E5F80346184609F06FF90346184609F032
S3150803083094F97860F3F712F802467B6802930192FB
S315080308404FF400430093074B4FF48042054906488B
S3150803085005F0E0F900BF0837BD4680BD4CD805084A
S31508030860A8D4002000040242DCD4002080B500AFDF
S31508030870024805F017FA0346184680BDDCD4002063
S3150803088080B582B000AF0346FB71FB79194604486D
S3150803089005F060FA034618460837BD4680BD00BF13
S315080308A0DCD4002080B500AF024805F0EBF9034617
S315080308B0184680BDDCD4002080B500AFF2F7CEFF22
S315080308C003461946024805F068FA00BF80BD00BF13
S315080308D0DCD4002080B58AB000AF00237B624FF4D6
S315080308E07A71104822F03EF90346002B06D10520FB
S315080308F0FFF7C6FF78620B4822F08EF9786AF2F79B
S31508030900B9FFFFF7D9FF381D7B6A0522064927F089
S3150803091039FF3B1D184610F02FFD00BF2837BD468B
S3150803092080BD00BFA8D4002064D8050880B584B06C
S3150803093000AF4FF00003BB604FF00003FB6040F6C7
S31508030940B831214822F00EF90346002B0BD10120BA
S31508030950FFF796FF07EE900AF8EEE77AC7ED037AF4
S31508030960194822F059F9F2F779FF07EE900AF8EEDB
S31508030970E77AC7ED017A09F039F80346184609F00C
S31508030980C3F80346184609F0E8F807EE900AF8EEA6
S31508030990E77AC7ED007A97ED037AD7ED017A77EE12
S315080309A0676A97ED007AC6EE877A9FED087A67EE4F
S315080309B0877AC7ED027ABB6807EE903AB0EE670A04
S315080309C01037BD4680BD00BFA8D4002000004843A9
